:020000041000EA
:10000000002008205D0100101301001015010010F0
:100010001101001011010010110100101101001058
:100020001101001011010010110100101701001042
:100030001101001011010010190100101B01001026
:100040001D0100101D0100101D0100101D010010F8
:100050001D0100101D0100101D0100101D010010E8
:100060001D0100101D0100101D0100101D010010D8
:100070001D0100101D0100101D0100101D010010C8
:100080001D0100101D0100101D0100101D010010B8
:100090001D0100101D0100101D0100101D010010A8
:1000A0001D0100101D0100101D0100101D01001098
:1000B0001D0100101D0100101D0100101D01001088
:1000C0001D0100101D0100101D0100101D01001078
:1000D0001D0100101D0100101D0100101D01001068
:1000E0001D0100101D0100101D0100101D01001058
:1000F0001D0100101D0100101D0100101D01001048
:100100001D0100101D0100101D0100101D01001037
:1001100000BE00BE00BE00BE00BE00BEEFF3058004
:10012000103800BEF2EB88710002001020020010AF
:10013000A801001090A31AE7D3DEFFFF42012110AF
:10014000FF010000E8090100793512AB4FF0000013
:100150002349086006C881F3088810474FF05040D3
:10016000006810B14FF00000F2E70FA40ECC002998
:1001700002D000F015F8F9E71A491B4A002000E008
:1001800001C19142FCD1002080F30A8817498847B9
:10019000174988471749884700BEFDE701C901C2D2
:1001A0009A42FBD3704700BF2002001010010020CC
:1001B000107300202074001010730020100A01201A
:1001C000200B01100000082000000820200B011067
:1001D00000100820001008200000000070470000F8
:1001E00008ED00E0100A012014400220713E0020BA
:0801F000090C0020693E00200B
:0801F800786B0010010000000B
:10020000B4060120C0060120CC060120D80601203A
:10021000E4060120F0060120FC0601204808012028
:10022000F8B500BF0348044B834202D0034B03B12F
:1002300018477047100A0120100A01200000000032
:10024000064B0749C91A891048BF0131491003D02C
:10025000044B0BB101481847704700BF100A01203A
:10026000100A01200000000010B5064C237843B9A5
:10027000FFF7D8FF044B13B10448AFF3008001230C
:10028000237010BD881401200000000010730020AE
:1002900008B5044B1BB104490448AFF30080BDE826
:1002A0000840CDE7000000008C14012010730020EE
:1002B0000120024A1368034413607047AC3F0120D9
:1002C0004078704700787047014B1878704700BF3E
:1002D0000D400220012A02D022B1002070470160A7
:1002E0000020704702600020704700BF034A0449A5
:1002F0001378087823F00203137070470F40022030
:100300000C400220012A02D022B100207047016077
:100310000020704702600020704700BF014B187832
:10032000704700BF0F400220012A02D022B10020F6
:10033000704701600020704702600020704700BFD6
:10034000014B1878704700BF0B400220012A02D0F1
:1003500022B1002070470160002070470260002039
:10036000704700BF012A02D022B10020704701600F
:100370000020704702600020704700BF704700BF38
:10038000012A02D022B1002070470160002070478E
:1003900002600020704700BF1378DA0709D54FF0DC
:1003A000000C094909480A7880F800C022F00102CF
:1003B0000A709B0707D50020034A05491378087087
:1003C00023F00203137070470F40022010400220F8
:1003D0000E400220012A02D022B1002070470160A5
:1003E0000020704702600020704700BF014B127868
:1003F0001A7070470B400220012A02D022B100205F
:10040000704701600020704702600020704700BF05
:10041000024B1078187003F021BF00BF0D4002207E
:10042000012A06D0022A0AD0032A00D022B10020D5
:1004300070470160002070470260002070470B6821
:1004400003600020704700BF012A06D0022A0AD0AC
:10045000032A00D022B100207047016000207047BD
:100460000260002070470B6803600020704700BFE7
:100470002DE9F041002386B088466E4600F5FF4224
:100480007832244F54002449E2B207EB021203935E
:1004900093689160D16802AD04930591CDF808800E
:1004A00095E8030086E8030092E80300DFF874C0D3
:1004B00085E8030096E80300C2F80CC082E8030058
:1004C0001BB10322294628469847621CD2B207EB8B
:1004D00002130022D9689C6805911049CDF8088064
:1004E00099600F4904940392D96095E8030086E867
:1004F000030093E8030085E8030096E8030083E81F
:1005000003001CB1032229462846A04706B0BDE8D7
:10051000F08100BF381601201103002039030020AC
:10052000B5010020B10100202DE9F043002406466A
:1005300087B008239046009422460F4606F07CFBC5
:1005400006F12F4505F560052D0D0635EDB2204667
:100550002946013400F07EFC082CF8D14FF0000948
:10056000234601244A4639463046CDF8009006F02D
:1005700063FB29461D2000F06DFC29461E2000F07B
:1005800069FC02231D2239460094304606F054FBD4
:1005900029461F2000F05EFC234639461F223046C4
:1005A000CDF8009006F048FB4FF48033114A0293D7
:1005B00008F1150305921B0308EB040243EAC2137A
:1005C00023F0FE4343F0F85303930B4B424604934E
:1005D000394602AB304606F075FB07EB470306EBE6
:1005E000C303C3F8D8803368BC401C43346007B0F1
:1005F000BDE8F0830074804000000C10F0B50025C9
:10060000284C83B00BE0D4F800249DF80710531C4D
:10061000B3F5806F28BF0023A154C4F80034012132
:100620000DF107008DF8075003F0A4FF0330EAD165
:1006300000271D4ED4F80054D6F8000405F5806C50
:10064000D4F80434AB4294BFEA1AACEB03021AB3F9
:10065000C3F30902A25CFAB1013A7D2A03F1010158
:1006600011D8E35CB1F5806F28BF00210A2B08BFC9
:100670000D2333540130B0F5806FC4F8041409D34E
:1006800001270020DCE7B1F5806F28BF0021C4F806
:100690000414D5E70127D3E70FB1C6F8000403B06F
:1006A000F0BD00BF80100120780C01200000000088
:1006B0002DE9F04FAB4893B003F012FE0122002465
:1006C000A94BAA4D1A70204655F8041F0134FFF7B4
:1006D000CFFE072CF7D147F6B52248F24B41A4488C
:1006E00003F080FEA34CA44EC4F5F545DFF8B892A4
:1006F000353505EB040814F8017FC32006F8017FA7
:1007000003F052FD4FEA182003F04EFD5FFA88F027
:1007100003F04AFD384603F047FDA145E9D147F60D
:10072000B5214FF00009954C9548B4F8BE5ACA4619
:100730006DBA11FA85F52A4603F054FE29460720C2
:10074000FFF796FE42F210738E4D0793A4F5E04337
:1007500008930DF13F0B8C4B8C491A788C4B8D48CC
:100760001B781A420B78027818BF43F001039A42B3
:100770000B7008D0162283F0010141EC40201922B1
:10078000037043EC4020FFF739FF7F4B19788A074D
:1007900019D4814BD3F80424D3F800349A4288BF8B
:1007A00003F580639B1A73B1774B41F00201197016
:1007B000531CB3F5806F28BF0023774977488A5CC4
:1007C000C1F80434027000234F464FF05046CDE983
:1007D0000A9A049300232B616B6813F48073FBD196
:1007E000286AB468A4B22146B26894B2A142FAD190
:1007F000002834DAB4F57F4F52D2089B1B5D99462E
:100800002B616B68DB05FCD48021D5F820804FEA92
:10081000142A049BC8F3806213F0806F18BFE02194
:1008200000230A4462F3070369F30F236AF31743B3
:1008300064F31F630F93C8203BBA0E9303F0B4FC1C
:100840000DF1370414F8010F03F0AEFCA345F9D104
:10085000079B01379F424AD0CDF81080BAE76B68FA
:1008600013F48073FBD1D5F82080B4F57F4FD2B25A
:100870004FEA142A5FFA88F94BD2089BC3200992E9
:1008800003F8049003F090FC504603F08DFC099AA5
:10089000104603F089FC484603F086FCA021B8E727
:1008A0003F49D2B201EB02190022D9F80880CDE904
:1008B0000E22CDE91022B8F1000F4FD00222494696
:1008C0000EA80993C047D9E90212099BCDE910127D
:1008D000002943D00D940DA90EA89047109B814686
:1008E0001BB10EA90322084698474B4688E741F200
:1008F0008833DDE90A9A0AF1010A09F51C599A457B
:1009000009F1100952D0079B03F51C5310330793CC
:1009100021E72449CDE90E3301EB0211CDE9103373
:100920008B68002BBAD002220EA80991984709992A
:10093000D1E90223CDE91023002AAFD00D940DF1A7
:1009400033020DA90EA88DF833909847109B002B09
:10095000A4D00EA90322084698479FE74FF000094C
:100960004EE700BFD07F0020064002206006012035
:10097000EC7F00201782002090BA0120DCAF01201C
:1009800018800020000020500F4002200540022067
:100990000B4002200A400220780C01200C4002206B
:1009A000381601203826012062060120484601F051
:1009B00057FF174B06461C6813A3D3E900230F46C5
:1009C00001F000FF4FF47A73CDE9040103FB04F05A
:1009D00001F058FF02460B463046394601F0F2FE60
:1009E000CDE90201204601F04DFF0022094B01F044
:1009F000E9FEDDE90423CDE90001074803F0F2FC3C
:100A00004FF0000A7FE700BF0000000080842E4105
:100A1000AC3F012000408F4048800020F8B5002402
:100A20000126254627460EE0132C15DD4FF0010365
:100A300043EC444043EC404006FA04F30134302CCC
:100A400045EA030512D0204600F036FA192CA4F12D
:100A50001D03E9DD012BE9D947EC44400022204683
:100A60000121013400F014FA302CECD12846F8BDF5
:100A700030B514234FF0000C4CEC40304FF47A703A
:100A80001E254FF001044FF01D0E164B0022196871
:100A900011440132642A1960F9D144EC405000221B
:100AA000196811440132642A1960F9D144EC40E01C
:100AB0000022196811440132642A1960F9D14CEC02
:100AC00040500022196811440132642A1960F9D19A
:100AD0004CEC40E00138D9D114234FF0010242EC34
:100AE000403030BD6C3B01202DE9F047074686B011
:100AF000492003F0B3FB00216D46754EFBB206EBB7
:100B00000312CDE90011734CD16873481F0193683B
:100B1000946002AC05910493D06092E8030084E8ED
:100B2000030095E8030082E803001BB1032221467D
:100B300020469847002207F1100906EB0903D968FF
:100B4000D3F80880059165490092996064496A600C
:100B5000CDF81080D96093E8030084E8030095E89D
:100B6000030083E80300B8F1000F03D003222146FD
:100B70002046C047002207F1200806EB0803D96889
:100B8000D3F808A0059157490092996056496A60C8
:100B9000CDF810A0D96093E8030084E8030095E83D
:100BA000030083E80300BAF1000F03D003222146BB
:100BB0002046D047002207F1300A06EB0A03D96825
:100BC0009E68059149490092996049496A60049676
:100BD000D96093E8030084E8030095E8030083E804
:100BE00003001EB1032221462046B0470022414E99
:100BF0000092F319D9689F6805916A603E493F4A9F
:100C000004979960DA6093E8030084E8030095E8AC
:100C1000030083E803001FB1032221462046B847A2
:100C20000022B144D9F80C10D9F8083005913449A4
:100C30000092C9F8081033496A600493C9F80C108F
:100C400099E8030084E8030095E8030089E80300BD
:100C50001BB103222146204698470022B044D8F811
:100C60000C10D8F80830059127490092C8F80810F0
:100C700026496A600493C8F80C1098E8030084E8D9
:100C8000030095E8030088E803001BB10322214616
:100C900020469847002206EB0A03D9689E68059112
:100CA0001B49009299601B496A600496D96093E8D9
:100CB000030084E8030095E8030083E803001EB105
:100CC000032221462046B04706B0BDE8F08700BFAA
:100CD00038160120C5010020B9010020F5010020CF
:100CE000DD010020190200200D0200203D0200203D
:100CF0003102002038260120550200200103002087
:100D0000710200206D020020C5020020890200202F
:100D1000E9020020DD0200202DE9F04188B02E48D4
:100D200007AB06AA05A901F00BFA18B92A492B4806
:100D300000F0E6F8DDE90612059801F03FF900241D
:100D400003F06CFD4FF00108FFF768FE244F1925F2
:100D500048EC4050C82000F089FF002646EC405087
:100D6000C82000F083FF21463846013403F03AFBE7
:100D7000032CECD11B4803F0B3FAFFF779FE1A48B5
:100D800003F0AEFA194805F03DFF1949174805F080
:100D9000BDFE314602461548FFF7C6FB154803F075
:100DA0009FFA4FF47F40FFF79FFE134806F02CF8A0
:100DB000124C00F0E1FD00F0E3FD11494FF47A72AE
:100DC0000023CDE90164009100F0C4FF40F2D2405D
:100DD00000F04CFFFAE700BF400D030060800020E8
:100DE000948000209C800020A080002000002050E3
:100DF00080060120A4800020A1050020100A012007
:100E0000A101002000220F4B03F58051C3E900220D
:100E1000C3E9022210338B42F8D100220A4B03F5BA
:100E20008051C3E90022C3E9022210339942F8D16C
:100E30000022002305480649C0E90023C1E9002338
:100E4000704700BF38160120382601208014012089
:100E50007810012010B44FF480740C4B53F820200C
:100E600003EB8003C00082F0400200F1804003F5F4
:100E7000805C02F0C00200F5203003F54053CCF84E
:100E8000002041601C605DF8044B70470480034003
:100E900010B4084CC90041EA820154F8202004EB48
:100EA0008003514003F5805301F00C015DF8044BC1
:100EB000196070470480034030B44FF0000343ECE6
:100EC000440043EC400005254FF480740B4BC200F6
:100ED00053F8201003EB800081F0400102F18043C1
:100EE00003F5203301F0C00200F5805100F54050B9
:100EF0000A605D60046030BC704700BF048003403E
:100F00000FB400B583B0049C074803F0E9F93CB185
:100F100005A92046019103F015F8044803F0E0F913
:100F2000012003F027F800BFA8800020B88000202F
:100F3000EFF3108072B6064BD3E8CF1F01220029D1
:100F4000FAD1C3E8412F0029F6D1BFF35F8F704774
:100F50001F3701200023034AC2E88F3F80F3108827
:100F6000704700BF1F37012070B58646EFF310852C
:100F700072B6124CD4E8CF6F0120002EFAD1C4E82B
:100F8000460F002EF6D1BFF35F8F4FF0010CC8085B
:100F900001F007030CFA03F31EF800C01CEA030675
:100FA00008D14CEA030C0EF800C0C4E88F6F85F33B
:100FB000108870BD1046FFF7A3FF00BF1F37012048
:100FC000F8B5EFF3108572B6234CD4E8CF7F012635
:100FD000002FFAD1C4E8476F002FF6D1BFF35F8F1F
:100FE0009A4227D80126D70810F807E002F0070C2C
:100FF00006FA0CFC1EEA0C0F00EBD2070DD125E01F
:101000004FEAD20E10F80EE002F0070C06FA0CFCC4
:101010001EEA0C0F00EBD20718D001329342EFD238
:101020004FF0FF300023C4E88F3F85F310889842CB
:1010300007DBF8BD0023C4E88F3F85F310884FF02D
:10104000FF300029F5D00698FFF75AFF4EEA0C0E44
:10105000104687F800E0E5E71F370120044A1078C2
:10106000431CDBB2182B28BF10231370704700BF3E
:101070001409012010B5054C82B001461F23182227
:1010800000940348FFF79CFF02B010BDBC80002015
:101090003C3B01204FF0E022936843F00053936003
:1010A000704700BF0021044B03F12002C3E88F1FEB
:1010B00001339342FAD17047143701204FF0E023F7
:1010C0004FF08032C3F80024C3F80424C3F8082486
:1010D000C3F80C24C3F81024C3F81424C3F818244C
:1010E000C3F81C24C3F82024C3F82424C3F82824FC
:1010F000C3F82C24C3F83024704700BF012300F04C
:101100001F029340400941B1800000F1604000F5AA
:101110006140C0F8803103607047024A203042F8D5
:101120002030704700E100E00123064A410952F8EF
:10113000212000F01F008340134214BF0120002033
:10114000704700BF00E100E001224309034900F0BD
:101150001F008240403341F82320704700E100E047
:10116000054A10309268054B52F82000C01A2F280B
:101170008CBF00200120704700ED00E0180901201D
:10118000F8B50D46EFF3108772B6124ED6E8CF2FA2
:101190000123002AFAD1C6E8423F002AF6D1BFF364
:1011A0005F8F0D4B00F110049B680C4A53F82430FC
:1011B000934203D0994201D001F094F9064B9B6809
:1011C00043F82450BFF35F8F0023C6E88F3F87F3B7
:1011D0001088F8BD1D37012000ED00E01D01001052
:1011E0002DE9F04F81468B46164683B0EFF310830E
:1011F00072B6DFF8D0A10093DAE8CF1F01230029EF
:10120000FAD1CAE8413F0029F6D1BFF35F8F664BA0
:1012100093F90040002CC0F2A080644D04EB440719
:1012200005EB870898F8061009F110091970604B52
:10123000BF009B6853F829006300411B2F292FD959
:101240005C49884240F0A4801C445B4B02372F4429
:10125000043BDB1BC3F34A036FEAC3434FF4214152
:101260006FEAD34325F8241005EB840463804BF622
:101270000153A380FF2348F00100E671C4F808B0D1
:10128000A3714B4B9B6843F82900BFF35F8F00238A
:10129000CAE88F3F009B83F3108803B0BDE8F08F4E
:1012A00020F0010E9EF80710B1422ED84FF42143D2
:1012B000EB53414BB91C2944043B04375B1A2F44C0
:1012C000AEF104013D4CC91BC1F34A012143A8F80A
:1012D0000410C3F34A033A492343A8F802304AF6FC
:1012E000AA2073465B1B5B415843000D88F80760DA
:1012F00088F80600C8F808B048F00100CEF80010E1
:10130000BFE7D179B1422ED996469EF906C00CEBC3
:101310004C02BCF1000F05EB8202F2DA4BF60151F0
:101320000EF10402A8F10407BF1AC7F34A076FEAD7
:10133000C7476FEAD7478EF8064003EB0408204CF6
:1013400005EB8803AEF8047045F82840998083F8CF
:1013500006C0DE71C3F808B093E701F0C3F8124B82
:1013600093F9004059E7724632F8041F490514D436
:101370004915023102EB410101916FF00701C91BD0
:10138000019F491B3944C1F34A0141F46041C9E757
:10139000019301F0A7F8019B56E701F5FF1101F554
:1013A000FF511F31E4E700BF04400220180901206B
:1013B00000ED00E01D0100104809012000E0FFFFE2
:1013C000014880471D370120F0B5EFF30585EDB2E8
:1013D000EFF3108C72B62649D1E8CF2F0123002AF3
:1013E000FAD1C1E8423F002AF6D1BFF35F8F214E08
:1013F00040F0010EB4684AF6AA2354F825701E4A3C
:101400000446A41A644163431B0D77455BB21BD0AD
:1014100092F906409C421CD092F912409C4223D083
:1014200092F91E409C4221D092F92A409C4208BF6A
:1014300003240FD0114A0024157813708571C1E878
:101440008F4F8CF31088F0BDB2680D4C42F82540E8
:10145000F0E7002404EB440402EB8402FF249471BF
:101460004BF601549480E5E70124F3E70224F1E709
:101470001D37012000ED00E0180901200440022082
:101480001D01001010B5074C82B001460523002253
:1014900000940548FFF794FD0028A8BFC0F1330071
:1014A00002B010BDD880002011400220014B0B4437
:1014B000036070471437012070B5104C104DAC42DA
:1014C0000ED2FF26236863B1FFF7C8FD0146204610
:1014D000FFF7ECFFA680BFF35F8F0834AC42F1D377
:1014E00070BDFFF7BBFD01462046FFF7DFFF267109
:1014F000BFF35F8F0834AC42E4D370BDB009012064
:10150000C009012010B50446FFF7A8FD014620469A
:10151000FFF7CCFFFF232371BFF35F8F10BD00BF28
:1015200010B504460120FFF7A5FD034B03442360DB
:10153000BFF35F8F10BD00BF14370120024B0B4477
:101540000360BFF35F8F7047143701200D4B1A689B
:10155000EFF3108172B6D2E8CFCF0120BCF1000FBB
:10156000F9D1C2E84C0FBCF1000FF4D1BFF35F8F8B
:1015700000221B68C3E88F2F81F3108840BF002032
:1015800000217047E43F02202DE9F04F2DED028B42
:1015900085B0EFF30583DBB2103B9A0818BF012238
:1015A0004FF0010103F0030018BFAF4DAF4B08BF70
:1015B000AF4D00EB820253F8226001FA00FB05F503
:1015C00041539FEDA78B0190C3F804B02EE0B38880
:1015D000180440F19280B379002B40F0DC80B6F91A
:1015E00008100029C0F21D81736901EB410103EB72
:1015F000C103D3E90247B7F1FF3F08BFB4F1FF3F92
:101600000DD0019B05EB8301AB6A0A69D21AE31A7C
:10161000934203D32B6A13EA0B0F00D10C612846C7
:1016200000F03AFCA042B941C0F2FB80B6F90830A4
:10163000C5F83CB0002B0093C9DBD6F8149003EB3F
:10164000430A284609EBCA07D7E9024800F024FC00
:10165000A04271EB0801BADBB8F1000FC0F2C38001
:10166000D7E90431834A934200F0ED807A88B6F9D5
:10167000080092B242EA0040984702460B4652EAFE
:10168000030100F0B080002B80F2D180B4EB020E99
:1016900068EB030839F93A30C7E902E8002B96DB1A
:1016A000716903EB430201EBC202D2E90270BE454D
:1016B00078EB000C4FEA430289DBB4462CF8083F74
:1016C0000BE031F93230A446002B0DDB03EB430075
:1016D00001EBC0005A00D0E90270BE451A4478EB15
:1016E000000001EBC204ECDA29F83A30009BACF8B8
:1016F0000030B38818043FF56EAF3369EFF3108202
:1017000072B6D3E8CF0F01210028FAD1C3E8401FF9
:101710000028F6D1BFF35F8F4FF6FF74B088002327
:10172000316900B2B480C1E88F3F82F310889842DB
:10173000FFF651AF0746A946746906F1080807EBA2
:10174000470E04EBCE03D3E90250B6F90830C44685
:10175000002B13DBB246009704E034F93630944690
:10176000002B09DB03EB430604EBC602D2E902714E
:10177000BD4270EB0101F0DA5646009FACF80070F4
:1017800034F93E7024F83E30002FD8DAB3794D4654
:10179000002B3FF424AF0023B371B6F9083006F1F3
:1017A0000808591C3DD01946776903E080465A1C49
:1017B0003FF417AF03EB430207EBC200B0F802C0DF
:1017C0001C461CF4004F9E4637F93230EED08C4256
:1017D00080ED028B05D0A8F80030318927F832104F
:1017E00034817146E3E739F83A3033813369EFF3F6
:1017F000108272B6D3E8CF0F01210028FAD1C3E8D6
:10180000401F0028F6D1BFF35F8F7388316929F834
:101810003A30009B73800023C1E88F3F82F3108829
:10182000D5E640BF05B0BDEC028BBDE8F08F284681
:10183000CDE9022300F030FB029A039B10EB020E6D
:1018400043EB010826E708460B69029198470028F8
:10185000C9D00299D1E9002311E700BFAFF300809E
:10186000FFFFFFFFFFFFFFFF00800B40BC3F012099
:1018700000000B40791400202DE9F84F364C256903
:101880002DB1BDE8F84F0A213448FFF70FBEDFF84D
:10189000E4800321404600F0EDFA0326C4F80C80F2
:1018A000FFF7DCFB4FF0504C2D4B267003442361B7
:1018B000DCF800300F216370636961801D834FF095
:1018C0000405A3F878504FF00505A3F890504FF0A9
:1018D0000605A3F8A8504FF007050E214FF6FF723A
:1018E00008274FF00A0EA3F8C0504FF001094FF03F
:1018F0000C0C4FF0020B4FF0090A0D204FF00B05B6
:10190000A3F868111749A280A3F808E1A160A3F821
:1019100048B0A3F8F0A0A3F82051A3F838C1A3F869
:101920005001A3F83090A3F86060A3F8D8701A8033
:101930000D4B3046C8F820700C49DC60FFF720FCE6
:1019400049463046FFF7DAFB094B0A211F6403487A
:10195000BDE8F84FFFF7AABD60090120E43F02206F
:1019600014370120FFFF1000BC3F01207914002034
:1019700000200B4000000B4008B5FFF77DFF08BDBD
:101980000048704760090120F8B59DF820700446B2
:1019900016461D4637B900F087FA864265EB01010D
:1019A00000295CDB2369EFF3108772B6D3E8CF1F01
:1019B00001220029FAD1C3E8412F0029F6D1BFF353
:1019C0005F8FB4F902C063690CEB4C01BCF1000FEE
:1019D0004FEAC10203EBC10138DB985A4FF0000E09
:1019E00060802069C0E88FEF87F310880698C1E90E
:1019F000026508610798486148880130C0F30E000D
:101A0000012838BF0120488040EA0C402169EFF3EB
:101A1000108572B6D1E8CF7F0126002FFAD1C1E838
:101A2000476F002FF6D1BFF35F8FA1889952A4F8BA
:101A300004C02369C3E88FEF85F310880122E368AF
:101A4000217803F501538A405A60F8BD00232269CA
:101A5000C2E88F3F87F310884FF0FF30F8BD38465B
:101A6000F8BD00BF0146F0B50069EFF3108772B60C
:101A7000D0E8CF5F0124002DFAD1C0E8454F002DFA
:101A8000F6D1BFF35F8FB1F902E04C690EEB4E0C5B
:101A9000BEF1000F4FEACC0504EBCC0C3DDB605BE4
:101AA000002648800869C0E88F6F87F31088BCF86B
:101AB0000200CCE902230130C0F30E00012838BF38
:101AC0000120059BACF80200CCF81030069B40EAE0
:101AD0000E40CCF814300B69EFF3108272B6D3E8E5
:101AE000CFCF0127BCF1000FF9D1C3E84C7FBCF187
:101AF000000FF4D1BFF35F8F8B886353A1F804E02C
:101B00000B69C3E88F6F82F310880122CB680978D4
:101B100003F501538A405A60F0BD00230A69C2E808
:101B20008F3F87F310884FF0FF30F0BD03464089A8
:101B3000B0EB214F37DD58690A1402EB420210B5B1
:101B400000EBC2001C69EFF3108C72B6D4E8CFEF43
:101B50000122BEF1000FF9D1C4E84E2FBEF1000FF3
:101B6000F4D1BFF35F8F428889B292B28A4207D024
:101B700000221B69C3E88F2F8CF31088002010BD52
:101B800042F4004242800121002218699971C0E8A4
:101B90008F2F8CF310881C78DA68084602F5015301
:101BA000A140596010BD0020704700BF40787047C9
:101BB0002DE9F041861F41F1FF35B04271EB05037D
:101BC00038BF002682B038BF354604460F4600F0C5
:101BD0006BF9301A65EB0103012873F1000306DA93
:101BE0002046394602B0BDE8F04100F067B900F088
:101BF0005BF9864265EB010100290ADB0021174BE6
:101C00003246009316482B460191FFF72BFF002820
:101C1000E6DB4FF0000C1348134A436A9D4204D898
:101C2000816AB142DCD29D42DAD11368EFF31081B0
:101C300072B6D3E8CF8F5FF0010EB8F1000FF8D184
:101C4000C3E848EFB8F1000FF3D1BFF35F8F13681B
:101C5000C3E88FCF81F3108820BFDEE73D1400205A
:101C60006009012000000B40E43F022010B504464B
:101C700000F01AF94FF47A734FF0FF3C6FF0004216
:101C8000E4FB0301BDE81040844572EB01033CBF57
:101C900060461146FFF78CBF2DE9F04306460D461E
:101CA00083B0EFF30584E4B23CB1274B586AA842F5
:101CB0001CD2002003B0BDE8F083244FD7F80C906D
:101CC00097F80080484600F0E7F808F1040859F852
:101CD00028301B1A301A65EB0101984271F100019E
:101CE00011DB20BF184B586AA842E2D39B6AB3426B
:101CF00003D3012003B0BDE8F083401B18BF0120CF
:101D000003B0BDE8F08300F0CFF8864265EB010137
:101D10000029CADB0E4B3846CDE9003432462B464B
:101D2000FFF7A0FE011EC0DD074B5A6AAA4208D386
:101D30009B6AB34203D30548FFF7F8FEB5E7AA4212
:101D4000F9D120BFF7E700BF00000B406009012078
:101D50003D1400202DE9F0410446DDE9071552EA63
:101D6000030070D0002B16461F4671DB0698C5E9AC
:101D700000232861AC60696100F096F84FF0FF32F3
:101D80006FF00043801947EB0107824273EB0701B4
:101D90003CBF1F4610462369EFF3108872B6D3E8A4
:101DA000CF1F01220029FAD1C3E8412F0029F6D123
:101DB000BFF35F8FB4F90260616906EB4603002E42
:101DC0004FEAC30C01EBC30346DB31F80C204FF0A4
:101DD000000E62802269C2E88FEF88F310885A886B
:101DE000C3E902070132C2F30E02012A38BF012201
:101DF0001F485A805D61186142EA06422369EFF389
:101E0000108072B6D3E8CF8F0127B8F1000FF9D157
:101E1000C3E8487FB8F1000FF4D1BFF35F8FA38808
:101E200021F80C30A6802369C3E88FEF80F3108877
:101E300001202178E36800FA01F103F501535960AC
:101E4000EA60BDE8F0810126002732463B468DE777
:101E5000564263EB430789E700202369C3E88F0FED
:101E600088F310884FF0FF32EA60BDE8F08100BFD0
:101E70007914002010B4054B054C064AA04214BF4B
:101E80001846581C5DF8044BFFF76EB8403B012024
:101E900000800B40F48000200346416A0A46986A9D
:101EA000596A8A42FAD17047034B596A0A46986ABE
:101EB000596A9142FAD1704700000B40074A536AB1
:101EC0009942FCD8994207D1044B02E05A6A9142E8
:101ED00002D19A6A8242F9D3704700BF00000B40DA
:101EE00000EB400C4FEA8C0C0CF1804C0CF5803C64
:101EF000F0B51646DCF80420051FB2F5803F38BF68
:101F00004FF48032EDB238BFCCF80420012D2AD92D
:101F10004FF40067254C0CF54052176054F8202010
:101F2000B2B9DCF80020012D82EA461202F0E0028C
:101F30000CF5805632602AD94FF4006144F8203005
:101F40004FF480330CF500521160CCF80430F0BD32
:101F50006769B7FBF2FE0EF1010E0EEB4E0EBEF1FD
:101F6000030EFCD2DDE70129D2D103240CF5405247
:101F70001460DCF80820D207FBD5DCF800200B4CFD
:101F800082EA461202F0E0020CF58056326001222D
:101F9000DCF800504D4005F00305356002FA01F110
:101FA000DCF808200A42FBD0C6E700BF443B012012
:101FB000014B53F820007047443B0120584B2DE95A
:101FC000F0431C6C1746B4F5803F38BF4FF48032A5
:101FD0000E464FF00301804638BF1A64514A504BF9
:101FE00083B0D1635C6CE507FCD5DA6B4E4982F0B7
:101FF000200202F0E002CA63DB6B494D83F001036B
:1020000003F00303CB636C6CA407FCD54FF40062B0
:102010004FF48039454B464CDA63464B4246636188
:1020200001213346C5F840904348009700F056F927
:102030004FF400616B6B07FB06F64B4538BFC5F8E4
:102040003490384B2269B8FBF6F619633AB16369EC
:10205000B3FBF2F3013303EB4303033BFDD2304BFD
:1020600031491A6B02F0E0020A631A6B82F0020235
:1020700002F003020A63996B4807FCD54FF4006530
:102080004FF4803229490D632C495A632161196C40
:1020900091424FF0030138BF1A64224B204AD963A2
:1020A000536CD907FCD5D36B1F4D03F0E003EB63F2
:1020B000D36B1B4983F0010303F00303EB634B6C09
:1020C0009B07FCD54FF480334FF40065174A6661D7
:1020D000D5630B64CA6C9A4238BFCB644FF400617D
:1020E000104BA26999643AB16369B3FBF2F301330F
:1020F00003EB4303033BFDD24FF400604FF4803108
:10210000074A094D936C83F0400303F0E003AB648E
:10211000064B084DA5619864D16403B0BDE8F08317
:10212000000001400030014000100140002001404B
:10213000443B0120006CDC0200000540001BB7009E
:102140002DE9F04F4FF4A078994685B0CDE9021201
:102150005F4CDFF884A154450AD908F1FF38A4F593
:102160003B54B8F10F0FA4F12004F4D1002069E032
:10217000072304F53722019403FB03F402F5D87218
:10218000B2FBF4FE70454FF0010C4FF002074FF028
:1021900003064FF004054FF005013FD0B3F1010EE7
:1021A00000F094800EFB03F4B2FBF4FB58454CD0D6
:1021B00019B301FB03F4B2FBF4FB58454FD0E5B172
:1021C00005FB03F4B2FBF4FB584553D0AEB106FB5C
:1021D00003F4B2FBF4FB584557D077B107FB03F487
:1021E000B2FBF4FB58455BD0BCF1000F05D00CFBF3
:1021F00003F4B2FBF4FB83455DD0734603FB03F4A9
:10220000B2FBF4FE704501F1FF3105F1FF3506F137
:10221000FF3607F1FF370CF1FF3CBFD104FB102460
:10222000002CBBD19E464A46DDF808B0DDF80C9084
:102230000120284901FB08F1CBF80010C9F8003053
:10224000C2F800E005B0BDE8F08F04FB1024002CBC
:10225000AED14A46DDF808B0DDF80C90E8E704FBA3
:102260001024002CABD14A468E46DDF808B0DDF8CC
:102270000C90DDE704FB1024002CA7D14A46AE46A3
:10228000DDF808B0DDF80C90D2E704FB1024002C38
:10229000A3D14A46B646DDF808B0DDF80C90C7E792
:1022A00004FB1024002C9FD14A46BE46DDF808B03E
:1022B000DDF80C90BCE704FB1024002C9DD14A46AD
:1022C000E646DDF808B0DDF80C90B1E7019C44E784
:1022D00050262F00001BB70050F80C0070B4039D6F
:1022E00004682D0345EA03451B4B002CB3FBF1F3B7
:1022F000B2FBF3F61FDB194A194B904214BF4FF49F
:1023000080424FF40042174C1A6003F580531A6064
:10231000A36832EA0303FBD1212200F540530433C2
:10232000016086601A600268002AFCDA0822C56033
:102330001A6070BC7047036803F03F038B42DAD128
:102340008368C3F30B03B342D5D1C36803F4EE2310
:10235000AB42D0D1EDE700BF001BB70000800540C5
:10236000002002400000024030B44FF080441C4B7B
:102370001C60E0B11B4CA3F54053DC611A4C40F0EB
:10238000010044401C62596298624FF080454FF052
:10239000E061134B1548164C1D60846019604AB902
:1023A00030BC4FF00042A3F580531A607047114BC8
:1023B000D861EAE74FF47A7303FB02F2B2F1807F4F
:1023C0002ABF6FF07F4313461A464FF080410A4CF4
:1023D00008482360094B426030BC1960704700BF59
:1023E00000B00D40D3C007B02D3FF84F00A0014012
:1023F000F3FFFF0100800D40A83F012000A00D4029
:10240000012300EB4000800000F1804000F58410C3
:1024100041600360704700BF002370B5DB8A04464B
:102420000D46002242E800F2520254BF102104215E
:1024300044F25220984786462B462246F446BDE891
:1024400070400A214FF48170604700BF0023DB8A8F
:10245000002242E800F2520201D410211847042160
:10246000184700BF08B503460846191E02DB1AB11B
:1024700040F03000FFF7D0FF40F02000FAE700BF47
:10248000034AD2F82838002BFBD0BFF35F8F704788
:1024900000000E400021044B044ABFF35F8F43F855
:1024A000041B9342F9D170470C080E402C080E40D3
:1024B00010B44FF48D704FF42A64064A064B074956
:1024C0001460D06019605368002BFCDA5DF8044B8F
:1024D000704700BF0080044000A0044000B0FA0034
:1024E000704700BF08B50148FEF70AFD18810020BB
:1024F00038B5054C054DAC4204D254F8043B98471E
:10250000AC42FAD338BD00BFC0090120000A012047
:1025100038B5054C054DAC4204D254F8043B9847FD
:10252000AC42FAD338BD00BFEC090120000A0120FB
:1025300010B40748074C084B084A094904601A6060
:102540008B6832EA0303FBD15DF8044B704700BF90
:10255000002002407F3BEFEF00300240F6FFF30324
:1025600000000240044BDB6CB3F5004F03D14FF485
:102570008022024BDA647047000011500020115095
:102580004FF0E022044BD2F8881D0B43C2F8883D7F
:1025900010EE3004704700BF030330006FF060415D
:1025A000044B054A19609368DB4333F06043FAD16A
:1025B000704700BF003002400000024010B545F2F5
:1025C0005320FFF743FFBDE810400346042018479F
:1025D00010B545F25320FFF739FFBDE81040034620
:1025E00001201847FEF75EBD10B5054B054C4FF4B2
:1025F00088721846A16804F017FEA06010BD00BFE5
:102600000000002000ED00E0002370B52B4C82B0EC
:10261000C4F88430FFF74CFF0122294BDA63636C66
:10262000012BFCD10321264A244B11639C6B012C06
:10263000FCD10226052521460523224A2248009680
:10264000FFF74CFE21462B46204A21480095FFF714
:1026500045FE0022042031461E4BFFF741FC214677
:10266000284600221C4BFFF73BFC002208201146A5
:102670001A4BFFF735FC002209201146174BFFF7D4
:102680002FFC002206201146134BFFF729FC0022E5
:10269000114B07201146FFF723FC0420FFF788FCAD
:1026A00000240F4BA3FB0035AD0CE0B229460134EA
:1026B000FFF7A6FE062CF8D102B070BD0000014065
:1026C00000300140002F685900000540008C86470B
:1026D00000800540001BB70080D1F008006CDC02D0
:1026E00083DE1B4386B003B451FC0804CDE902012C
:1026F00051FC0904CDE9040151EC0A04CDE90601BD
:1027000003BCF047BDE800504EEC00C4BDE80050EB
:102710004EEC01C4BDE800504EEC02C400BD000008
:1027200000B5FFF7DFFF02E010FE30F4F8D441EC13
:10273000100443EC112400EE010410EE010480EEBD
:10274000200451EC1004704700B5FFF7CBFF02E006
:1027500010FE30F4F8D441EC100443EC112400EEE8
:10276000010410EE210480EE200451EC3004704787
:1027700000B5FFF7B7FF02E010FE30F4F8D410B553
:1027800041EC100443EC112451EC040453EC0524F7
:10279000A0FB024C5FF0000EE0FB03CEE1FB02CE9B
:1027A0004CEC20440024E1FB03E444EC30E480EEF4
:1027B000200451EC5004BDE81040704700B5FFF70D
:1027C00091FF02E010FE30F4F8D441EC100443EC29
:1027D000112451EC2104A0FB01126FEA820252FB8A
:1027E000100052FB12F252FB1000A0EBD07C53EC15
:1027F00004245CFB13F153EC1524A1FB022001FB24
:10280000030053EC4424A2EB000050FB1CF24FEAFF
:10281000111312EB017043EBE27140EA515020EAD0
:10282000915020F0070053EC7524A0FB023C53ECC0
:10283000752400FB03CC01FB02CC53EC0424ACEB6D
:10284000824C40EA5C70A0F1010041EC400480EE53
:10285000200451EC7004704700B5FFF743FF02E01D
:1028600010FE30F4F8D440EC700400EE010410EED9
:10287000210480EE200451EC3004704700B5FFF7CE
:1028800031FF02E010FE30F4F8D440EC600400EEBA
:10289000010410EE210480EE200451EC3004704756
:1028A00000B5FFF71FFF02E010FE30F4F8D441EC52
:1028B000800400EE010410EE010480EE400410EEEE
:1028C0001304704700B5FFF70DFF02E010FE30F46F
:1028D000F8D441EC800400EE010410EE010480EE17
:1028E000400410EE3304704700B5FFF7FBFE02E032
:1028F00010FE30F4F8D441EC100443EC112400EE47
:10290000010410EE3004C0F30070704700B5FFF70B
:10291000E9FE02E010FE30F4F8D443EC102441EC60
:10292000110400EE010410EE30F48CBF01200020F1
:10293000704700BF00B5FFF7D5FE02E010FE30F48F
:10294000F8D441EC100443EC112400EE010410EE25
:1029500030F42CBF01200020704700BF00B5FFF706
:10296000C1FE02E010FE30F4F8D441EC100443EC58
:10297000112400EE010410EE30F48CBF0120002081
:10298000704700BF704700BF2DE9F04F83B09946F4
:10299000DDE90DAB0F9B884611469A07074616D115
:1029A000DA453AD20C460D46ABEB0A060E442246F7
:1029B0004B46414620200134B847B442F7D129465E
:1029C000BAF1000F08D1204603B0BDE8F08F0C46E5
:1029D000BAF1000F10D00E4655460C9B2E449A4477
:1029E0000191721B4B46013D41461AF8010D3446D8
:1029F000B847002DF5D101990F9B9B07E3D5651AC8
:102A0000AB45E0D922464B46414620200135B84728
:102A10005D4504F10104F5D3D5E7BAF1000FDAD131
:102A20000C46D0E72DE9F04F0F9FDDF824E017F0BA
:102A3000020F0A9C9DF82C900E9DDDE90C8629D191
:102A4000002D6FD1B44225D2202C07F0010B00F0ED
:102A5000128104F1FF3C4FF0300AF44401E0202CD5
:102A60007AD00134A6420CF801AFF8D8BBF1000FC0
:102A700010D0AC420ED2202C74D004F1FF3C4FF0A9
:102A8000300AF44401E0202C29D00134AC420CF887
:102A900001AFF8D117F0100F3AD017F4806F28D19A
:102AA0001CBBB8F1100F00F0CA80B8F1020F00F0A3
:102AB000D48030248EF800400124B9F1000F67D192
:102AC0007E0740F1AA802B260EF804600134CDE980
:102AD0000B57CDE909E4BDE8F04FFFF755BFFC0601
:102AE00040F189807C0535D42024A6426AD0AC42CE
:102AF00068D0B8F1100F00F08780B8F1020F5AD0FB
:102B0000202CE4D0264601344FF0300C0EF806C0DD
:102B1000202CD2D1CDE90B57CDE909E4BDE8F04F27
:102B2000FFF732BF17F0010B3ED0B9F1000F47D1CC
:102B300017F00C0F44D1B4429BD2202C89D1202D08
:102B400010D8FC0657D57C0555D4202E00F0B9804E
:102B5000202D10D02024CCE7BBF1000F00F0A58081
:102B6000202DBCD9FC0646D57C0544D4202E00F08F
:102B7000A880202D3FD12C461F26B8F1100F7FD002
:102B8000B8F1020FC0D14FF0620C0EF806C0B7E7E3
:102B90002D260EF804600134CDE90B57CDE909E488
:102BA000BDE8F04FFFF7F0BEB442BFF473AF202C86
:102BB0007FF44FAFD6E7202C89D026460134E2E7D8
:102BC000013DB8E7661ED8D1B8F1100F64D0B8F156
:102BD000020F7FF46EAF62268EF800603026444606
:102BE0008EF80160B9F1000F3FF46AAFD0E7B8F199
:102BF000100F7FF46CAF2024CDE90B57CDE909E429
:102C0000BDE8F04FFFF7C0BEBE060ED4202CF2D0B8
:102C100078260EF80460013472E73E077FF557AF5F
:102C200020260EF80460013451E7202CE3D04FF049
:102C3000580C0EEB040686F800C0013460E7BE06AF
:102C400017D558248EF8004030248EF80140022415
:102C5000B9F1000F3FF434AF9AE762248EF80040D8
:102C600030248EF801400224B9F1000F3FF428AF60
:102C70008EE77824F2E7BBF1000F7FF462AF71E7D3
:102C800017F0200F0CBF4FF0780C4FF0580CA61E19
:102C90000EF806C0013C35E7BC06EAD558248EF88C
:102CA000004030248EF80140DDE717F0100F3FF4AC
:102CB0000EAF17F4806F9AD1202E7FF418AF1F2625
:102CC0005BE734461F2658E700B9704701F0C6BAE3
:102CD00010B1D1E900311847704700BF0000000073
:102CE0002DE9F04F9FB09DED287BDDE92AA558EC3A
:102CF000177B83461E460D91109243463A4638464E
:102D000041468DED087B2C9CFFF7F2FD002840F03A
:102D1000D880384641464FF0FF32754BFFF722FE10
:102D2000002840F0CE80384641464FF0FF326FF425
:102D30008013FFF7EFFD002840F0C380DDE908783D
:102D40000022384641460023FFF7E4FD002840F00A
:102D5000C081CDE90A78DDE90A2390461F4614F4C4
:102D6000806308BF4FF0060A139304F4006258EA28
:102D70000703119240F0C080002A00F0A2819FED6D
:102D80005A7B00278DED0E7B4FF00009BA45CCBF72
:102D9000AAEB070A4FF0000A4F46C8BF0AF1FF3AF4
:102DA00044F480644D4594BF4FF00008A5EB09083A
:102DB00014F00203119304D0B9F1000F18BF4FF0C3
:102DC00000083FB1DDE90A01DDE90E23FFF7FAFC57
:102DD000CDE90A01DDE9080100220023FFF79AFD91
:102DE00030B1DDE90A01024601F10043CDE90A23D1
:102DF0009DED0A7BCDE902A8DDF834A024F4006340
:102E000004938DED007B334651465846109A00F0EE
:102E100097F98046B9F1000F4FD014F0200F024609
:102E200000F1010433460CBF652045205146D847C8
:102E300009F1FF3087EAE77C0DF1580900224B4683
:102E4000DFF8B080ACEBE77C4FEAD77E01E0202AC8
:102E500010D0E246A8FB0C71C90801EB8107ACEB6E
:102E600047073037BAF1090F8C4602F1010203F827
:102E7000017BECD805230590069300200A230D9FC3
:102E8000CDE90330CDE9012E334622463946584676
:102E9000CDF80090FFF7C6FD119B80466BB1109BEB
:102EA000C41AA54209D94246334639462020013486
:102EB000D847A54208F10108F5D840461FB0BDE843
:102EC000F08F9DED087B33465846109A0D998DED95
:102ED000287BCDE92B54CDF8A8A01FB0BDE8F04F5A
:102EE00000F02EB9AFF300800000000000000000E9
:102EF000FFFFEF7FCDCCCCCCC7F30A50A0F2FF3060
:102F0000FFF7AEFC8AA3D3E90023FFF735FC8AA3C1
:102F1000D3E90023FFF708FCC7F31307CDE90E013F
:102F200047F07F51404600227B4B41F44011FFF7B0
:102F30000FFC6BA3D3E90023FFF71EFC02460B46F0
:102F4000DDE90E01FFF7F0FBFFF7AEFC0746FFF7E8
:102F500087FC65A3D3E9002380468946FFF70CFC74
:102F600000226E4BFFF7E0FBFFF79EFC034649464D
:102F7000404612935EA3D3E90023FFF7FDFB804692
:102F800012988946FFF76CFC5BA3D3E90023FFF797
:102F9000F3FB02460B4640464946FFF7D9FB024683
:102FA0000B4680468946FFF7E7FB42464B46CDE994
:102FB0000E0140464946FFF7B7FB0022CDE9140158
:102FC000DDE90E01564BFFF7FDFB0022554BFFF7E5
:102FD000ABFB02460B46DDE90E01FFF7F3FB0022D7
:102FE000514BFFF7A1FB02460B46DDE90E01FFF74F
:102FF000E9FB42464B468046894600204FF080411F
:10300000FFF7A6FB02460B4640464946FFF78CFBFE
:1030100002460B46DDE91401FFF7D4FB0022434BC7
:10302000FFF782FB129B002203F2FF3C4FEA0C5396
:10303000FFF7A2FB80468946DDE90A0142464B467E
:10304000CDE90E89FFF766FC68BB4346494607F1A8
:103050006302C62A119A8CBF4FF005094FF004098C
:10306000002A3FF49FAE0B433FF48EAEDDE90A0128
:1030700023A3D3E90023FFF761FC48B1DDE90A018E
:1030800021A3D3E90023FFF745FC00287FF47CAEA1
:10309000BAF1000F3FF486AE139B002B3FF482AED3
:1030A0000AF1FF3A7EE600221E4B40464946FFF7F2
:1030B00089FB0A4601460346CDE90E12013F11463F
:1030C000C5E79FED137B17464FF004098DED0E7B8E
:1030D00068E608F100430A970B933CE6AFF30080E3
:1030E00061436F63A787D23F71A379094F930A4069
:1030F0001655B5BBB16B0240EF39FAFE422EE63FE2
:103100002D431CEBE2361A3F0000000080842E4164
:1031100000000000000000000000F83F0000E03F59
:1031200000002C4000002440000018400000F03F48
:10313000FB799F501344D33FB3C8608B288AC63FA6
:103140002DE9F04F97B0DDE92089CDE90401DDE9F3
:10315000224BCDE90623404642464B464946DDF820
:1031600090A0FFF7C5FB002840F0C58140464946C6
:103170004FF0FF326FF48013FFF7CCFB002840F0D4
:103180001D81404649464FF0FF32C14BFFF7EAFB35
:10319000002840F0E380B8A3D3E900234046494625
:1031A000FFF7E0FB002840F0CB80B5A3D3E9002374
:1031B00040464946FFF7AEFB002840F0C18040463C
:1031C000494600220023FFF7A5FB002840F0E080DD
:1031D0001AF480650D9000F0E980092C40F2968188
:1031E0000EAB1A460C9330210023A4F109050133DC
:1031F000202B02F8011BA4EB030600F03A81AB423E
:10320000F5D19FED9D7B8DED087B49464046FFF74C
:103210004BFB0446FFF724FB02460B46404649465B
:10322000FFF796FADDE90823FFF7A6FA02460B46F8
:10323000CDE90A23FFF74AFB0746FFF723FB0246C7
:103240000B46DDE90A01FFF783FA02460B46CDE99A
:103250000A2300228F4BFFF785FB002800F0DB805C
:1032600001373846FFF70EFBDDE90823FFF766FB61
:1032700008B100270134002E40F0B1802046FFF74E
:10328000EFFA02460B4640464946FFF761FA002234
:10329000804B06460F46FFF73DFB40B930463946A6
:1032A00000227C4BFFF75EFB002800F015810C9B91
:1032B000691E7948194410E080FB0462C3EBA20345
:1032C00003EB8302A4EB420404F1300201351C46F7
:1032D00001F8012F002B00F0AB80202D4FEAE473A2
:1032E000EAD10AF00303012B1CD1BBF1000F19D066
:1032F0000D9B002B40F0F9801AF00C0F40F0F58088
:10330000AB4540F2D380202D0BD030220C996B1EA0
:103310000B4401355D4503F8012F00F08D80202D11
:10332000F7D12025DDE90623DDE904010C9CCDE978
:1033300002BA01950094FFF727FB17B0BDE8F08FA4
:10334000CDE92089DDE90623DDE90401CDE923BAD1
:10335000229417B0BDE8F04FFFF7C2BC4F4DCDF837
:103360008CA00AF0040ABAF1000F4D4C18BF2C468D
:10337000DDE90623DDE9040120940CBF03240424C5
:10338000CDF888B0219417B0BDE8F04FFFF7FCBA34
:103390004B46424600200021FFF7DAF901231AF4D8
:1033A0008065804689460D937FF417AF9FED367B8D
:1033B0000EAB06268DED087B0C9326E70424DDE991
:1033C0000623DDE90401374DCDF88CA0CDF888B097
:1033D0002095219417B0BDE8F04FFFF7D5BA0C9BAC
:1033E000681EDFF8C4C018440DE0ACFB0721C90813
:1033F00001EB8102A7EB42023032092F00F8012FC6
:1034000027D90F461D46202D05F1010306F1FF3691
:10341000EBD120254BE70022DDE90A011D4BFFF728
:1034200079FA00287FF427AF002F5AD1013722E71D
:103430000AF00303012B75D0202D3FF473AF0D9BD1
:10344000BBB32D2205F158036B4403F8202C013542
:1034500068E7202BDDD0AEB30C9A1E441544302211
:1034600001E0B3422ED00133202B05F8012FF8D113
:10347000CFE71D46C5E600BF0000000065CDCD4189
:103480000000000065CDCDC10000000080842E4109
:10349000FFFFEF7F0000E03F676666666481002003
:1034A0006C81002074810020CDCCCCCC202D3FF449
:1034B00039AF1AF0040F0DD11AF0080F3FF432AFF4
:1034C0002022BFE72E2103F158026A4402F8201C93
:1034D0005D1CECE62B22B5E7E3077FF5E8AE01348F
:1034E000E5E6FA077FF5C7AEA0E70BF1FF3BAB457A
:1034F0003FF609AFA0E70324DDE90623DDE9040177
:103500000A4DCDF88CA0CDF888B061E7084B26466F
:1035100003EBC40393ED007B0EAB8DED087B002520
:103520000C9372E6BBF1000F86D0E1E670810020BB
:10353000080701202DE9F04F9A469BB0249C964D38
:103540000B94964C0B1E18BF834625609AF800001A
:10355000934C0A9308BFA3460992002800F0BC824E
:103560004FF000090AE04A46099B0A9909F101094E
:10357000D8479AF80000002800F0CE8025280AF1EC
:10358000010AF0D10023524612F8010BA0F12001EC
:1035900010290AD8DFE801F04009093C09090909A6
:1035A00009090938093409093000A0F13001092955
:1035B00040F28C802A2800F0F58000210C912E2802
:1035C00000F099800027A0F1680112292DD8DFE8CA
:1035D00011F057012C0051012C0045012C002C004A
:1035E0002C002C002C002C002C0027002C002C0080
:1035F0002C002C002C002700924643F00103C2E768
:10360000924643F00203BEE7924643F00403BAE752
:10361000924643F01003B6E7924643F00803B2E740
:103620009AF8010043F4807301326728924600F251
:103630008280242840F2C680A0F12502422A00F2AE
:10364000C180DFE812F05F01BF00BF00BF00BF0014
:10365000BF00BF00BF00BF00BF00BF00BF00BF0072
:10366000BF00BF00BF00BF00BF00BF00BF00BF0062
:10367000BF00BF00BF00BF00BF00BF00BF00BF0052
:10368000BF00BF00BF00260145012601BF00BF00EB
:10369000BF00BF00BF00BF00BF00BF00BF00BF0032
:1036A000BF00BF00BF00BF00BF00BF00D301BF000D
:1036B000BF00BF00BF00BF00BF00BF00BF00BF0012
:1036C000D3016701D301260145012601002100E055
:1036D000013201EB810100EB410110789246A0F12B
:1036E0003004092CA1F13001F2D92E280C9102F1FD
:1036F00001027FF467AF9AF801001146A0F130068D
:10370000092E43F4806340F231812A2800F03E8183
:1037100092460027013256E74C46099B994501D352
:1037200003F1FF394A460020099B0A99D8472046F1
:103730001BB0BDE8F08FA0F16902D2B20F2A41D8C8
:10374000012649F2410196400E4040F001810A2ACB
:103750003FD0072A36D10B9C54F8042B002A00F0E6
:10376000288143F021010DF1480E704603E0202E20
:1037700000F029811A4602F00F052B46092D94BF4F
:10378000303337330F2A00F8013B06F101064FEAC8
:103790001213ECD817E100BF25340020A43F01200C
:1037A000752800200B9C9AF8010054F8045B92469F
:1037B000002DBDBF694243F002030C910C950B94A0
:1037C0000132FCE64A46099B0A9909F10109D847EA
:1037D000CFE60B9951F8048B98F800201046002F83
:1037E00040F0E18072B16FF0010C0CF1010C464623
:1037F000C44401E0664503D016F8014F002CF9D10E
:10380000A6EB080613F4806C02D0BE4228BF3E46E9
:1038100013F0020400F08781002A00F02B81BCF134
:10382000000F00F041810B940D964A46DDE90954E2
:103830000E464F4408E02B462146D84718F8010FA2
:1038400009F1010910B14A464F45F4D131460B9CAC
:103850000D9E002C40F00E810B918AE69AF8010033
:103860006C287FF4DFAE9AF8020043F440730AF14B
:103870000302DAE69AF8010043F400730132D4E659
:103880009AF80100682800F0208143F0800301329B
:10389000CBE6672800F0E780472800F00081452844
:1038A00000F0FF800B9C04930C9B0734CDE902735E
:1038B00024F007031C46DDE90931F4E802674A46B3
:1038C0005846CDE900670B94FFF70AFA814650E6A7
:1038D00046280B9C08BF43F0200304930C9B07343D
:1038E000CDE9027324F007031C46DDE90931F4E851
:1038F00002674A465846CDE900670B94FFF720FC63
:10390000814636E64A462520099B0A9909F10109B4
:10391000D8472EE60B9A9C0702F1040709F101062D
:1039200040F1E6801078099B4A460A99D8470C9BDB
:10393000012B40F22C81DDE90954994432462B4693
:10394000214620200136D8474E45F7D10B9710E687
:103950006F2800F08B8040F26581782800F00881A4
:103960004FF00A0823F01003C44647E0002707EB96
:10397000870700EB4700A0F1300711F8010FA0F115
:103980003002092AF3D98A464A1C1CE60B9C9AF895
:10399000020054F8047B0AF1020A0AF101020B94B6
:1039A00027EAE7770FE6002A3FF42CAF07F1FF3C48
:1039B0001BE723F0100113F4806241F021013FF472
:1039C000D2AE0DF1480E08231020059300234A467D
:1039D000CDE9023006915846DDE90931CDE900E62E
:1039E0000497FFF71FF80B948146C2E5582879D059
:1039F000622840F051824FF00208C44613F4806000
:103A00006DD123F00C0313F4007240F0C2800B99C7
:103A100004310D9113F4807140F02E825E060B9AF2
:103A200040F1AA801278002A40F0DA8023F01003D7
:103A3000002800F0D58011460DF1480E06930C9B2E
:103A4000CDF80CC0CDE90473019100234A460293DE
:103A50005846DDE90931CDF800E0FEF7E3FF0D9BA4
:103A600081460B9385E543F400631BE74FF008089C
:103A7000C446C3E70C9B4C46B3427FF6EDAE0F46FF
:103A80004B44A3EB0609DDE9096522463346294686
:103A900020200134D8474C45F7D13946DCE643F4C1
:103AA000006343F02003FDE60F460B94DDE9095463
:103AB0004A462B462146D84718F8010F09F101095B
:103AC0000028F5D139460B9CC3E69AF8020043F072
:103AD000C0030AF10302A8E5044681461DE623F06F
:103AE0000D0390E74FF0100843F02003C44685E72C
:103AF0000C9B012B45D9DDE909544E4609F1FF38ED
:103B0000984432462B46214620200136D847464568
:103B1000F7D10C9B324699440B9B1878DDE90931AB
:103B2000D8470B9725E50C9BB34240F2EE81CDE9D7
:103B30000D48DDE9095488464B449E1BCDF82CC046
:103B40004A462B462146202009F10109D847B145B4
:103B5000F6D14146DDF838800C9BDDF82CC00D9C79
:103B600098F800205E1C1046002A7FF458AE73E6D9
:103B70004FF01008C44641E71D064CBF128812687A
:103B800051E713464A461878DDE90931D847B1466E
:103B9000DCE60B9C073424F007042246656852F8E3
:103BA000084B0B9254EA050240F02C8123F01003DD
:103BB000002800F0278100260DF1480E06930C9B8B
:103BC0004A46CDE904730023CDE900E6CDF80CC0E8
:103BD00002935846DDE90931FEF724FF8146C8E427
:103BE00013F0200F14BF412061200DF1480E7646DE
:103BF000A0F10A0803E020293FF420AF2246B2FBDF
:103C0000FCF40CFB1425E8B2092D00F130058ABF45
:103C10004044E8B2C0B2624506F8010B01F101016F
:103C2000E9D20BE723F0100269280D9240F06F8172
:103C300013F4806204D04FF4806223F011030D93DB
:103C40000D9B13F4007640D10B9B03F104080D9BF0
:103C500013F4807040F09880590640F1C6800B9BA9
:103C600019780C46CB0F002900F0B98022460DF1DF
:103C7000480E74461646DFF8A0C201E020280FD097
:103C80003546ACFB0621C90801EB8102A6EB4202D6
:103C90003032092D0E4600F1010004F8012BEDD859
:103CA0000D9ACDE9010306920C9ACDE904720A231C
:103CB0004A4603935846DDE90931CDF800E0FEF7A6
:103CC000B1FECDF82C80814653E40B9C073424F0E0
:103CD000070421460846636850F8081BDC0F0B9068
:103CE00051EA030000F0C3800A46191E48DB134660
:103CF0000DF1480EF4460026CDE90E94DFF8188247
:103D000001E0202E2DD05A1842F10002A8FB0259E2
:103D100029F0030505EB9905521B1C469B1A61F11E
:103D2000000508464FF0CC3101FB03F108FB0511FB
:103D3000A3FB08531944052305F00109A9FB033926
:103D40009B180A2C03F130034FEA550570F100006F
:103D50000CF8013B06F1010645EAC1734FEA510137
:103D6000CFD2DDE90E940D9B4A4606930C9BCDE91C
:103D70000164CDE904730A23CDF800E0039328E73A
:103D8000524261EB4101B2E70B9B1968CB0F00294E
:103D900000F0AB8081EAE172A2EBE1720DF1480E16
:103DA0007046DFF874C101E0202E10D01546ACFB40
:103DB0000241C90801EB8104A2EB440404F1300282
:103DC000092D00F8012B06F101060A46ECD80D9AE0
:103DD000CDE9016306920C9ACDE9047267E7002AE7
:103DE0003FF445AF0DF1480E5AE713F0800F0B9BDF
:103DF00000F08180B3F9001081EAE174A4EBE17472
:103E0000A4B22FE713F0200F14BF412261220DF15D
:103E1000480E0A3ACDE90D97CDF844B00026774612
:103E2000F3469146CDE90F3C03E0202E17D004461F
:103E30000D46294642460023204603F009F8D2B237
:103E4000092A02F1300388BF02EB09034445DBB2C3
:103E500075F1000507F8013B06F10106E5D2DE46E3
:103E6000DDE90D97DDE90F3CDDF844B0A6E6002A58
:103E700047D1134611463BE70B990968A1B923F0D6
:103E8000100388B10DF1480E06930C9BCDF80CC0C1
:103E9000CDE904730192D8E513F480627FF4CBAED0
:103EA00023F010030D93CBE613F0200F14BF412035
:103EB00061200DF1480E7646A0F10A0802E0202AA2
:103EC000E2D02146B1FBFCF40CFB1415E8B2092D3D
:103ED00000F130058ABF4044E8B2C0B2614506F83F
:103EE000010B02F10102EAD2CEE7002A3FF456AFFD
:103EF0000DF1480E6BE7196881EAE174A4EBE174F7
:103F0000B0E600260DF1480E2DE701362BE64FF006
:103F10000A081346C44671E5CDCCCCCC70B59446A6
:103F20001E4605460C4684B04FF0FF32634602A998
:103F300000960348CDE90254FFF7FCFA04B070BDC7
:103F4000C12B002010B5094B84B01C684CB103464E
:103F500000914FF0FF3203A90548A047012004B0AB
:103F600010BD00F0BDF9204604B010BDA43F0120F3
:103F7000B92B002000BEFDE708B5FFF7FBFF00BF2F
:103F800038B5064C064DFEF7B3FAAC4204D254F8ED
:103F9000043B9847AC42FAD338BD00BF000A012069
:103FA000100A01200368084611461847437D2DE991
:103FB000F04781460F461646002B43D0002A3BDDD2
:103FC000037D00204D1E014615F8012FDFF8848087
:103FD0000A2A01F101040ED0A6421CD02B782146FA
:103FE000A3F10D03B3FA83F315F8012F5B090A2A35
:103FF00001F10104F0D1002BEED18142A1EB0001CF
:1040000038441BDC02214046D9F800309847A642CC
:1040100008D02046E2E7864204DD311AD9F80030A4
:1040200038449847374417F8013CA3F10D03B3FA1D
:1040300083F35B0989F81430BDE8F087D9F80030C4
:104040009847DFE73846D9F800301146BDE8F04719
:10405000184700BF580701200B682DE9F041802B5D
:104060000D46064605D05A1C2B442A601E71BDE839
:10407000F0810F4B1C68A4B10E4F01F1040801E060
:10408000246974B12368002BFAD03B680BB1A342BA
:10409000F6D1204641462A68FFF788FF2469002CA4
:1040A000F0D1002301222B442A601E71BDE8F0816B
:1040B000983B0120A03B01202DE9F04782B00D463E
:1040C000924699460746FDF7EFFE4FF0FF366FF038
:1040D00000442F4A821841F10003964274EB030119
:1040E0003CBF324623462B4803F0FAF96B1C80464E
:1040F00003D1384603F014F90546274B274E1C68B8
:10410000274BB9F1000F18BF1E46B4B1BAF1000F2A
:104110001AD1DFF8909001E0246974B12368002B74
:10412000FAD0D9F800300BB19C42F5D120462A468E
:104130003946B0472469002CF0D1B8F1000F1FD1E7
:10414000284602B0BDE8F0874FF00A0ADFF8549025
:1041500002E02469002CF0D02368002BF9D0D9F8B4
:1041600000300BB1A342F4D12A4639462046B0476D
:10417000012220460DF107018DF807A0B047E8E7BE
:10418000044803F0FFF9284602B0BDE8F08700BFFD
:1041900040420F00B8090120983B0120953E0020C5
:1041A0009D3E0020A03B0120F0B583B006468DF86F
:1041B0000700FDF779FE4FF0FF356FF00044174A16
:1041C000821841F10003954274EB03013CBF234682
:1041D0002A46134803F084F9124B07461C689CB129
:1041E000114D01E024697CB12368002BFAD02B68C3
:1041F0000BB19C42F6D1204601220DF10701FFF7D9
:10420000D1FE2469002CEFD117B9304603B0F0BDC0
:10421000034803F0B7F9304603B0F0BD40420F0049
:10422000B8090120983B0120A03B01200A4A1368ED
:104230004BB1834202D109E0984207D003F110024A
:104240001B69002BF8D101B1106070470029FCD127
:104250000369136001617047983B0120F0B583B09A
:1042600006468DF80700FDF71FFE4FF0FF356FF093
:104270000044174A821841F10003954274EB030190
:104280003CBF23462A46134803F02AF9124B07463F
:104290001C689CB1114D01E024697CB12368002B9E
:1042A000FAD02B680BB19C42F6D1204601220DF1C9
:1042B0000701FFF77BFE2469002CEFD117B93046C8
:1042C00003B0F0BD034803F05DF9304603B0F0BD24
:1042D00040420F00B8090120983B0120A03B01207B
:1042E00038B5044603F01CF8012305461A4620465B
:1042F0002946FFF7E1FE084B1C682CB163682BB11F
:1043000098472469002CF9D1284638BD2469002C2F
:10431000F4D1284638BD00BF983B01202DE9F0417B
:10432000A2B004460D46FDF7BFFD4FF0FF376FF01A
:104330000046274A821841F10003974276EB0301B9
:104340003CBF3A463346234803F0CAF800262B46C2
:1043500007462246204801A90196FFF7DFFD019B91
:1043600006467BB91D4B1C682CB1636843B1984766
:104370002469002CF9D10FBB304622B0BDE8F08192
:104380002469F1E7DFF85480D8F80050EDB1144CFF
:1043900001E02D6975B12B68002BFAD023680BB1B1
:1043A000AB42F6D12846019A02A9FFF7FFFD2D691D
:1043B000002DF0D1D8F800400195D5E7054803F06D
:1043C000E1F8304622B0BDE8F0810195D3E700BFA7
:1043D00040420F00B8090120493F0020983B0120CE
:1043E000A03B01200FB400B583B004A951F8040B21
:1043F0000191FFF793FF03B05DF804EB04B0704741
:10440000704700BF0022014B1A707047074002201E
:104410004B79FF2B0BD1887948B9CB79012B07D188
:10442000082A05D9034B8A7809201A7070470020A2
:10443000704700BF0740022001207047012901D0CA
:104440000120704708B5104B91881B78994201D024
:10445000002008BD5378012B08D0022BF8D1002191
:1044600064220846FDF780FF012008BD5188CB0576
:104470004BBF4A0A4A0A10464FF0FF3002F00102D1
:1044800001F07F01FDF7EEFF074002200048704772
:1044900024080120012907D15378012B02D19388E8
:1044A000072B03D000207047012070471146A62338
:1044B000014A01F041BA00BF7C07012003460122F6
:1044C00001481A70704700BF5C07012008B50B68EF
:1044D000B3F5966F00D008BD00224FF0FF301146B3
:1044E000FDF7C0FF024A034B10601960704700BF20
:1044F000343B0120383B0120184B70B51A68002A64
:1045000028D0EFF3108172B6D2E8CF4F0120002CF3
:10451000FAD1C2E8440F002CF6D1BFF35F8F00221E
:104520000F4C186859602270C0E88F2F81F31088F3
:10453000002400250B4E3078FCF7F6FD20B900244E
:1045400000252046294670BD3078FCF7FDFD204649
:10455000294670BD4FF47A740025EBE7B43F012083
:104560000940022008400220014B1878FCF7ECBDFE
:104570000840022038B5044600200D4601F008FB33
:10458000A8B3002001F01AFB88B3FDF78DFC4FF0B3
:10459000FF3E6FF0004C174A821841F10003964528
:1045A0007CEB03013CBF72466346134802F098FF60
:1045B000E8B1002001F0ECFA58B900214FF0FF30CB
:1045C00000F012FD6FF002040B4802F0DBFF204602
:1045D00038BD002001F0F2FA0028EED021462A462C
:1045E000002001F0F7FA04460028EDD1EAE76FF069
:1045F0000204ECE740420F00E83F022008B5FDF757
:1046000053FC4FF0FF3E6FF0004C0F4A821841F10F
:10461000000396457CEB03013CBF724663460B48A2
:1046200002F05EFF70B14FF0FF30002100F0DCFCC3
:10463000002001F015FB0028F5D1BDE80840034833
:1046400002F0A0BF08BD00BF40420F00E83F0220BB
:104650002DE9F84307460E46FDF726FC4FF0FF35DF
:104660006FF00044334A821841F10003954274EB25
:1046700003013CBF2A4623462F4802F031FF08B908
:10468000BDE8F883002001F083FA002848D0002E0E
:1046900041DD0025DFF8A480DFF8A49013E0224676
:1046A000002001F023FB002104464FF0FF3000F012
:1046B0009BFC002001F0D4FAFDF7F6FBC8E90001ED
:1046C0002544AE4227DD002001F032FB741B8442FA
:1046D000A8BF04467919002CE1D121464FF0FF30E4
:1046E00000F082FC204601F0BBFA204601F050FAAF
:1046F00088B1204601F01CFB0028E2D1FDF7D4FB75
:10470000D8F80030D8F8042013EB090342F1000276
:1047100083428A41D5D20848BDE8F84302F032BF4F
:1047200000200021054BC3E90001BDE8F843024821
:1047300002F028BF40420F00E83F0220700C012029
:1047400020A1070030B5002185B02E4802F068FE98
:10475000F0B92D4B1A68CAB1EFF3108172B6D2E8E6
:10476000CF5F0124002DFAD1C2E8454F002DF6D1CC
:10477000BFF35F8F254C1D6822785960D3B20122A8
:104780002270C5E88F0F81F31088CBB105B030BD22
:1047900000214FF0FF3000F027FC002001F00EFA5E
:1047A0000446184802F0EEFE002CEFD0184B1B68B0
:1047B000002BEBD0174A106805B0BDE83040184711
:1047C000FDF7DEF80446FDF76FFB4FF0FF3C6FF09E
:1047D000004510F57A7241F10003944575EB030131
:1047E00038BF2B464FF000014FF0010520460A4C20
:1047F00038BF6246CDE901150094FDF7C5F805B054
:1048000030BD00BFE83F0220B43F01200940022034
:10481000343B0120383B0120E94300204FF0504356
:1048200030B585B01C68FDF7ABF8FDF7BFF9A042C5
:1048300002D0002005B030BD00212A4B08461B786D
:1048400001F046FD28480368002B47D00120FCF703
:1048500019FE0346254C2649C0B22370FCF790FC94
:1048600020780121FCF74AFC0E20FCF779FC40BBC4
:10487000204B0125C3E90000FDF782F80446FDF74F
:1048800013FB4FF0FF3E6FF0004C10F57A7241F1D0
:10489000000396457CEB03014FF000012046164CC7
:1048A0003CBF72466346CDE901150094FDF76CF8F4
:1048B0000028BEDB01211148FFF7B8FC012005B03C
:1048C00030BD0120FCF7D6FB01460A48FCF736FE56
:1048D00000220E200A49FCF783FCEBE7FCF712FEEE
:1048E000B4E700BF1C020010E83F0220084002208D
:1048F00035460020B43F0120E9430020780901201B
:104900005944002000487047C00801200048704703
:104910006C08012038B5184B04461A780AB344B91C
:1049200040F209424FF44173144D6A8013482B80C2
:1049300038BD052C1AD8124B104D53F824102846B8
:104940000023013903E0132B20F8022F10D011F8B7
:10495000012F0133DBB2002AF5D15B0043F4407331
:10496000E4E71121184600F025F8D8E7002038BD0B
:104970004FF44A73DAE700BFF03F0220703B01209A
:104980005408012000B545F247308BB0FDF75EFDBD
:1049900001220346092101A89847DDE903320449B1
:1049A00012BA1BBAC1E900230BB05DF804FB00BFCB
:1049B000DC3F0220012901F1FF3300F0B3805D49A3
:1049C0000A784FEA121C9F2A8CBF0CF1370C0CF1AD
:1049D000300C012B80F800C000F0A78002F00F021D
:1049E000092A8CBF37323032022B427000F09D8092
:1049F0004A784FEA121C9F2A8CBF0CF1370C0CF13D
:104A0000300C032B80F802C000F08F8002F00F0200
:104A1000092A8CBF37323032042BC27000F08580F7
:104A20008A784FEA121C9F2A8CBF0CF1370C0CF1CC
:104A3000300C052B80F804C077D002F00F02092A51
:104A40008CBF37323032062B42716ED0CA784FEAB3
:104A5000121C9F2A8CBF0CF1370C0CF1300C072B69
:104A600080F806C061D002F00F02092A8CBF3732ED
:104A70003032082BC27158D00A794FEA121C9F2A93
:104A80008CBF0CF1370C0CF1300C092B80F808C0EE
:104A90004BD002F00F02092A8CBF373230320A2B7A
:104AA000427242D04A794FEA121C9F2A8CBF0CF105
:104AB000370C0CF1300C0B2B80F80AC035D002F00B
:104AC0000F02092A8CBF373230320C2BC2722CD025
:104AD0008A794FEA121C9F2A8CBF0CF1370C0CF11B
:104AE000300C0D2B80F80CC01FD002F00F02092AE9
:104AF0008CBF373230320E2B427316D0CA7911096F
:104B00009F2A8CBF373130310F2B81730DD002F0CB
:104B10000F02092A94BF30323732102BC27318BFEC
:104B2000103002D000230370704718440023037034
:104B3000704700BFDC3F022070B500F033F90C2352
:104B400040261B4CFF22A3670E201A49FCF748FBA6
:104B5000194B32460021184602F014FB034600218F
:104B600001258020154A58849A60843A5D701E831E
:104B70001E875960C2F88410C2F8801002F5807256
:104B8000DA60DA62803A83F8211083F83B105962C8
:104B90009A624FF0005602F013FD4FF4803208493C
:104BA000084B25642846E664C4F89010DA6470BDAA
:104BB00000001150A9750020A43B01208400105072
:104BC00010D001000020115001210E20FCF796BAF0
:104BD00000220248114600F005B900BFC43B012085
:104BE000044B197021B14FF40032034BC3F89020ED
:104BF000704700BF02400220002011500B785B0676
:104C000002D14B78052B00D070474B88014ADBB2AC
:104C10001360704700001150CB782DE9F04103F08C
:104C2000030EBEF1010FC3F301005DD0002791F820
:104C300002C0354C0CF07F035E00898806EBDC1265
:104C400004EB42124FEADC15D076C1F30A0185F07D
:104C50000100507082F802C01183D77018B2DA00D8
:104C60008DBB2A48043204EB831C02EB0008CCF80D
:104C7000088017508BB3264ADB001A44CCF8042076
:104C8000244B3F311A6821F03F01BEF1020F08BFEB
:104C9000490011441960204B771904EB47179942DA
:104CA000FA602CD82E4404EB4613D97E82F0A04241
:104CB00082F480125B6842EA816242F000421A602C
:104CC0000120BDE8F081DFF844C004EB83186244A2
:104CD000C8F828204CF830704BB900220F4904EB7B
:104CE0004513D9605A60EBE70020BDE8F081DB0096
:104CF00003F1A04303F58013C8F82430C0E7FDF7A3
:104D0000F1FBFA68CEE700BFA43B01208000105001
:104D100004001050B03F0120FF0F10500001105050
:104D200002F04EBC8C4608B5114607481A460CF0F6
:104D30007F034FEADC1C0CEB430C00EB4C1000F043
:104D400051F8012008BD00BFA43B0120CB0911F0A0
:104D50007F0103D1064AC3F102009066054803EBC8
:104D600041034FF40062002100EB431003F034B81C
:104D700000201150A43B012011F07F0300D17047A7
:104D8000002210B4C809064C00EB430004EB4013AA
:104D90006FF4006118465DF8044BDA7003F01CB83C
:104DA000A43B01204FF0805209480A4908B50A4B3C
:104DB00002600A609968C94311F08051FAD14FF43A
:104DC0008052064802F0DEF90922054B5A6708BDF9
:104DD000002002400030024000000240000010505D
:104DE0000000115000234FF0010C10B580F81AC0DC
:104DF0008282C3820161044602F0C0FF20B14FF4F9
:104E00000032074BC3F89020204602F0CBFF10B1D0
:104E10000123237710BD2046BDE8104002F0FEBFFD
:104E2000002011502DE9F04100241D4E0546234677
:104E30003278DFF878801B4F0DE03B6813EB4413AA
:104E400025D0DB682846984732780134E4B2511CFB
:104E5000A142234606DBA242A3EB0203EDD808EBF6
:104E60004313EEE7104C54220021204602F08AF949
:104E70004FF0FF33251D6360C5E90133EB6004F19A
:104E800014002022BDE8F041FF2102F07BB94FF071
:104E9000E023D3F8F03DDB0700D500BEBDE8F0818C
:104EA000014002203836012040370120D40801207B
:104EB000704700BF704700BF002070470020704758
:104EC000704700BF704700BF704700BF704700BF0A
:104ED000024B5878003818BF012070474037012036
:104EE000024B1878C0F38000704700BF40370120A4
:104EF0002DE9F047DFF8E8A09AF80030FF2B02D048
:104F00000120BDE8F0870E4600293ED00021542242
:104F10000746294802F036F90022284C284B204643
:104F20001A70FCF7EFFA274B27481C60274CFCF758
:104F3000F7FA204601F0B0FD254A264B264D1460B5
:104F400063B32846FFF7BAFA244B2A781860002486
:104F5000DFF890902346DFF884800EE0D8F8003028
:104F600013EB441311D05B687BB198472A78013466
:104F7000E4B2511CA142234612DBA242EED89B1A96
:104F800009EB43135B68002BEFD14FF0E023D3F81C
:104F9000F03DDB0700D500BE0020B2E72A78D6E757
:104FA000314638468AF80070FFF7C6FD0028ECD07D
:104FB0003846FFF709FEA3E74037012038370120C4
:104FC0000340022094370120A40901209009012008
:104FD00098370120AD4300200140022038360120DF
:104FE000AC090120D40801202DE9F04FDFF8C89268
:104FF0008BB099F80030FF2B00F0F180A84CA94D40
:10500000DFF8B0A2DFF8B4B226687369EFF310825C
:1050100072B6D3E8CF0F01210028FAD1C3E8401FB0
:105020000028F6D1BFF35F8FB261304607A901F0C7
:1050300081FB00237269C2E88F3FB36983F3108854
:10504000002800F0CC809DF81D30013B072B00F2BA
:105050007D83DFE803F0A7B1959D8E350A04089B98
:10506000002BD1D009989847CEE79DF8201001F089
:105070007F0605EB460000EBD11090F8343023F0AA
:10508000010380F8343090F8343023F0040380F8C2
:105090003430002E00F0A680037D9AF80020934261
:1050A00080F09380804A126812EB431300F09080E6
:1050B0009E699DF82120099B9DF81C00B047A3E73D
:1050C0009BF80030002B00F083809BF80030013B00
:1050D000DBB28BF800309BF8003003F0FF00002BB0
:1050E00092D1704F9DF81C803B7843F001033B70D8
:1050F00097F8343060F3000387F8343097F8343091
:1051000060F3820387F8343097F8353060F300039A
:1051100087F8353097F8353060F3820387F83530FB
:1051200000F06AFC9DF8203003F06002602A6CD029
:10513000402A7CD003F01F03012B00F0C180022B1A
:1051400000F08180002B60D1202A00F0E981002A44
:105150005BD19DF82130092B57D8DFE813F0B0015F
:10516000A2015600C101560095016B015600600175
:10517000F4002B78D9077FF547AFFFF7A7FE43E789
:10518000EB78DA077FF540AF0898FFF793FE3BE72F
:105190002B78D8077FF538AF2878C0F3C000FFF729
:1051A00093FE31E79DF81C00FFF73CFE00F01AFC6F
:1051B0009DF82030AB7027E79DF81C00FFF732FE0A
:1051C00000F010FCFFF77EFE1EE7501C984211DA3B
:1051D0004FF0E023D3F8F03DDC0700D500BE0BB064
:1051E000BDE8F08F099B9DF821209DF81C0000F080
:1051F00017FC09E79B1A2D4A02EB431358E7FFF708
:1052000085FB0246002840F082814FF0E023D3F86E
:10521000F03DDE0700D500BE9DF81C000021FFF721
:1052200095FD80219DF81C00FFF790FDECE62048DD
:1052300000F0E2FB0121404608AAFFF72BF9002805
:105240007FF4E2AEE8E79DF8241011F0700FDCD196
:1052500001F07F0607EB4600164B00EBD1101B78E0
:10526000007D7600019698424FEAD116009659D3F8
:105270005E1C8642C0F26681C01A0C4B03EB4016DE
:10528000002A00F06381706900F0B6FB01214046FE
:10529000736908AA984700287FF4B6AEBCE700BF40
:1052A000983701204037012038360120D4080120EA
:1052B0008543002001400220AC0901200340022068
:1052C0009DF824300F2BA7D8AE4A3B441B791278A7
:1052D000934232D3511C99429EDBAB4E9B1A06EB94
:1052E0004316706900F088FB01214046736908AAE3
:1052F000984700287FF488AE9DF8203013F06006B0
:105300008AD19DF821300A3B012B85D800F074FB2F
:105310009DF821300A2B00F0F281404608A900F0E8
:10532000F1FA71E6994B1B6803EB4016002A00F076
:105330000D81002E3FF470AFA5E7944A166816EB76
:105340004316CED168E77B789DF822609E4200F03C
:105350004F817B78002B40F0BE817E70002E00F0E4
:105360004581701EC0B2FFF7D1FA0346002800F055
:105370005F814278022A40F05B81C17903F109061E
:10538000C1F340121201C1F3801142EA41123146C9
:10539000387820F0300002433A705A88CDF80C80FB
:1053A0009A180192019B8B4240F2A4814A780B2A01
:1053B00000F0AF810123042A40F03A810026019ACF
:1053C0000096521A92B202926E4A049312781DE02D
:1053D0006E4B1B6813EB461800F02A81029AD8F82E
:1053E000103003980591984708280246059906F160
:1053F000010303D90298904280F0FF80DEB2614B36
:1054000000961A78531C9E4200F31281009BB24210
:10541000A3EB0202DCD85C4B03EB4218DEE77B789F
:1054200040468DF81A300DF11A02012308A900F048
:1054300083FAE9E5BDF82200030A013B020AC0B283
:105440000E2B3FF6E9AE01A151F823F05155002093
:10545000ED5300208D5500200951002009510020F6
:105460006F550020ED530020095100200951002004
:105470000951002009510020095100200951002044
:10548000095100204355002008A800F0BBFA40460F
:105490009DF82210FFF79CFB3B7843F002033B7022
:1054A000B2E5BDF82230012B7FF4B6AE3B78404622
:1054B00023F0080308A93B7000F024FAA4E5404655
:1054C0003B789A0802F00202C3F340131343ADF88D
:1054D0001A300DF11A02022308A900F02DFA93E503
:1054E000BDF82230012B7FF497AE3B78404643F065
:1054F000080308A93B7000F005FA85E5022A3FF48D
:105500007EAEFFF7DBFC024600283FF485AE404646
:10551000538808A900F010FA00287FF475AD7BE6E7
:105520009DF824300F2B3FF677AE164A3B441B798B
:10553000127893421DD2154A166816EB43167FF473
:10554000A2AE69E6002A7FF467AE00269DF821200E
:1055500002F0FD03012B1BD0002A7FF456AE019B05
:10556000009A3B44134493F834304046C3F340035D
:10557000ADE7511C9942FFF64FAE034E9B1A06EB66
:10558000431680E601400220D4080120383601206D
:10559000BDF82230B3B9012A99F8000000F08680E6
:1055A000FFF7D4FB019B009A3B44134493F834204B
:1055B00042F0020283F8342093F8342042F00102D2
:1055C00083F83420002E3FF41FAD706900F014FA08
:1055D0007369012108AA40469847002000F00CFAA0
:1055E00097F83530DF073FF50FAD96E6FFF76AFC19
:1055F000404608A900F086F906E5049B012B00F05F
:105600009E80002B00F08A80002091F8028005E047
:105610008CF804605FFA80FC63457FD908EB000CCE
:1056200057FA8CFC9CF804E00130BEF1FF0FEFD07C
:105630004FF0E023D3F8F03DDA0700D500BE4FF07D
:10564000E023D3F8F03DDB0700D500BE00237B70DC
:10565000E2E5FEF71BFF024600287FF458AFDBE5CA
:10566000FFF750F9024600283FF4CFAD4046122321
:1056700008A900F061F900287FF4C6ACCCE5FFF77B
:105680001BFC024600283FF4C7AD4046137808A92A
:1056900000F052F900287FF4B7ACBDE5BDF8241046
:1056A000FFF738F902460028EFD1B5E50293FFF77E
:1056B00063FB019A009B3A441A4492F83410029B0F
:1056C00063F3410182F8341092F8341063F300015F
:1056D00082F8341076E700214046FFF781FA404611
:1056E000FFF71EFBBB7840460093FFF79BFB009B38
:1056F000BB7032E6DDF80C80FFF7E2FB78E740464E
:10570000012308A90DF11A028DF81A6000F014F9AE
:105710007AE40A78CB7811444A784CE6334610484C
:105720000492029100F07CFE0E4B049A02991B78C1
:105730001144009A01339342BFF634AE78E7D8F8AB
:1057400010C00948844508BF02235DE74FF0E023FD
:10575000D3F8F03DDB077FF557AC00BE54E400BF43
:105760005437012001400220215D00202DE9F84F2F
:10577000DDF82880002A3FD00C461E4615464FF023
:10578000000B1F4FDFF87C9017E0204699F80210BD
:1057900000F014FEF8B121465046FFF73DFA08B379
:1057A000A3780BF1010BDA0916BF0B9A88F80030C9
:1057B00013702378AB451C441ED06378052B11D1A0
:1057C000E17801F00301B1420CD1A37897F800A071
:1057D00013F0700FD9D04FF0E023D3F8F03DDA0783
:1057E00000D500BE4FF0E023D3F8F03DDB0700D535
:1057F00000BE0020BDE8F88F0120BDE8F88F00BF93
:10580000AC0901204037012038B50E4B1D788B784C
:1058100013F0700F08D04FF0E023D3F8F03DDB0712
:1058200000D500BE002038BD074B0C4608469978CD
:1058300000F0C4FD0028EED021462846BDE83840DF
:10584000FFF7EAB9AC090120403701200B46064AB0
:1058500006481168DA09343203F07F0302EB430390
:10586000184400F065BD00BF943701204037012087
:105870000B46064A06481168DA09343203F07F0302
:1058800002EB4303184400F07DBD00BF94370120B4
:105890004037012010B5194C01F07F0E04EB4E0487
:1058A00004EBD11494F834C015481CF0010F04F136
:1058B0003004007808D04FF0E023D3F8F03DDA0749
:1058C00000D500BE002010BD94F804C04CF0010CBF
:1058D00084F804C0FFF726FA0028F4D14FF0E02145
:1058E000227960F300022271227960F38202227130
:1058F000D1F8F03DDB07E5D5E3E700BF40370120F5
:10590000AC09012030B50B4C8C46A646054608680C
:1059100049680023AEE803009CF800102846C943FC
:10592000C4E90233BDE830401A4601F08001FFF7B8
:10593000B1BF00BF003701202DE9F041274F4FF0E4
:105940000008BE468C46064608684968BA60AEE85C
:105950000300A7F80E801546BCF80620934228BF26
:105960001346BB819AB11C462BB3DDB197F90030C9
:10597000402C28BF4024002B28DB414623463046DC
:10598000174AFFF787FF68B10120BDE8F0819CF856
:1059900000101346C943304601F08001FFF77AFF3B
:1059A0000028F1D14FF0E023D3F8F03DDB0700D51C
:1059B00000BE0020E9E71A46397801F0800123464D
:1059C0003046FFF767FF0028DED1EBE72246294685
:1059D000034801F029FC8021014AF0E7003701204B
:1059E000C03601200022034BC3E90022C3E9022292
:1059F0001A61704700370120014B1861704700BFE2
:105A00000037012030B40246044C002523460068CC
:105A10005168C4E9025530BC03C370470037012008
:105A200070B53C4CC90922780646B1EBD21F1D4621
:105A300082B017D053B14FF0E023D3F8F03DDB072D
:105A400002D4002002B070BD00BEFAE72146FFF785
:105A5000D5F823691BB1224603213046984701201F
:105A600002B070BD94F90030A068002B05DB00285F
:105A7000E7D02A46284901F0D7FBE089A168E388EE
:105A8000284480B229448342E081A16016D03F2D92
:105A900014D9A28994F90040131A9BB2402B28BF55
:105AA0004023002C26DB90424FF0000130D01A4AF0
:105AB0003046FFF7EFFE0028D1D1BCE7236923B1C0
:105AC00002213046134A984758B121780023C94330
:105AD00030461A4601F08001FFF7DCFE0028BED1F7
:105AE000A9E701463046FFF731F980213046FFF73C
:105AF0002DF9B4E7904208D01A460748019301F007
:105B000093FB8021044A019BD2E780210022CFE74A
:105B10000A46CDE700370120C03601202DE9F041CB
:105B20000446FFF7D5F908B9BDE8F081FFF7D8F9C9
:105B300007460028F8D1C822134B02FB0436F1783F
:105B40000029F1D006F11005284600F0E1FD3F28BC
:105B5000EAD93846F178FFF779FE0028E4D02846E4
:105B600000F0D6FD3F2809D9084A3846F17802EB03
:105B7000C4124023BDE8F041FFF78CBE3846F178EF
:105B8000BDE8F041FFF774BE280A01203C36012031
:105B900010B50446FFF79CF908B9002010BDFFF7C7
:105BA0009FF90028F9D1C822034B02FB043318796E
:105BB00000F0010010BD00BF280A0120C82108B56F
:105BC000102301FB0030024A104400F087FD08BD9D
:105BD000280A01202DE9F8434FF6FF734FF0C8085B
:105BE00010249A4228BF1A4618FB00441A4F064652
:105BF0003C44204692B200F0E7FD0546FFF768F905
:105C000010B92846BDE8F883FFF76AF981460028F5
:105C1000F7D108FB0677FB78002BF2D0204600F086
:105C200077FD3F28EDD94846F978FFF70FFE0028A9
:105C3000E7D0204600F06CFD3F2808D9074A4846C7
:105C40004023F97802EBC612FFF724FED9E7484655
:105C5000F978FFF70DFED4E7280A01203C36012031
:105C60002DE9F0410546FFF733F910B90020BDE8F2
:105C7000F081FFF735F906460028F7D14FF0C80844
:105C8000242418FB0544174F3C44204600F026FD11
:105C90000028EBD008FB05773046B978FFF7D6FD32
:105CA0000028E3D04022104B204602EBC5141C44D0
:105CB000214600F089FD054680B103462246304664
:105CC000B978FFF7E7FD38B94FF0E023D3F8F03D9E
:105CD000DB07CBD500BEC9E72846C8E7B978FFF790
:105CE000C7FDC3E7280A01203C36012038B54FF62E
:105CF000FF734FF0240CC8249A4228BF1A4614FBA5
:105D000000C40A4B92B21C440546204600F018FE1F
:105D1000034620461C4600F0E1FC3F2801D82046FF
:105D200038BD2846FFF79CFF204638BD280A0120D1
:105D3000C82108B5242301FB0030024A104400F0BA
:105D4000E7FC08BD280A0120F0B5194C83B0C82231
:105D50000021204601F016FA0025FF234FF4E1311F
:105D60000822144804F1B8070570009504F11000EA
:105D70006371A160A27304F138010123402200F095
:105D80007DFC0123402204F17801009304F12400FA
:105D900000F074FC04F1C0063846FBF7B3FB304654
:105DA000FBF7B0FBC4E90757C4E90C6503B0F0BDCD
:105DB000280A0120BC360120094B196B49B11A6A27
:105DC00012B10022C3E907220022C3E90C220120FC
:105DD00070471A6A002AFAD00120C3E907117047F8
:105DE000280A0120002210B50E4C0F4823780260CB
:105DF0000271DA0707D59B070BD5BDE810400121DA
:105E00000A4800F065BE103000F046FE23789B077C
:105E1000F3D4064800F040FEBDE8104001210348DD
:105E200000F056BEBC360120280A01204C0A012091
:105E3000F0B54B7983B0022B03D00025284603B080
:105E4000F0BD8B79022BF8D1264FBB783BB14FF0D8
:105E5000E023D3F8F03DDB07EFD500BEEDE78B780C
:105E600006463B700B780925CC18617824290BD1A4
:105E7000082A02D80FE0AA420DD323781C44617887
:105E80002B4424299DB2F6D005290AD0042902D139
:105E900063790A2B13D00020FFF740FE284603B099
:105EA000F0BD21463046FFF7AFFC0028CFD0A378E5
:105EB0007B7023781C442B4461789DB2E6E70A4B43
:105EC0002778019301330093022330461A46E119E3
:105ED000FFF74CFC0028BAD00E3517FA85F5ADB2A5
:105EE000D9E700BF280A01202A0A0120137803F00D
:105EF0006003202B08D170B5264C938894F800C01D
:105F00009C4503D0002070BD002070475378203B93
:105F1000032BF7D8DFE803F027230D0201292ED049
:105F200003291ED11C4BE3B100205188AFF3008040
:105F300017E0012923D0032913D15588174805F00C
:105F4000010686F00101257100F0C2FD144B43B13A
:105F500031460020C5F34002AFF3008001E0012983
:105F600011D0012070BD01290DD00329F9D10D4BAD
:105F7000002BF6D000200C49FEF7A8FAF1E71146F5
:105F8000FFF7C0FCEDE711460723074AFFF7D4FCF3
:105F9000E7E700BF280A0120000000004C0A0120AA
:105FA00000000000BD430020300A01202DE9F04729
:105FB000364F0C46FA7806468A421D4697F802C0CC
:105FC0003CD08C4513D04FF0E023D3F8F03DDB07F5
:105FD00000D500BE0020BDE8F0872D4B23B12D4831
:105FE00000F08CFB00284ED00020FFF797FDBB7817
:105FF000A34202D00120BDE8F087274B13B1002057
:10600000AFF300800020FFF72BFE0028F2D12348D9
:1060100000F064FB0028EDD1002DEBD015F03F051A
:10602000E8D13046B978FFF711FC0028E2D02B46C2
:106030002A463046B978FFF72DFCDBE7DFF86480AD
:106040009AB2414607F1100000F07AFC144B002B85
:10605000C3D07B79FF2BC0D0002DBED007F1100933
:1060600008EB050A02E0C245B7D07B7918F8012B8E
:106070009A42F8D1484600F041FB0028F3D17979E3
:10608000AFF30080EFE7AFF30080ADE7280A01200F
:1060900000000000380A0120000000004C0A012026
:1060A000000000003C360120F0B5144C85B04FF4E0
:1060B00013720021204601F065F8402700234FF4B9
:1060C00080760F4D04F5A6721946CDE9025700926D
:1060D00001961A4604F5947000F0CEF9002304F1FD
:1060E00028013D44009101221946CDE9025701964D
:1060F000201D00F0C1F905B0F0BD00BFE838012057
:106100006838012010B5054C204600F0E1F9A4F5EF
:10611000927000F0DDF9012010BD00BF103A01209F
:1061200038B50025064C04F59870257000F0B4FCD5
:1061300004F10C0000F0B0FC84F82951657138BD01
:10614000E83801202DE9F84F4B79FF2B02D00020D1
:10615000BDE8F88F394D0E4695F829310C78002BA3
:10616000F5D16F79002FF2D18B780C442B700B791D
:10617000002B3ED0804604EB020B05F5987A05F51E
:1061800094796378052B09D0A34502D831E05C45AA
:106190002FD223781C446378052BF8D1A34528D946
:1061A00021464046FFF730FB00283ED0A378DB09AC
:1061B00023D1504600F070FCA37895F8281185F89B
:1061C0002931A3884046C3F30A03A3F50073B3FA49
:1061D00083F35B0963F3410185F82811494600F018
:1061E000E5F910B32378317901371C44FBB29942A9
:1061F000C7D8A11B88B2BDE8F88F114800F04CFC4D
:10620000A37895F804C06B71A3880E49C3F30A0301
:10621000A3F50073B3FA83F35B0963F3410C002029
:1062200085F804C000F08AF9DCE74FF0E023D3F8EA
:10623000F03DDB078BD500BE89E700BFE8380120C1
:10624000F4380120EC38012070B51B4C064694F858
:1062500029C11D468C45627904D08A4218BF0020AE
:1062600018D070BDB4F8343163B9144B23B1002099
:106270001349AAB2AFF300803046124900F096F9F4
:10628000012070BDD4F82C11AAB204F5987000F06A
:1062900057FBEAE70C4B1BB10020A9B2AFF300801B
:1062A00030460A4900F04AF90028E9D12A4630462A
:1062B000064900F00FF9E3E7E8380120000000008C
:1062C00068380120103A012000000000EC3801205D
:1062D00010B582B0B9B101280CD80B7853B1134C6A
:1062E000012B235402D0012002B010BDFEF700FEA6
:1062F0000028F8D14FF0E023D3F8F03DDB0700D5BC
:1063000000BE0020F0E70124084601A9ADF80440D2
:10631000FEF7EEFD38B94FF0E023D3F8F03DDA0791
:10632000E2D500BEE0E7014B1C70DDE73437012009
:10633000F8B5037813F001041AD1037805465A071B
:10634000C3F3800701D52046F8BD0E464FF0FF315C
:10635000304601F0FBF82B7813F001040BD12B78B9
:106360005B0709D42B78012443F004032B7003E06E
:1063700000242046F8BD3C46304601F003F9204693
:10638000F8BD00BF70B50C4605464FF0FF31204602
:1063900001F0DCF82B78C3F380065B0708D52B7877
:1063A00013F0010311BF00262A7863F382022A70DA
:1063B000204601F0E7F8304670BD00BFC378828800
:1063C00003F003000228C2F30A021FD0032803D0FF
:1063D00001280AD000207047022914BF40234FF43F
:1063E0008063934209D301207047022940F2FF33B2
:1063F00008BF4FF480639342F6D24FF0E023D3F806
:10640000F03DDB07E6D500BE00207047022902D030
:10641000402AE8D9F1E7B2F5007FE4D0EDE700BF0C
:106420000A44914226D291F801C0BCF1050F05D073
:1064300091F800C061448A42F5D8704700B591F8E0
:1064400002C00CF07F0E00EB4E0E4FEADC1C0EF883
:106450000C3091F800C061448A4209D991F801C01A
:10646000BCF1050FEBD091F800C061448A42F5D829
:106470005DF804FB704700BF2DE9F0418E4682B005
:10648000009390F800C0089EBDF824706EF3000CD5
:1064900004461546012331463A4600F808CBBDF8BC
:1064A0002C8000F0EBF806B13FB901200A9BA4F85C
:1064B0000280636002B0BDE8F08104F11C06304642
:1064C000FBF720F80DB135460026C4E90556ECE788
:1064D00001207047F8B50746084640F2FF131546FD
:1064E00010F8082B0C4612F0020F0CBF3F261E4678
:1064F00000F0F4F828B925B12E4202D12378DA074A
:1065000001D50020F8BD38466178FFF79FF90028D3
:10651000F7D0237813F0010307D04FF0E023D3F82E
:10652000F03DDB07EDD500BEEBE71A463846617853
:10653000FFF7B0F90028F0D0F8BD00BF70B501F149
:106540000805064628460C4600F0C8F810B1237826
:10655000D80701D5002070BD30466178FFF776F985
:106560000028F7D028466288616800F02DF923786A
:10657000054648B1D9070ED54FF0E023D3F8F03DDA
:10658000DA07E7D500BEE5E7DB07E3D430466178FC
:10659000FFF76EF9DEE70346626830466178FFF781
:1065A00079F90028E8D0284670BD00BF8A892DE916
:1065B000F0410B780C4605468AB9DF0725D44978A7
:1065C000FFF744F908B322786388D6073FD54FF028
:1065D000E023D3F8F03DDA0717D500BE15E003F04D
:1065E000020301F10808002B40460CBF40274FF47E
:1065F00000774FF6C07618BF4FF47E4600F088F85B
:10660000874202D82378D80702D50020BDE8F08160
:1066100028466178FFF71AF90028F6D0404600F0C6
:1066200077F887421FD823786288D907CFD43040C3
:10663000904228BF104661780646E0B16268334652
:106640002846FFF727F90028C1D03046DEE76178F9
:106650003BB162682846FFF71DF90028B7D0608873
:10666000D4E71A46F6E72378DB07CED428466178CC
:10667000FFF7FEF8C9E70246E1E700BF2DE9F04168
:10668000B2F5004F9DF8188024D80446C06817461C
:106690000E461D4618B14FF0FF3100F057FF20693C
:1066A00018B14FF0FF3100F051FF0022C5F30E0387
:1066B000E06843EAC83362812660A780E3802281D4
:1066C00008B100F05FFF206908B100F05BFF012016
:1066D000BDE8F0810020BDE8F08100BF0389428958
:1066E0009BB292B28088934236BFC2EB40029B1AA3
:1066F0009B189BB2984228BF18467047028943896D
:1067000090B29BB2C01AB0FA80F04009704700BF47
:10671000038942899BB2808892B2934236BFC2EB12
:1067200040029B1A9B189BB2984286BFC01A80B247
:106730000020704738B5044600690D4618B14FF087
:10674000FF3100F003FF2189638989B29BB2A288DF
:10675000994236BFC3EB4200C81A401880B250B30A
:10676000824209D291422CBF891A89188BB29A426F
:10677000638103D89B1A9BB29A42FBD9E2882168B5
:10678000C2F30E0202FB0311284600F04DFD6189A1
:10679000012589B24B1C9BB29942A2880ED90023D5
:1067A00002FA05F15B1A9BB22069638108B100F01F
:1067B000E9FE284638BD054663899BB2B3EB420F1C
:1067C0004FEA4201F0DBEDE72DE9F04706460069AC
:1067D0008846914618B14FF0FF3100F0B7FE33897B
:1067E00074899BB2A4B2B588A34236BFC4EB4507F7
:1067F0001F1BFF18BFB2002F4AD0BD4240D3B9457E
:1068000028BFB946A5421FFA89F703D8641BA4B272
:10681000A542FBD9B6F806A02B1B31689BB2CAF380
:106820000E029F42924602FB041123D913FB02F38E
:106830001FFA83F94A4640467D1B00F0F5FC6219B9
:1068400012FB0AF2316808EB090092B200F0ECFC8E
:106850007289B58892B2D3199BB29A421AD96A004A
:106860009B1A9BB23069738108B100F08BFE3846E9
:10687000BDE8F087404607FB02F200F0D5FCE7E7F1
:10688000AB422CBF5B1B5B199CB22F467481B6E7F1
:1068900073899BB2B3EB450F4FEA4502E2DBDFE7BA
:1068A000F8B50446C0680E4618B14FF0FF3100F04D
:1068B0004DFE2589238961899BB289B2A2888B42CA
:1068C00036BFC1EB42015B1A5B189BB29A42ADB274
:1068D00008D8E779FF0905D1E06808B100F052FE59
:1068E0003846F8BD954219D32B469B1A9BB293426A
:1068F000FBD2E2882068C2F30E0202FB030031469D
:1069000000F092FC6B1C9BB29D42A28812D900231E
:1069100051005B1A9BB201272381DDE7E2882068E2
:10692000C2F30E0205FB0200314600F07DFC01358A
:10693000A288ABB2B3EB420F4FEA4201EBDBE8E7D0
:106940002DE9F04F164683B0002A4CD00546C068AA
:10695000884618B14FF0FF3100F0F8FDEA792F8931
:106960006989D209AB88BFB289B240D18F4236BFA4
:10697000C1EB4301791AC91989B2994241D2591A16
:1069800089B28E4228BF0E46B5F806A007EB06096D
:10699000A6EB030BCAF30E0A1FFA89F91FFA8BFB49
:1069A0009F423C4603D3E41AA4B29C42FBD21B1B79
:1069B00028689BB2B3420AFB04004BD341460AFB52
:1069C00006F200F031FCAA884F454FEA420302D894
:1069D000B9EB420F03DBA9EB03031FFA83F9E86865
:1069E000A5F8089088B9304603B0BDE8F08FB5F837
:1069F00006A09E42CAF30E0A0DD3002B3FD11E46BD
:106A000000E00026E8680028EDD000F0BBFD30462D
:106A100003B0BDE8F08F8F4236BFC1EB43027A1A54
:106A2000D21992B258003244A6EB030B82421FFAED
:106A30008BFB0ADB01EB03091FFA89F9A9EB0607B7
:106A4000BFB2B94218D9381A87B206EB07091FFA44
:106A500089F9A5E713FB0AF35C4414FB0AF49AB224
:106A60004146019200F0E0FB019A286808EB020120
:106A7000A2B200F0D9FBA6E7B84291DCE3E7F61A30
:106A800001EB03090AFB06880F461E464FF0000B78
:106A90001FFA89F984E700BF10B50446C06818B131
:106AA0004FF0FF3100F052FD206918B14FF0FF3177
:106AB00000F04CFD0023E0686381238108B100F001
:106AC00061FD206908B100F05DFD012010BD00BF2F
:106AD00038B50446C0680D4618B14FF0FF3100F0DC
:106AE00035FD206918B14FF0FF3100F02FFDE3793B
:106AF000E06865F3C713E37108B100F043FD206956
:106B000008B100F03FFD012038BD00BF2DE9F0477E
:106B100089460546FAF70CFA012399F8042099F9F9
:106B200005C005F12F4EDFF8D8800EF5600E9340BA
:106B30004FEA1E5EBCF1000F58F82E7003F1FF33D0
:106B400046DBC2F120018C45644631DC03FA0CF1CE
:106B500039422DD16646D5F868A199F80710BAF1E7
:106B6000000F2CD0C9072CD4BCF1000F01DB664507
:106B700027D1B3401F423CD1D9F8001082B1B446AE
:106B800001EB420931F8022B0CF1120AB2F5005F59
:106B900038BF921949450CF1010C45F82A20F1D172
:106BA0003B4348F82E30FAF7D5F92046BDE8F08788
:106BB0004FF0FF34FAF7CEF92046BDE8F0874907D9
:106BC000D2D56FF00A04FAF7C5F92046BDE8F08780
:106BD000D2F120040DD403FA04F13942264603D140
:106BE000B9E739422646B6D0013C661C03FA04F1E7
:106BF000F7D16FF00804FAF7ADF92046BDE8F08749
:106C00005C38012010B50446FAF792F9002304F12C
:106C10002F42084902F56002120D41F8223003F1BB
:106C2000120244F822300133202BF8D1BDE8104085
:106C3000FAF790B95C3801202DE9F041D0F86841AD
:106C40009DF81860121B1F2A38D84EF29F044EF28E
:106C500080054FF4003801EB410C002E18BF25468B
:106C600000EBCC0404F5435400EBCC0C052BDCF812
:106C7000DC704FEA410EDCF8CC60C4F80C800CD913
:106C80005401053B44F0A0540532052BCCF8DC4000
:106C900002F01F02CCF8D850F2D8714400EBC101C9
:106CA0000020520142EA8363C1F8DC30C1F8D850B9
:106CB000C1F8DC70C1F8CC60BDE8F0816FF0040071
:106CC000FAE700BFF0B5012504688D4024EA050409
:106CD0000460B3B3D3E901561F68DC6801EB4103DC
:106CE00000EBC303C3F8C8704FEA410CC3F8D0608F
:106CF000C3F8CC50C3F8DC400CEB01034FF0013576
:106D000000EBC30C4FF0004600EBC30E01230EF561
:106D1000865E0C1D01F108078D40CEF8106003FA65
:106D200004F4CEF8106002F01F028560BB4000F54D
:106D3000005004600EF1100E03600020CCF8D82043
:106D4000F0BD4FF480374FF440264FF4F83501EB97
:106D5000410400EBC404C4F8C8704FEA410CC4F805
:106D6000D060C4F8CC50C4F8DC30C5E703BD00BF28
:106D700010B50446FBF7CCFB2346BDE8104018478E
:106D8000F0B5054687B0192017460E46FAF7CCF93C
:106D9000002104461920FAF7B1F90021CDE9046574
:106DA00003970026002701224FF050438C46CDE97F
:106DB00000670292B9B11A6D9507FCD5596540BFBD
:106DC0001A6DD00703D420BF1A6DD207FBD59A6D78
:106DD0008A420DD04FF0000C06AA02EB8C0252F84A
:106DE000181CE7E79A6D1A6DD607FBD440BFE2E79F
:106DF0000CF1010CBCF1060FEED12146192007B0B1
:106E0000BDE8F040FAF77AB90C4B0D4A93420ED325
:106E10009C4603F2F4710B4A9268CCF8F4070A48D6
:106E2000CCF8F837CCF8FC070848FFF7A9BF4FF0BB
:106E3000FF3340F2F3719C46EDE700BF00080820E5
:106E40000000082000ED00E0616C00205D6C002077
:106E500053B94AB9002908BF00281CBF4FF0FF31C1
:106E60004FF0FF3000F08CB9ADF1080C6DE904CEA5
:106E700000F006F8DDF804E0DDE9022304B0704715
:106E80002DE9F04F099D0E4604460F46002B47D1D1
:106E90008A429446B2FA82F35AD943B102FA03FC09
:106EA000C3F120029F409C4020FA02F217434FEAB0
:106EB0001C461FFA8CFE220CB7FBF6F106FB11777D
:106EC00001FB0EF042EA0742904208D91CEB020295
:106ED00001F1FF3702D2904200F23C813946121A8A
:106EE000A4B2B2FBF6F006FB102200FB0EFE44EA51
:106EF0000244A64508D91CEB040400F1FF3202D27B
:106F0000A64500F22A81104640EA0140A4EB0E0497
:106F100000211DB1DC400023C5E90043BDE8F08F2E
:106F20008B4205D90DB1C5E9000100210846F5E7FE
:106F3000B3FA83F100294FD1B342C0F002818242FB
:106F400040F2FF800846002DE8D0C5E90047E5E79C
:106F5000002B40F0AF808A1A4FEA1C4E1FFA8CF7C4
:106F60000121B2FBFEF60EFB1620220C42EA004283
:106F700007FB06F090420FD91CEB020206F1FF3826
:106F80002CBF4FF001094FF00009904203D9B9F12D
:106F9000000F00F0DC804646121AA4B2B2FBFEF0ED
:106FA0000EFB102200FB07F744EA0244A7420FD968
:106FB0001CEB040400F1FF322CBF4FF0010E4FF028
:106FC000000EA74203D9BEF1000F00F0C9801046A1
:106FD000E41B40EA06409CE7C1F120048B4006FA1E
:106FE00001FC00FA01FE22FA04F7E6408A401F4342
:106FF00020FA04F34FEA174843EA0C031FFA87FC10
:107000004FEA1349B6FBF8F008FB106649EA06465A
:1070100000FB0CF9B1450ED9BE1900F1FF3A2CBFA7
:107020004FF0010B4FF0000BB14503D9BBF1000F3E
:1070300000F0A2805046A6EB09061FFA83F9B6FBC2
:10704000F8F308FB136603FB0CFC49EA0646B4455B
:107050000ED9BE1903F1FF382CBF4FF001094FF0D4
:107060000009B44503D9B9F1000F00F0828043460E
:1070700043EA0040A6EB0C06A0FB028C66454346A3
:10708000E14602D307D1C64505D2B8EB02036CEB4B
:10709000070C0138E1465DB1BEEB030266EB090661
:1070A00006FA04F422FA01F3CE401C43C5E9004677
:1070B000002133E702FA03FCC3F1200299409C400F
:1070C000D6404FEA1C4E20FA02F21FFA8CF7B6FBAC
:1070D000FEF00A430EFB1066110C41EA064100FB6C
:1070E00007F68E420ED91CEB010100F1FF382CBFD0
:1070F0004FF001094FF000098E4202D9B9F1000F9B
:1071000034D04046891B92B2B1FBFEF60EFB16113D
:1071100042EA014206FB07F191420ED91CEB020242
:1071200006F1FF382CBF4FF001094FF000099142E2
:1071300002D9B9F1000F16D04646521A46EA00416C
:107140000FE7841A66EB030201201746FBE6023EB6
:10715000624421E702396244C1E664440238D3E65E
:107160006444023834E7023E6244E6E70238614490
:10717000C8E7023B3E447BE702383E445BE700BF82
:10718000704700BF70B5860747D0541E002A3ED016
:10719000CAB2034601E0013C39D303F8012B9D0735
:1071A000F9D1032C2CD9CDB20F2C05EB052505EB1D
:1071B000054535D9A4F1100C03F1100E1A462CF038
:1071C0000F064FEA1C1CB644C2E90055C2E902553D
:1071D00010327245F8D10CF1010214F00C0F04F0DA
:1071E0000F0C03EB021213D0ACF1040323F00303E2
:1071F0000433134442F8045B9342FBD10CF00304C4
:107200002CB1C9B21C4403F8011BA342FBD170BDD1
:1072100064461346002CF4D1F9E703461446C0E750
:107220001A46A446E0E700BF844641EA000313F093
:10723000030349D1403A23D30B6803604B68436092
:107240008B688360CB68C3600B6903614B694361E2
:107250008B698361CB69C3610B6A03624B6A4362CA
:107260008B6A8362CB6AC3620B6B03634B6B4363B2
:107270008B6B8363CB6BC36340304031403ADBD2CE
:1072800030320BD30B6803604B6843608B688360BC
:10729000CB68C36010301031103AF3D20C3205D3F2
:1072A00051F8043B40F8043B043AF9D2043208D0C8
:1072B000D2071CBF11F8013B00F8013B01D30B883A
:1072C00003806046704700BF082A13D38B07B1D0F4
:1072D00010F00303AED0C3F10403D21ADB071CBFC6
:1072E00011F8013B00F8013BA4D331F8023B20F830
:1072F000023B9FE7043AD9D3013A11F8013B00F869
:10730000013BF9D20B7803704B7843708B78837014
:1073100060467047002301461A46184600F042B8FE
:1073200020F0030110F00300C0F1000051F8043B0D
:1073300000F1040C4FEACC0C6FF000021CBF22FAE3
:107340000CF213434FF0010C4CEA0C2C4CEA0C4CA1
:10735000A3EB0C0222EA030212EACC1204BF51F89A
:10736000043B0430F4D0C2F1000102EA0102B2FA97
:1073700082F2C2F11F0200EBD200704738B5074D10
:10738000074C2C1BA41005D0013C55F8043D984730
:10739000002CF9D1BDE8384000F040B8100A0120B7
:1073A000100A012070B4164D2C681CB365681F2D9F
:1073B00023DC38B96B1C00200235636044F82510CB
:1073C00070BC704704EB850C0228CCF888204FF085
:1073D0000102D4F8886102FA05F246EA0206C4F80E
:1073E0008861CCF80831E5D1D4F88C311343C4F866
:1073F0008C31DFE7034C2C60D8E74FF0FF30DFE73C
:1074000034160120A4140120024B13B10248FFF7E7
:1074100081BF7047000000006D720020F8B500BF0A
:10742000034600B50268EFF3108C72B6D2E8CFEFD6
:107430000120BEF1000FF9D1C2E84E0FBEF1000FDE
:10744000F4D1BFF35F8F93F90420002A0ADB01B166
:107450000A60002000221B68C3E88F2F8CF310887D
:107460005DF804FB4FF05042126801201A71F1E7F9
:107470004FF050412DE9F0410027044616461D46C5
:10748000D1F8008009E02368C3E88F7F8CF310886F
:1074900030462946FAF700FCF0B92168EFF3108C6A
:1074A00072B6D1E8CF2F0123002AFAD1C1E8423FBA
:1074B000002AF6D1BFF35F8F94F904E0BEF1000F0C
:1074C000E1DA0023226884F80480C2E88F3F8CF35D
:1074D00010880120BDE8F0810020BDE8F08100BFE8
:1074E00030B501460468EFF3108C72B6D4E8CFEFE4
:1074F0000125BEF1000FF9D1C4E84E5FBEF1000FC7
:10750000F4D1BFF35F8F90F90440002C11DB002110
:107510000568C5E88F1F8CF310884FF0504C9CF91C
:1075200000C0A44501D1084630BDBDE83040FFF79A
:107530009FBF4FF05040006800230A680871C2E8FE
:107540008F3F8CF31088012030BD00BF70B5054619
:107550000C46FAF7A9FC02460B464FF47A704FF03E
:10756000FF3E6FF0004CE4FB002396457CEB0301EB
:1075700038BF72462846BDE8704038BF6346FFF703
:1075800077BF00BF0368EFF3108272B6D3E8CFCFA6
:107590000121BCF1000FF9D1C3E84C1FBCF1000F71
:1075A000F4D1BFF35F8F4FF0FF0C0023016880F828
:1075B00004C0C1E88F3F82F3108840BF704700BF0E
:1075C000002108B5134B4FF4707299601248D960CE
:1075D000196159619961D961196259629962D962D7
:1075E000196359639963D963196459649964D964B7
:1075F000196559659965D965196659669966D96697
:10760000196759679967D967FFF7BCFD034B044AAF
:107610001A6008BD00001050E43B0120B03F01207B
:10762000800110502DE9F04F204B85B09E6D0EB3B8
:10763000002401251E4F01E0202C1BD006EA050383
:10764000621C2146AA46D4B26D00002BF4D002235E
:1076500004F001084FEA510913FB098B154B07EBA6
:107660004B1B5846C3F858A000F00AFC28B936EA6C
:107670000A06E1D105B0BDE8F08F4FF4E062ADF845
:107680000420002208EB490307EB43138DF809207F
:107690009A78DB8A01A801218DF80820039300F075
:1076A0000DFC584600F092FBE1E700BF00001150CE
:1076B000A43B012000301150F0B5B24B85B0D3F897
:1076C000985015F4003674D0AF4BB04C996A94F8CA
:1076D0003B30AF4A022B116000F0F980002694F88D
:1076E0007B30022B00F0D48194F8BB30022B00F0E9
:1076F000C58194F8FB30022B00F0B68194F83B3141
:10770000022B00F0A68194F87B31022B00F09681C9
:1077100094F8BB31022B00F0868194F8FB31022BE8
:1077200000F0768194F83B32022B00F0658194F8EA
:107730007B32022B00F0548194F8BB32022B00F014
:10774000438194F8FB32022B00F0328194F83B33F2
:10775000022B00F00A8194F87B33022B00F0C980E1
:1077600094F8BB33022B00F0EC8094F8FB33022B2F
:1077700000F0D6803EB9874B1B7823B94FF4003216
:10778000854BC3F890204FF440727E4B01219B6CD7
:1077900001A8C3F30A03ADF80420029300F08EFBA6
:1077A000EA064FF400367D4C07D5FFF73BFF26462F
:1077B00003E0EA064FF01004F7D4EB0332D5734C24
:1077C00046F48036A37E9BB10221754B6D4A196643
:1077D000536E9F07FCD54FF4405200216B4800F0D8
:1077E000FBFA6A4800F0F2FA02226B4B5A661A66FC
:1077F000012394F83A20E370FAB901234FF4C061F1
:10780000684A84F82330ADF8041092E8030004AA13
:1078100002E90300194601A800F050FB4FF40032C2
:107820005D4B1A65E9041DD46A0432D42B043FD49D
:10783000AE4240F0A58105B0F0BD594A1366A2F5ED
:107840000052536ED807FCD54FF4405200215648E1
:1078500000F0C2FA544800F0B9FA01224E4B5A66C1
:107860001A66CAE70024474B46F480561C60FFF7AF
:10787000A7FE4FF48073012101A8ADF804308DF804
:10788000084000F01BFB4FF40022434B1A656A04CA
:10789000CCD54FF48063012101A8ADF8043000F08D
:1078A0000DFB10223C4B46F480461A652B04BFD5D5
:1078B0004FF4A063012101A8ADF8043000F0FEFAF6
:1078C0004FF40062344B46F400461A65B0E794F872
:1078D0003A60002E3FF403AF94F83C30002B3FF4A5
:1078E000FEAE002304F1200084F83C3000F096FA4C
:1078F000F5E694F87A73002F3FF432AF94F87C33B6
:10790000002B40F0368194F8BB33022B23D194F83E
:10791000BA33DBB994F8FB33022B7FF434AF3E4625
:1079200094F8FA33002B3FF425AF94F8FC33002B86
:107930003FF429AF00231D4884F8FC3300F06EFAB1
:1079400021E794F8BA33002B3FF40FAF94F8BC331F
:10795000002B40F0A78094F8FB33022B7FF413AF89
:1079600094F8FA33002BE0D10DE794F83A73002F26
:107970003FF4F1AE94F83C33002B40F0F2803E46E9
:10798000E9E600BF0000115000000B40A43B0120BD
:107990009C3B0120024002200030115010000200E8
:1079A0000020115000001050C43B0120843F0120F2
:1079B00094F8FA72002F3FF4C9AE94F8FC32002B11
:1079C00040F0C7803E46C1E694F8BA72002F3FF4FB
:1079D000B8AE94F8BC32002B40F0B3803E46B0E61F
:1079E00094F87A72002F3FF4A7AE94F87C32002B03
:1079F00040F09F803E469FE694F83A72002F3FF495
:107A000096AE94F83C32002B40F08B803E468EE6DA
:107A100094F8FA71002F3FF485AE94F8FC31002BF6
:107A200077D13E467EE694F8BA71002F3FF475AEEA
:107A300094F8BC31002B64D13E466EE694F87A711E
:107A4000002F3FF465AE94F87C31002B51D13E46B7
:107A50005EE694F83A71002F3FF455AE94F83C314D
:107A6000002B3ED13E464EE694F8FA70002F3FF4CC
:107A700045AE94F8FC3063BB3E463FE694F8BA70DE
:107A8000002F3FF436AE94F8BC30D3B93E4630E612
:107A900094F87A70002F3FF427AE94F87C3043B905
:107AA0003E4621E60023394884F8BC3300F0B6F99D
:107AB00051E70023364884F87C303E4600F0AEF9AA
:107AC00012E60023334884F8BC303E4600F0A6F9A5
:107AD0000FE60023304884F8FC303E4600F09EF963
:107AE0000CE600232D4884F83C313E4600F096F920
:107AF00009E600232A4884F87C313E4600F08EF9DE
:107B000006E60023274884F8BC313E4600F086F99B
:107B100003E60023244884F8FC313E4600F07EF959
:107B200000E60023214884F83C323E4600F076F916
:107B3000FDE500231E4884F87C323E4600F06EF9D5
:107B4000FAE500231B4884F8BC323E4600F066F993
:107B5000F7E50023184884F8FC323E4600F05EF951
:107B6000F4E50023154884F83C333E4600F056F90E
:107B7000F1E50023124884F87C3300F04FF9C2E6A7
:107B8000104886EA0501F9F7BBF900BF443F012020
:107B9000043C0120443C0120843C0120C43C0120E1
:107BA000043D0120443D0120843D0120C43D0120CD
:107BB000043E0120443E0120843E0120C43E0120B9
:107BC000043F0120BC8100202DE9F043828A048B10
:107BD00003469442C07828BF1446051E18BF0125ED
:107BE00080F00100121B5E78D87092B244F480607D
:107BF0009A8240EA453006BBDD6804F1FF3805EBA8
:107C0000811C1D69ACB1B8F1050F05F1010203D962
:107C1000ACEB0207022F17D80CF1FF3C254400E023
:107C2000013212F8016CAA420CF8016FF8D11D69FB
:107C30009A8A25441D6140F400400AB940F480400E
:107C400001B10004BDE8F0832F46E6463246261F08
:107C5000B608013657F8049B013296424EF8049B51
:107C6000F8D8B4EB860FA8EB860205EB860E0CEB7A
:107C70008607DCD015F826500CF82650002AD6D0FE
:107C80009EF80150012A7D70D1D09EF80220BA7072
:107C90001D699A8ACDE700BF83680246186801B162
:107CA000000C5378C0F3090013B3F0B5D2E90354C4
:107CB0008F0105EB8113461E78B1052E04D90137DB
:107CC0003D44651B022D1CD8611E1D1813F8014B85
:107CD0009D4201F8014FF9D11469D38A0444034449
:107CE000D382138B1461834284BF00239382F0BD3F
:107CF000D38A0344D382138B834284BF00239382AD
:107D000070479E4625460021A0F1040C4FEA9C0CCA
:107D10000CF1010C5EF8047B0131614545F8047BF0
:107D2000F8D3B0EB8C0FA6EB8C0603EB8C0504EBC1
:107D30008C01D1D013F82C3004F82C30002ECBD08D
:107D40006B78012E4B70C7D0AB788B701469C4E789
:107D500010B50446836800211B68FFF79DFF636828
:107D60001B685B0002D5238B834200D010BD2046E8
:107D7000BDE810400121FFF78FBF00BF084B1B6C0F
:107D800013F0020302D18278D20901D1002070479A
:107D9000C07EA0F10200B0FA80F04009704700BF39
:107DA0000000115008B5FFF7E9FF50B1054A064B36
:107DB000906A1B68A0F54870C01AC6288CBF0020C6
:107DC000012008BD00000B409C3B01200023C0E9BE
:107DD00004338376704700BF10B5836809B11C680F
:107DE000214082B1114352050DD51A6854050CD4B7
:107DF000084A21F480641C60126C920703D40C239F
:107E0000033BFDD28368196010BD81780248F9F701
:107E100077F800BF00001150D081002030B54368D2
:107E2000002183B004461D68FFF7CEFE134B40F4DB
:107E300080521B6C13F0020FA3780ED05B060ED09D
:107E400025F0A04545F000550021204663681D60DF
:107E500003B0BDE83040FFF7BFBFDB09F0D0A38A15
:107E6000002BEDD0012120460192FFF7ADFE019AD3
:107E700025F00055024345F0A045E5E7000011500C
:107E800038B5857E044695B1FFF762FFA38A0BB92A
:107E9000284638BD2046FFF785FF20B10123237710
:107EA0000025284638BD2046FFF7B8FFF8E781785F
:107EB0000148F9F725F800BFF08100202DE9F043D3
:107EC00043788146023B0D4685B0042B13D8DFE88A
:107ED00003F0034A6A73440000217B4B1A7822F0B6
:107EE00001021A701A7822F002021A7059701A7878
:107EF00061F382021A70754B1C686369EFF310829C
:107F000072B6D3E8CF0F01210028FAD1C3E8401F91
:107F10000028F6D1BFF35F8FA26149462046FEF7E5
:107F2000BFFC00236269C2E88F3FA36983F3108816
:107F300048B94FF0E023D3F8F03DDB070AD500BE87
:107F400005B0BDE8F0832A4699F8011099F80000C1
:107F5000FCF7AEFF05B0BDE8F0835D4A137801334E
:107F6000DBB21370C7E700245A4E23463178DFF89E
:107F70006C81594F11E03B6813EB441307D0DB6968
:107F80002BB1D9F8041099F80000984731780134E2
:107F9000E4B24A1CA242234617DBA142EBD85B1A8B
:107FA00008EB4313EBE7484B1A78D607D2D51A787B
:107FB00042F004021A709EE7434B1A78D407C9D5E1
:107FC0001A7822F004021A7095E73F4C237858077C
:107FD0003AD4E378DA07BDD5032300263B4A99F863
:107FE00000101468D9F804208DF804108DF80530BD
:107FF0006369CDF80660CDF80A60ADF80E600292B4
:10800000EFF3108272B6D3E8CF0F01210028FAD126
:10801000C3E8401F0028F6D1BFF35F8F2046A2615E
:1080200001A9FEF73DFC6369C3E88F6FA36983F381
:10803000108800283FF47DAF2A469DF805109DF872
:108040000400FCF735FF85E72378002723F00403BD
:10805000237005231D4A8DF80530166899F8002015
:10806000ADF80E708DF804207369CDF80670CDF868
:108070000A70EFF3108272B6D3E8CF0F0121002807
:10808000FAD1C3E8401F0028F6D1BFF35F8F304616
:10809000B26101A9FEF704FC7369C3E88F7FB3697D
:1080A00083F3108838B94FF0E023D3F8F03DD907B7
:1080B0008FD500BE8DE72A469DF805109DF8040077
:1080C000FCF7F6FE85E700BF403701209837012016
:1080D000034002200140022038360120D40801204C
:1080E000446F547572626F396F7320496E73746197
:1080F0006C6C5F4F532E2E2E00000000446F5475A1
:1081000072626F396F7320496E7374616C6C5F4F6C
:10811000532E2E2E206E3D253034782062656769FF
:108120006E3D253034780A00446F547572626F39A1
:108130006F7320496E7374616C6C5F4F532E2E2EDB
:1081400020626567696E3D2530347820656E7472F3
:10815000793D253034780A005B4D633D256720204A
:10816000733D256720204D6370733D25675D0000DA
:1081700053797374656D20636C6F636B206F662039
:108180002575206B487A2063616E6E6F742062657E
:108190002065786163746C792061636869657665D0
:1081A000640000003A25643A0A0000003A723A007E
:1081B0003A703A003A673A000A2A2A2A2050414E79
:1081C0004943202A2A2A0A000A0000004E6F207321
:1081D00070696E6C6F636B7320617265206176618C
:1081E000696C61626C6500004E6F2075736572206A
:1081F000495251732061726520617661696C6162D8
:108200006C650000486172647761726520616C6121
:10821000726D20256420616C726561647920636CE5
:1082200061696D6564000000486172642061737368
:108230006572740052656C6561736500626F6F747E
:10824000325F77323571303830000000322E312EF7
:10825000310000007069636F32000000766572794A
:10826000747572626F730000417567203139203276
:1082700030323600666E692B00000000666E6900C1
:108280006E616E00666E692D00000000555342203D
:10829000737464696E202F207374646F75740000AA
:1082A000526173706265727279205069000000003B
:1082B0005069636F00000000426F617264204344A4
:1082C000430000005265736574000000556E6861DC
:1082D0006E646C65642049525120307825780A001C
:1082E000657020253032582077617320616C72658B
:1082F00061647920617661696C61626C650000007F
:1083000043616E277420636F6E74696E75652078A3
:10831000666572206F6E20696E6163746976652090
:10832000657020253032580087CD0D4E000DC1807C
:10833000BA001400006B65726E65EC018E002010AF
:108340008E03E04F5FED81313E26FA4C4CDD20CBB1
:1083500020DD22CB02DD46CB70DD445F4CDD269F65
:108360002832890100308CC09F243410308D0C6F6E
:10837000108E0100C629A680A7A05A26F935101034
:108380008EFF00170C40318D0CDD308DFF9A3410BC
:108390008E002CECA1E3E4ED818C003623F53262F3
:1083A000308D00F29F71308D00E99F3C308D01943B
:1083B0009F40308D01089F3E9F38308D01AD9F4218
:1083C0009F2E308D0B789F3A308D01049F6E318D3A
:1083D0000C3617072586C0308D0C88103F001025FD
:1083E0000064DF2AA6C81C850127020C75EC4E2705
:1083F0000B30CB86C0103F002502ADA49E20C6F8EE
:10840000E7844FD624501F02501705579E49103F4E
:108410003025339F49109F4B1F404AC601ED2786E8
:1084200080A72DDE2A8D212405170B5C8D1A8D2641
:108430002405170B538D1FECC81030CB86015F103D
:108440008E0000103F0520FE5FECC812270730CBDE
:108450008605103F86395FECC81430CB8603103F89
:108460008425119E4BA78826103F82A78827103F9E
:1084700082A78828393494C618200F3494C6162051
:10848000093B6E9F00383494C614BE004BAE85AFD6
:10849000633594318C194F1F8B9E4BDC42DD2EDCF3
:1084A0003EDD3833E4EF04A60D8A80A70D6EA4AD3F
:1084B0009F003A2406E6E4CA10E7E41600954F1F31
:1084C0008BAD9F003A2406E6E4CA10E7E43B53393B
:1084D0009E512727A60D85402721EE04EC448300FA
:1084E00001ED442616EE0E8D2F30C4270CA60D8507
:1084F000402706EE04EC4427EC9F510A48261096CC
:108500005F97489E4B2708A60D8A20A70D2A013B9E
:10851000318D003F2080AE443460CE003F2007E61E
:108520004C5C2702E74CEE4E26F5CE003FA60BA78B
:108530000C1A5031C4EE4E2704A14C23F6EF0EAFB7
:108540002E5F35E0318C051A5016FF4A1CAF109E85
:10855000448D239E4B27551A50E60DC47FE70DC569
:10856000202760C4DFE70D8DAF20414F1F8B33E420
:10857000109E468D013B3440AE4AE680AF4A5824F7
:108580000756AE3E270C2008C16E241BAEA5271748
:10859000AD8435401FA82402E742E6C4C4F0E7C416
:1085A000840FAAC4A7C43953C6D020E64F5FDD4B61
:1085B00020023CAF1A509E4D27F8EC0EDD4D9F4B2C
:1085C00010EE04E60D2B33C5022630E6883627214F
:1085D0005A271BEE8837272310AE8839EC6634669D
:1085E000EE6AA68836E6691F02EC6634665FE788A5
:1085F00036EC8816DD2EDC3CDD383BE60DCA80E724
:108600000DE688361CAF103F063440EC41AE4417EF
:10861000002D2404C6DD202510AEC4E627C5802623
:10862000096D42270553C6D120136C42EEE4AF44D6
:1086300010AF48EC26ED41EC2930ABAF4635C0CE4B
:1086400000001F8984F0C40F34768D4F812F274896
:108650001704032544DE263464EEC4272AEC443193
:10866000CBE6E417044E2527A6652706A84684F026
:10867000261DA6662706A846840F26133554EF66E6
:108680008D19AF624F2012EC6B2604EC63ED6B3555
:1086900064334411932825BF5335F68620A18027E3
:1086A000FCA682393440AE448D053520EF28398D43
:1086B00056254BA6063412EC04308B35028D8035DE
:1086C00010253CC6E7ACC4273CA607840F34021033
:1086D000AEC4A627840FA1E0242B3430E64226192D
:1086E000AEC49C6A2413EC02C300FF1F894F1F0213
:1086F000E6C49E20103F136F423530AFC45F39315E
:10870000C426F8C6CE4339EC84108387CD260631C3
:10871000088D15240453C6CD39967526025F393469
:108720001010AE028D0F359034304FA880AC62230C
:10873000FA81FF35B0CCFFFF340634063361A680E2
:108740008D2C313F26F86F5FA6C481802608EC414E
:1087500010830FE3270353C6E835B0AE4410AE468E
:10876000270AEE48A6808D06313F26F85F39A8C457
:108770003402EC41EDC44FE6E45849A841ED415FB5
:10878000A6E444564456A841E842ED41A6E448A870
:10879000E4A7E44848A8E4A7E448484848A8E02AF1
:1087A0000BCC8021A8C4A7C4E842E742399E4910F7
:1087B0003F30256C9E4B3410EC09ED29A60B5FED84
:1087C0002BC680E72D109F4BEC883BEDA83BEC8837
:1087D0003DEDA83D30881A31A81AC60CA680A7A086
:1087E0005A26F9C603A6803404103F8224014FA7FD
:1087F000A035045A26EF8D64251B3520109F4BA60B
:1088000084A741E623A723A6A4ED01E60DC47FE7D4
:108810000D103F2C393404103F065335149F4B394B
:1088200053C6E5398D2625121A50E60DC47FE70D93
:10883000103F2C103F2D8D1424F63404E78836E6C3
:108840000DCA02E70DC6FFE70B53358434409E4B3B
:10885000EE8812103F02EEE48D0235C09E4B34507C
:10886000DC40ED8814ED8816ED88184F5FA7883638
:10887000ED8837A641AE44103F002405103F012586
:108880006F109E4BEFA8128111270981C127055354
:10889000C6EA205C31C4EE62AF44A6425F10A32B4F
:1088A0002402EC2BC300002600103F072542830062
:1088B0000CA3462539AE48EC463406270A308BA671
:1088C00082A7A2AC4822F89E4B10AF38313410AFCB
:1088D00004A6075FED28A723AB08ED263506ED219A
:1088E000C680E7A4EE8812EC4933CBEF2A5FC6E6D8
:1088F00035D0EC41C300FF5FED419E22CC01FF3437
:1089000006200A6A61E66168E4240869E4301F9C75
:10891000202516A684A4E426EA6A61E061E14146C6
:10892000EB614925E2E6614F5C326225119E201F12
:1089300002E6414F1E028D2B1E89ED484F3953C66A
:10894000CF39EC41C300FF1F894F1F02EC4827ECD1
:108950005D270453C6D2391E899E202059EC41332D
:1089600044373034368D324D34022B0EA684AAE4BF
:10897000313F271E64E424F6A7801F20A7E486FF6A
:108980002002A780C00824FA6AE42AF6485C26FC84
:10899000AA84A7844F326135B63404445644564401
:1089A00056308B35048680C4072704445A26FC3988
:1089B000EC413344373034368DDF4334022A0EA67F
:1089C00084A4E4313F271A67E425F6A7801F2020FE
:1089D000026F8083000822F92707485C26FC43A425
:1089E00084A7846FE035B63440EC41AE4410AE4607
:1089F000EE488D083540ED4110AF463934763426C7
:108A00006F686F691F028D913402200D312110AF04
:108A10006564E4240866E43001AC6B241EA684A4DB
:108A2000E426E931211F20A36510A363241410A3B9
:108A30006923DEED69EC65ED6120D6EC61ED6543FF
:108A40002002ED69326535F6AE448D0AED4125020E
:108A5000AF4410AF4639A684812F260230013184FD
:108A60005FA6A0847F8D2825125CA63F2B0AA6A0B6
:108A7000847F8D1724F3A6A21CFE39812C2602A622
:108A8000A0812027FAA6A253C6EB39812E27438165
:108A90003025188139233B815F27378141250C819F
:108AA0005A232F81612504817A23271A0139E6424E
:108AB000334437303436A6A02B0D5A2706A88084BD
:108AC000DF27F31A0135B65A26F9A884845F26F306
:108AD00035361CFE3910AE4620201F98847F817FDA
:108AE00027088137250453C6E33958DE4633C5ECE1
:108AF000A130ABAFC42503AFC870E6A0C18026DAB1
:108B000039EC4827439E2610A384270830049C286C
:108B100025F52034A60227054AA702262B10AE848D
:108B2000109C6A2423E626C1D02509103F33240473
:108B30006C0220154F5FED84EDA4EC221701461E58
:108B4000021E899E20103F134F39109E4B9E49A64E
:108B500023260453C6E239103F2FA62D8501261384
:108B6000A62226F36F419E4B1A50DC4FED0E9F4F0D
:108B70001602299E4BA6A4E6A836ED4134723101B7
:108B80009E492003103F2FA622A1E426F7EE63E6BC
:108B900042E722103F3135F29E4BE642E78836C667
:108BA00010318826A6A027073404103F8F35045AB9
:108BB00026F2A6071F03A608103F29EE8812103FD1
:108BC00002DE4B31419E4920126F22103F2FA62D0D
:108BD00085012705A6A4103F316F21A62226EA8E23
:108BE0000041A641260D9E49A6C4103F312022A176
:108BF00084270E3184AE0E26F6A64D8A01A74D209D
:108C000010EC0EED2E103F2C31C4EE04EE4117FF98
:108C1000644F5FDD4B399E4BEC41275A8D67E0086E
:108C2000275425321F02AE073470E6E42702EB61B9
:108C30009E20DE22103F112547E762E6E42706EB7F
:108C400061E162263BE662103F12EC62A061EB61DB
:108C500035709E4B201E501F0250EB08EB07E104BD
:108C6000220453C6DF399E20103F131F20509E4B15
:108C7000EB08A607ED07A6085FED41AB07ED463907
:108C800053C6CF35F0C300FF5F1E8939A641260EBB
:108C90004C9E4BA18427028D054C26F55F399E49D9
:108CA000103F2F2408C6E03953C6E035A23422E62F
:108CB0004226119E4BEC09270510A32926EAA62D72
:108CC0008A02A72D1A50A6A83627084A270553C698
:108CD000E935A2E642E7A8368E00432026AC61269D
:108CE00022A60D8540272FEE04EC442729EE0E27FF
:108CF000253406A64D85403506271BEE44E344ED9A
:108D00004420133184AE2E26D48E00413184AE2E01
:108D10002714AC6126F6EC0EED2EA688364A260303
:108D2000A78836103F2C5F35A29E4B1A50A6883676
:108D3000270B4A2603A78836103F2C205FEC4427D8
:108D400048830001ED4427F034508E00433184AE57
:108D50000E27123406A60D854035062708EE04A31B
:108D60004424EAE3443550ED44EC2EAF2EED0EA63C
:108D70000D8A40A70DAE0E2723A60D8540271DAEF8
:108D800004EC04A344ED042013A60D84BFA70DCC6E
:108D900000431F02EC2E26FAAF2EED0E318C11345B
:108DA00020109E4BEC24AE44347F10EF24103F2D56
:108DB000ED24AF445F399E4BEC44ED8837EC48ED31
:108DC00088395F39A6419E49103F2F250E9E4BECF6
:108DD0000910A3292605A642A72B3953C6E0399EC0
:108DE0004BA684A741EC09ED465F39A641AE448D00
:108DF00006250310AF463934064D270F5F4456440D
:108E000056A6861F0227046DA42601433586AE446C
:108E100026088D10250DAF84AF448D1E2505A74172
:108E200010AF46393440CC0100103F2830C43540E3
:108E300025074F5FA78B5C26FB3934504F34025F08
:108E4000A686270B1F024F6DAB2706CB4024F81ACE
:108E50000131AB350224254C814025E14F6D862739
:108E60000A4C814025F7C6C843201E34128DB52513
:108E70001A31841F101F893512E7865F58495849F7
:108E8000C63F6FA55A26FBA7A435D0326335D0A6BE
:108E900041AE4434765F445644563402A6862718C1
:108EA0001F026FA45F1F034F6DCB260CCB4026F82B
:108EB0004C103F29A6E46F866FE035F6AE44E68499
:108EC000AE014F340134149E2AE60C9E6610AE4467
:108ED000273B6D6127625A86093D308BA6032658D1
:108EE0001A50E662E11F250DC609A682A7095A2677
:108EF000F99C6622EDEC41ED84ECE1A702E703E684
:108F0000E0E708EC46ED04EC48ED063581326410EC
:108F1000AE4810AC06270730095A26F65F393405EB
:108F20001A502007E609E7804A26F986096A612671
:108F3000F36F804A26FB3583326453C6CA39109ECC
:108F4000669E2AE60C200531295A27EEA6B4A822EF
:108F5000A52327F3EE263424ADB804352425E839BB
:108F60003476DE2A8D1424088D1E250C8D0C2508E0
:108F7000ADA43576AE3E6E8435F6308C0686C110D3
:108F80003F0039494F4D41CE3440530D7026350CCA
:108F900070ECC816272E30CB86C1103F002525ADBA
:108FA000A425219F249F6A338BDF6CEC8410838778
:108FB000CD260B103F2E2506EC02308B200230010F
:108FC0009C6C25E735C0342017F6E42506EC02300A
:108FD0008B2006C1E727063001ACE425EB35A02045
:108FE0000F1220101220111220121220131220141E
:108FF0006E9F002C6E9F002E6E9F00346E9F003679
:109000006E9F00326E9F003000F5FE03F79F05F85B
:109010001385F8220FFA3110FA9411F9CA12F93DAA
:1090200013F98D16F735A8F8C9A9F916ACF4E7AD10
:10903000F57AAEF66F32FA9D7FFF2502FAC304FB84
:109040000906FB5407FBCF08FC420AFCDC09FD665D
:109050000BFD8C0CFD6EAFFD92B0FDB2B1FE30AADF
:10906000FE5A80496E69F4014D01530159015A01BC
:109070005E0159EC829C87CD0036001EC080DD0069
:10908000FE001527002300250027002A002F0100DD
:1090900001000000696E69F40174EB67EF2F64E46E
:1090A0002F746572ED626F6FF41ED39B87CD0195AF
:1090B000000DC1816C002D000074EB0114015B15E3
:1090C000000427011180AE44EC84DD53EC02DD5531
:1090D000EC04DD57863C975D39CC3B01DD58C63C3E
:1090E000D75EC606D75FD748308D00119F32318CCE
:1090F000CB103F3234018601B7FF0335814F1F8B00
:10910000B6FF02850126046E9F00388601B7FF0274
:109110000A5D2649D6585CD758C13C2D3C96574C21
:10912000813C2532DC555CC11825284C308D01016D
:10913000D654A185231CC102260AD653C40310832A
:109140001D00270EDC535CC10D25034CC601DD5309
:1091500086015FDD554F5FDD57965E975D109E730C
:1091600027424F34022019EC848300012610860127
:10917000A7E4A60426028D518A01A704EC02ED841F
:10918000AEA126E3A6E0271C9E4B27046D0D2A18EE
:10919000AD9F003A24FA0C5C260A0C5B26060C5A9A
:1091A00026020C596E9F006E318D00046E9F007177
:1091B000AD9F003A24FA9E4BE60DC47FE70DEC8884
:1091C00016DD2EDC3CDD3820DB3430AEA1AF3C2692
:1091D000FA3530313E3934011A50109E739E2AE61A
:1091E0000CAE44271F6DA4270FC0025831A56DA4F3
:1091F00026226DA327FC3122AE46AFA410AE41104B
:10920000AF84200C30466DA42706ACA126F88DB99A
:1092100035015F39350153C6CA39AE44DC53ED849C
:10922000DC55ED02DC57ED04DC59ED06DC5BED08A6
:109230005F391F1C1F1E1F1E1F1F1E1F1E1F26F80B
:10924000B287CD070A000DC180F400130000696FDA
:109250006D61EE019E2AA60CC6093D3406A60DC618
:10926000093D3406E362C30018C300FF5F103F28C6
:10927000253030C46F8083000122F9DF66ECE130D5
:10928000CB9F64E3E130CB9F739E68103F30251283
:109290009F68103F31308D05189F3A318C08103F80
:1092A00032396E9FFFFE7F007B0105270E05C8AB9C
:1092B00005FCFF0074AA0477B3000180AE44DE2AE7
:1092C000E64DDE6410AE44270CAC44270FACC42737
:1092D0000BAC46270733495A26EA5F3953C6D139C2
:1092E000005F016901E1021802180241025E029466
:1092F000032803360367033603670382032803C585
:10930000029A003D014701D602090209021F023CF0
:109310000272030B0319034A0319034A0366030B82
:1093200003B20278308CB92003308CD6C190220B66
:10933000340458EC85308B35046E8453C6D039C65E
:10934000116FE25A2AFBEFE810A641A769AE4486E6
:10935000F0103F002524EF6410AEE810AF24EC4F6E
:10936000ED6CEC4B30CB86E0103F00250DEFE4EECA
:1093700064EC4930CB86D0103F00240EE7E811336F
:10938000E4103F8132E811533584EF669E2AE60DE2
:10939000A60DDE64AE442731AC642613AE42260D22
:1093A0003402A6482703103F2B350220E7EF6EAEAC
:1093B0004410AE0F10AC6C2610AEC4ACE4260AAE5E
:1093C00042AF626D482702A76A33495A26C6EE6E3D
:1093D00010260053DE64AE44270D33494A26F7C6F3
:1093E000CC2099C6CB2095AE6210260031EF6EAE30
:1093F000E4EC0BC300FF5F103F281025FF7EEF62F7
:109400006FC083000122F9EC6CEE626FC4ED411075
:10941000AE64AEE4EC09AD8B1025FF60EE6EC608BD
:10942000A6E5A7C55A2AF9AE44E607A669A40DAE7B
:10943000C4A40DA1691026FFAA6C4826026A48AE92
:10944000E810EF0832E8125F39EE48AE446D482765
:109450000E86FFA148102700636A481026004B9E25
:109460002AE60D3444AE426F426F43109E64AC2234
:10947000272E31295A26F7109E4BE6A4E74810AE56
:1094800044EEC41E13EC09308B3440AD0F3540AEB2
:1094900061AE84EC0BC300FF5F103F29AE61AE04E8
:1094A0003544AE446F446F456F4810AEC4EE46106D
:1094B0003F0233A4103F023384103F021702535F70
:1094C000398D1F251C3412A641A6868D0D25073522
:1094D00014E741A785393592A64117017725026C1B
:1094E00022399E4B3088264F6D8627094C811025E6
:1094F000F753C6C8391CFE398DE8250E34528D0B42
:1095000035522506E641E786A741393404E6418D08
:1095100071250C35041701C62514A6A4A7413935B9
:10952000823404C6828D5B25F635041701B03405FC
:10953000EE23103F81A6A49E68103F313585340488
:10954000E641CA808D3C25D7350417019125DFDE21
:109550004BE621C51B270BAE23AFC81A6C082602A9
:109560006A08C524270BAE23AFC8206C0826026A00
:10957000085F20BA3404C60220ABC6873404E64133
:1095800020A334409E68103F3025566C22E721AE60
:1095900044A680812027FA301FAF44E621812F277F
:1095A000169E4BC5242705AE88202003AE881A27B7
:1095B00032AE04EC04308B3420103F0F35202523CD
:1095C000A621103F80EF23251CAE44308811E68091
:1095D00033A820C1202306C61FA680A7C05A2AF997
:1095E0005F35C0C6D73404A6A49E68103F31350449
:1095F0004320EEA6418110240B9E4B3088261CFE92
:10960000A686260353C6C9398DE9240339A6418DA0
:1096100043102400C9398DDB240339A6413404C624
:10962000058D31251FE5212719EC462704E3442544
:109630000535041600A8C6F4A6E485022706C6F57B
:109640002002C6CB63E0398DAA240339A641340435
:10965000C60220CD34109E68103F2F35101025FF14
:10966000A33917FF8E240339A6413406A642A76109
:1096700035028D9B35023405E6A820C10427074D2D
:109680002706810E2715358530A82010AE44C62048
:10969000A680A7A05A26F932625F39AE23AE04EC49
:1096A00004308B20E617FF4B25B73404E6416F8565
:1096B00035042002A6418D9C25A76A226D2526022D
:1096C0008D1C6D22269B16FE65103F2B53E68836B7
:1096D000260B9E4BE6844FA62526EEE725393474EB
:1096E0008DF02516EF26A6A820AE23AE06EC093095
:1096F0008BE6E4C08386033DAD8B34058D1410AE3C
:1097000065A6A8209E4BA684A12526026F253505B7
:1097100035F23430109E4BA6A81127106FA811C641
:1097200001103F089E49103F2F6FA8105F35B0AE63
:1097300044E684AE014F340134149E2AE60C9E6642
:1097400010AE44273B6D6127625A86093D308BA6D7
:109750000326581A50E662E11F250DC609A682A706
:10976000095A26F99C6622EDEC41ED84ECE1A70252
:10977000E703E6E0E708EC46ED04EC48ED0635814A
:10978000326410AE4810AC06270730095A26F65F3F
:109790003934051A502007E609E7804A26F9860978
:1097A0006A6126F36F804A26FB3583326453C6CA4A
:1097B00039109E669E2AE60C200531295A27EEA60E
:1097C000B4A822A52327F3EE263424ADB80435240B
:1097D00025E8393440AE448D1C25186C4210AEC4C7
:1097E000EEE4AF4410AF48A626E627ED41EC293061
:1097F000ABAF4635C08604103F84256F3276CE006D
:10980000003470A766EC642602EF64A66630671029
:109810008E0009103F89253FEC84108387CD2635C3
:10982000EC69103F282530C609A680A7C05A26F942
:10983000A66630C4EE693157103F893017250510F0
:109840003F2E24C134443384EC02103F293544C1F7
:10985000E727B22002C6CD3570A6E4E7E4103F8FBB
:10986000E6E4326A11830000260143394552524F23
:109870005220232F3A300D9E4BA68828272F327571
:10988000308CE931E4A680A7A0810D26F8E6426C71
:1098900067C06424FA6A68CB0A24FACB30E7699E71
:1098A0004B30E4DE4BA6C828103F8C326B39109E3B
:1098B0004BA6A8112723A14126186FA8119E491075
:1098C0003F2F102500816FA810C601103F08DE4B06
:1098D00020129E49103F2F24D8A641DE4B9E4910EE
:1098E0003F2F256330A4A6A811271E9E49103F2FA5
:1098F0002555E64CE12C23ECE6C4E78811E684E725
:10990000C8106FA8101E2320DBA6C4A7A811A6A408
:10991000A7C8108E0000103F0ADE4BA6C8102724EF
:109920009E49103F2F251DA6A8112718A6C811A7CC
:10993000A81127106FC8119E49103F2F2506A6C8F1
:1099400010A7A8106FC81039AECAC487CD06D000C2
:109950000DD1803F029400007363E6017777772E84
:109960006E6974726F73392E6F72670D352053C62E
:10997000D739AE23AFA83BEE263420AE44103F0FBC
:1099800025EA4D2B0730A4103F0F24E010AF4435DB
:1099900020CC0100103F2825D8EF28308CBEA680AF
:1099A000A7C05A810D26F7A7C05A26FBEE2327BE73
:1099B000AE42A6A828A707AE44ECA8362712308BE3
:1099C000A62144564459495649103F802557EF2A4D
:1099D000EE424F5FEDA83DA7A83F3406AEC816275C
:1099E00013A62185402606A6018540270F32625323
:1099F000C6FA203110AFC81620121F01E6883F2694
:109A0000026C61EC883D26F210AF883D8629340255
:109A10006C62170178A662326325084A261F250367
:109A200016015F8D4034058D29358534011A50AEFD
:109A3000238D6BAE2A8D673501A62227024F398D03
:109A400024862AAE23AE02E6062B07341217013D08
:109A50003263EE2A2703103F81EE282706CC01004F
:109A6000103F294F398E00013477EE232729EE422B
:109A70002725AEC8162720ECA83D10ACC816260E28
:109A8000EDC81626126F64200EAE883D270E10AC6E
:109A9000883D26F5ED883D4F5FEDA83D35F7279EC3
:109AA000AE02E6A4A6253436A103263CBE004B3008
:109AB00088264FE18627314C811025F73420CC1BB6
:109AC0000C8D533520BE004BA601A7E49E49103FE4
:109AD0002F30A826E6614FE18627074C811025F735
:109AE0006FE4A6E4AE62A70335B6A6A83F1026022F
:109AF0002AAE26A602261D34328628A702EE063498
:109B0000408D1135403532A702EC06EF062503EDF6
:109B1000A8345F39C609AE23EE023406AE84EC09E0
:109B2000308B35063460AD8535E01701C88D26349D
:109B300005170172358581A126DC3470BE004BA665
:109B4000463402A680A7C0313F26F8A6E42B04863F
:109B50000DA7C535F2C60CA64226DBAEA8273430C9
:109B6000AE4431A820C61AA680A7A05A26F93530DF
:109B70003410ECA82710A3E12708EE23EE422702B9
:109B8000E747AEA834862834128D0235923470AE81
:109B900026EE06A6023472ECE810ED06A66FA702C8
:109BA00017015717FF873572EF06A7022405C1D0AA
:109BB00027014335F017013D2401396C2CAE4627AF
:109BC0007234108E0000EE288D6B250A4D274CA1B3
:109BD000A82C263FC6D3326234048D5153358416E7
:109BE000FD9016FD8D16FD8616FD8316FE4F16FEA2
:109BF0004C20C21216013B16008E16013116FEEAE9
:109C000016FF2716FE251F105D26048D50EE288DA9
:109C10002425C3E6A8242703170233C6013AA7C0A8
:109C20002705A1A82B2704ACE425DB32628D2EEE9C
:109C300026AF4620713470AE232720EE2A2707EE88
:109C400042E6A828E7471F30EE02ED494FA745340A
:109C500006AE84EC09308B3506AD0335F03430ECBC
:109C6000E427235D26014A5FEE26EE4433CB4FE620
:109C70006126014C3406AE2835203440A680A7C0AA
:109C8000313F26F8354035B08D6B240139EC46273D
:109C9000154D2703CC01003406CCFFFFED2D8E00BF
:109CA00000EE281601DDBE004BA684AE238D02AE69
:109CB0002A2709AE02A10426034FA704393412AEA5
:109CC00002E604271AE1E427298DDB1F98103F2BB9
:109CD0006C2FBE004BE68836A6E427E3433592A7F7
:109CE00004A703A6A82FA70DECA830ED0BECA8380D
:109CF000ED0F4F3592A6A83F261FBE004B4FA72F52
:109D0000A684AE238DB7250EAE2A27048DAF250677
:109D1000A62F26E1A72CEE26393262C6DC81022569
:109D200007A625C600103F086CA83F1A01398DC54B
:109D300020048DC16C2CAE461027008234108E009A
:109D40000020051F305D263434301F10EE26AE444F
:109D5000308BEC46A3E4108300202303CC00203496
:109D600006EC284CA3E41F03860DA75F3520344082
:109D7000A680A7C0313F26F835403530A6C0E62C76
:109D80002618E6A82127028D38810A260D860DE6C1
:109D9000A82526068D3E2534860A8D38252EC60137
:109DA0003AACE42413E62C1026FF98A65F1027FF98
:109DB00092A1A82B1026FF8B3262EE26AF4616FE2C
:109DC000E581612506817A220280203932623405DC
:109DD0008DE835853472AE23810D267CEE02E6488F
:109DE0002620E62C262CE6A82727276A472623C606
:109DF000FFE74820163470AE2A2705EE2316FE3FF3
:109E000035F08DF12505A1A82F26F78DE8A1A82F03
:109E100027F9EE024FA748860D8D1EA62C2618E6C0
:109E2000A8263404A6A8252706860A8D0C25064FE9
:109E30006AE42AF74F326135F2EE0234305FE745CB
:109E40003406AE84EC09308B3506AD0635B034727D
:109E5000AE2A2715810D27BAEE025FE7453406AE1C
:109E600084EC09308B3506AD0635F2E6A8242601D0
:109E700039812024D9810D27D53402862E8DCF3506
:109E8000828DEE17FDAF102501204D102700A1E6B1
:109E9000A82DC10410270098A1A82D261AAC2D27A3
:109EA000E2C6013AACE4240BA6C027D5A1A82B2614
:109EB000D0335F301F20CC811326193440170105A1
:109EC000A6A83211A3E42708335F301F8D8020F34A
:109ED000326220AF8111261934401F30C6FF1F03A4
:109EE000A6C2A74111A3E426F78620A7C4326220A8
:109EF000CA811026233440A6C4A1A82B2716A64148
:109F0000A1A82B2704A7C020F58620A1C42603A65C
:109F1000A82BA7C4354020A3A1A82B26133440208A
:109F2000093402862017FF263502A1C026F33540EA
:109F30004D270BC629A1A5272D5CC13123F7AC2DD8
:109F40002302AF2DC6013AACE4250BA6A83317FEB9
:109F5000FD301F16FF2DE6A821270317FE63A7C0BB
:109F600017FF0816FF1D3490308C0DC029583AAFEA
:109F7000623510ADF116FF0B207F2064200C2020ED
:109F8000203620413912205820563262A7C417FECD
:109F9000DAEE26C6013AAF4617FCC2326216FD065B
:109FA000326230841027FC2C20943404860DA7C420
:109FB00017FE9B350416FC1EA6A82BA7C48E000016
:109FC000EE2817FEACAC2D2714C6013AAC62240B68
:109FD000A6C027EEA1A82B26E9335F301F398D1DBF
:109FE00030842712E6A82327F5E6A8242705860D46
:109FF00017FE5B8E0000EE2839308427E0335F3097
:10A000001FE6A82427F2E6A82227078D0586201739
:10A01000FE3CA6A83216FE3653DFA087CD0107000E
:10A020000EE180DC0013011F03736376F401160058
:10A030001D160039160074160076160091EC41C307
:10A0400000028E0000318D0087103F2A5F393420D6
:10A05000EC41C30002308D00C3318C74103F2A35AF
:10A06000202509B6FF038A02B7FF035F3930C90014
:10A070009FE6C9009E1A10E1C9009D270C3AA684EC
:10A080008D22E7C9009E1CEE39A644A7451CEF8E21
:10A090000000103F0A6F459E4BE6883627CFC1046B
:10A0A00024CB43395CC17F23015F39B7FF005F399F
:10A0B00081062714AE268101260EA6C9009DA0C9DF
:10A0C000009EA702102700025F3953C6F6395F3998
:10A0D000AE41A60284FDA702A601E6C9009D30C9D3
:10A0E000009F3A17FFBEE1C9009E2704E7C9009D03
:10A0F000A784271CA14D2608AE492714A7082010C5
:10A10000C603A14B2706C602A14C2604A643200481
:10A11000C601A6452703103F086F453900020A36DD
:10A1200037E787CD003C002EF187D1003200354360
:10A13000FFFF001C00000100010100001808180DBD
:10A140001B040117030508070002002E0000501829
:10A15000746572ED7363E6736376F4FA6FBE87CD50
:10A160000032000D11811A001000C867EF01308C19
:10A17000178D088E0000103F0A20F84F5F108E00E8
:10A1800000103F03103F04397368656CEC1668A932
:10A1900087CD060F000D118020002B03007368652A
:10A1A0006CEC160000000000000000000A53686517
:10A1B0006C6C0D0A544F533AD70E3B327B3436C683
:10A1C0006F17012F308CF1103F093516DD06270976
:10A1D000170126256B0D0C266610EEE1308CCD0D97
:10A1E0001226118D64255F308CC9108E00050D126A
:10A1F00026028D594F30C870108E00C8103F8B2436
:10A2000011C1D327310D0F26040D142633103F0E34
:10A2100020D5108C0001220A308DFF98108E00048A
:10A2200020CC0D1327028D211700CE24BA5D26D530
:10A2300020B5656F660D0D122605308CF58D0A5F11
:10A24000960F10260269103F06108E0050860210ED
:10A250003F8C391702DB102502113410C60E30C8AE
:10A2600016862FA7804F103F8D3510102501FC0C4E
:10A270000F0C101701F50F103901E3AA0360D70185
:10A28000BF4348C401B64348D8018B45D804D44BDA
:10A29000494CCC01C1D801C22DD801AAD001AA2DA8
:10A2A000D001ABD401AC2DD404E553455450D2FFBA
:10A2B000A449BD012CBB00000455A102FBBB031146
:10A2C000A602EE8D02693C3E3EBE02793C3EBE02D5
:10A2D000673CBE027D3E3EBE01FB3EBE01F2BC01BC
:10A2E000FBBE02ABA300000D2829FF0D2123263B56
:10A2F0003C3EFF6FC55A2AFB39C60E8DF60F030F81
:10A300000E318DFF741700852552810D274E970C55
:10A3100081282624318DFE85109F0430019F080C72
:10A320000D318CC38D7F812827F5812926260A0DC2
:10A3300026EF860DA71F20048D252520318CAC8D9E
:10A34000641F109308DD06301F318DFF6B8D3E2595
:10A350000B109E041026014C810D26A116010C9FA6
:10A36000048D0F250C8D0B24FC318DFF578D1E9F06
:10A370000839103F0F240CA680812E260AA18027C1
:10A3800004311F30A44F3953301FC6D7398D3034B4
:10A39000208D4F2509ECA4ADAB352024F0394FA614
:10A3A0008435A035203420A6806DA42BF68122268A
:10A3B00008A680812226FAA680A1A026EC35A0342A
:10A3C00010A6808120270E812C270A308DFF1CA12A
:10A3D0008022FC359032628620A18027FC301F1C31
:10A3E000FE3934303122AEE4A6808161250280201E
:10A3F000A8A048260F24F1A63F81C125048DC025C1
:10A40000034F35A6313FA6A02AFC10AF62ECA1266F
:10A41000D55335B017FF484F8D1C8D198D178D3CC6
:10A4200030011F109308DD0632C900FF1701E61046
:10A430003F0516FE0B4C340220578684200286818D
:10A44000103F86394F20028601971239860120017C
:10A450004F971339860120014F971439860DA1803B
:10A4600026FCA1823934078601200434078602972E
:10A47000114F8D094C911123F966E0358634020D98
:10A48000102B16260C6DC62713103F8FA6C6103F43
:10A4900082E6E4A6C527056FC5103F8F3582574871
:10A4A00041543F0D8DC5308CF517FD9D5F43390C30
:10A4B000108DB886FF97108DAC30C8168D7C102596
:10A4C000FD8486028DB71700910F1016FD0ECC008B
:10A4D000012019CC020DE71E20028601C602200CC5
:10A4E0006DC626C034060D102B1A200A6DC626B480
:10A4F0003406C60DE71F103F82252BE6E4A7C5A64C
:10A50000E4103F8FA6612B07E6E48D534D2A0784A4
:10A510000F103F82200E85022605103F842005C6BD
:10A520000B103F83E76135864FC60320B3860DA726
:10A530001C8D07242539860DA71E8DEC25F7CC012F
:10A5400080209D860DA71D8DDF25EACC02802090FE
:10A55000860DA71D86018DD125DBCC02812081349B
:10A5600016EC8110832F30252210832F32221C34C9
:10A570001617FE4B35162513C403E1612604E66168
:10A58000E6C5CA80E7E435063262393596C60DE77E
:10A590001FD6031026FF0D1701D5884B84DF260A2E
:10A5A000300186043D4D1026FEFAD70316FE10300A
:10A5B0001F170094200317008B251117FEAD8D1D6A
:10A5C000250A17FDFA810D260232645F16FE9C8D66
:10A5D0007325F98DF7C62617016020E44F34021069
:10A5E0003F040D0E2711D60EC1022623A6E4271F15
:10A5F000103F086FE420E8251AA1E427126DE42734
:10A60000035D27DB34048DC4C62D17012D35045D91
:10A6100027014335828611D6039E04109E06DE086C
:10A62000398604103F84256630C85E108E000D10F8
:10A630003F893405103F8F3505102500C7A6061049
:10A64000AE0B2021860DA71F34704F9E043440109E
:10A650003F00354025CB9E043476103F00103F026A
:10A66000103F0235768111274C109F0A308DFB3345
:10A670006D841027008CA18027066D802AFC20F0B5
:10A68000DC089304D306DD06DC04DD0820259E06E5
:10A6900030059F069E04EE6417FE332567DE08CC66
:10A6A0005820EDC3CC5020EDC3C62DE7C2DF0830E3
:10A6B0008DFAEA9F049E0486113440103F001F3239
:10A6C0003540240B3440103F011F323540253510F2
:10A6D000AE2B0D0326091F20D30AC300FF970317D3
:10A6E000FF33103F03340725068E0001103F0A8612
:10A6F000119E040F040F05103F00103F02103F028F
:10A7000035F7C6EA4335F02F706970650D341030A7
:10A710008CF5CC010317FDC83510255217FF2525F0
:10A720004DA6C42607103F822544A7C44F103F8F73
:10A730008601103F82860116FD4334363434306181
:10A74000C62F5C806424FBE780C63A5A8B0A24FB40
:10A75000E7808B30C60DED8430E417FAEC326535B6
:10A76000B68D0CC10223231F98C600103F08395F25
:10A77000A6808030810922093402860A3DEBE0245C
:10A78000EFA68225035D26E6326216FD178DE0D71F
:10A790001517FC2B8DD99615103F0C39F4145087E2
:10A7A000CD0128000D1180000048021F6D66726502
:10A7B000E5010A204164647265737320207061674B
:10A7C00065730A2D2D2D2D2D2D2D2D2D202D2D2D6B
:10A7D0002D2D8D0A546F74616C2070616765732034
:10A7E00066726565203DA0314D109F0B318CC38D85
:10A7F0006A8D73BE00209F00BE00229F024F5F97AC
:10A8000005DD06DD08D70A9E00A6808D159C022571
:10A81000F88D1F318CBD8D43D6058D5F8D485F103F
:10A820003F068D008D008D004825070C050C0A0C95
:10A8300006393406D60A2719DC088D74862D8D66F4
:10A84000DC068300018D698D538D51D60A8D2C8DC8
:10A85000150C06DC06DD080F0A3586A6A4847F8D5C
:10A8600045A6A02AF6393432860D8D3A304D9F0B1D
:10A87000108E00508601103F8C35B286FF0F044CBD
:10A88000C06424FB8D0D860A4ACB0A24FB8D041F6D
:10A89000980C044D270297040D04260286F08B3095
:10A8A000813A25028B0734109E0BA7809F0B3590B1
:10A8B0000F048D021F983402444444448D02350233
:10A8C000840F20CFF947B587CD01BD000D118095CC
:10A8D000007902236D6469F2070A20204D6F6475C8
:10A8E0006C65206469726563746F7279206174A00D
:10A8F0000A416464722053697A6520547970205249
:10A900006576204174747220557365204D6F6475AF
:10A910006C65206E616D650A2D2D2D2D202D2D2D40
:10A920002D202D2D2D202D2D2D202D2D2D2D202D8B
:10A930002D2D202D2D2D2D2D2D2D2D2D2D2D2D0D74
:10A940009F040F06CC0C30DD0F318DFF8C30C81109
:10A950009F071700EE3049103F14304C17010517C0
:10A9600000ECBE00269F00FC0028DD02301C109E7B
:10A9700004ECA0C4DF10832D452633308DFF711009
:10A980008E00508601103F8C9E00206C10AE8427F4
:10A990001DEC2431AB1700AB170095D608C012D1BF
:10A9A000102208D00F22FC26EF20031700A030044D
:10A9B0009C0225D8170097204310AE842738EC84DA
:10A9C0008D3EEC228D3A8D68A6268D3E8D62A6279F
:10A9D000840F8D36E62786728D6286778D5E86338C
:10A9E0008D5A863F8D568D488D46A6028D1CEC24CF
:10A9F00031AB8D4F8D5830049C0225BD5F103F0652
:10AA00000C060C068D080A061F988D0220220C06E3
:10AA10003402444444448D043502840F26040D0658
:10AA20002E0C0F068B30813923088B0720040A0671
:10AA3000862034109E07A7809F0735905925F386FE
:10AA40002E20EFA6A4847F8DE9A6A02AF639343201
:10AA5000860D8DDE30C8119F07108E0050860110C4
:10AA60003F8C35B28D068D00863A8DC6E680C06477
:10AA700024FC863A4ACB0A24FB8DB71F988B3020E2
:10AA8000B15DEFCB87CD0279000D11805200D00B64
:10AA90001570726F63F30A0A5573722023202069C0
:10AAA000642070747920737461206D656D207072FC
:10AAB00069206D6F640D2D2D2D2D2D202D2D2D2018
:10AAC0002D2D2D202D2D2D202D2D2D202D2D2D2DDD
:10AAD0002D2DAD20616374A020776169A020736C77
:10AAE00065A00A5573722023202069642070747950
:10AAF000202073746174652020206D656D20707254
:10AB0000696D617279206D6F64756C650D2D2D2DE9
:10AB10002D2D202D2D2D202D2D2D202D2D2D2D2D8C
:10AB20002D2D2D202D2D2D202D2D2D2D2D2D2D2D6F
:10AB30002D2D2D2D2DAD202061637469766520A00B
:10AB4000202077616974696E67A020736C656570F9
:10AB5000696E67A00F00EC80C4DF10832D452602CC
:10AB60000C00304C9F0A1A50BE004D9F01BE004F92
:10AB70009F03BE00519F05BE004BEC09DD0734402A
:10AB800033C9095386019E0117012786029E0317C8
:10AB9000012086039E051701191CAF4F5F3606364C
:10ABA000063540318DFF3B17007517007D318DFF55
:10ABB0005C17006B17007330C909533017EC052779
:10ABC0005AEC071700B5170099E6841700711700B3
:10ABD00091E603170069A604318DFF5A8101270C05
:10ABE000318DFF5C81022704318DFF5E8D31E602DD
:10ABF0008D4D8D6E10AE05EC2431AB8D228D6386AC
:10AC00003C8D63A6011700D8250C10AE2310AE248E
:10AC1000EC2431AB8D098D1216FFA05F103F06A604
:10AC2000A4847F8D41A6A02AF6393432860D8D3654
:10AC3000304C9F0A108E00508601103F8C35B20FA9
:10AC40000986FF4CC06424FB8D0F860A4ACB0A2478
:10AC5000FB8D061F988B30200D4D270297090D099B
:10AC6000260286F08B3034109E0AA7809F0A35900A
:10AC7000271003E80064000A0001FF3436308CF02E
:10AC8000108E2F2031A90100A38424F8E38134061B
:10AC90001F206D842B16108E2F3010833020260637
:10ACA000108E2F2086208DBE350620D88DB83262BA
:10ACB00035B6342630842726EC090D00260510937E
:10ACC0000726173606A60BE6E410AE88123626A62F
:10ACD000083602A684E688263606AE0E26DA35A6A3
:10ACE0003416BE00684D270F5F44564456A6861F93
:10ACF0000227046DA42601433596022E2F87CD002E
:10AD00004D000D118064001300C8736C6565F0027E
:10AD10004F5F8D118D0F8D0D8D0B8D091F01103F14
:10AD20000A5F103F063406E684C0302518C10922A8
:10AD30001430013404C60A3DE761A662C60A3DEB41
:10AD4000E0A9E4EDE4358606BE4D87CD5A29001B07
:10AD500011804C0775200000DD1C71251731903BD8
:10AD6000744FE80000426173696330B916070C2024
:10AD70002020202020202020202020424153494311
:10AD800030390A20202020203638303920564552CC
:10AD900053494F4E2030312E30312E30300A434F40
:10ADA00050595249474854203139383020425920AF
:10ADB0004D4F544F524F4C4120494E432E0A2020B4
:10ADC000414E44204D4943524F574152452053591B
:10ADD0005354454D5320434F52502E0A20202052A9
:10ADE0004550524F445543454420554E444552200A
:10ADF0004C4943454E53450A202020202020205412
:10AE00004F2054414E445920434F52502E0A202087
:10AE10002020414C4C20524947485453205245531E
:10AE200045525645442E8A3416E6F804308C08EC18
:10AE300085308BAF6435960E57115B075C07521750
:10AE40009C0D390D330D551A8111CB18900FD50E6D
:10AE5000EA0F720F77007202010150415241CD0298
:10AE600001545950C503014449CD0401444154C122
:10AE7000050153544FD006014259C5070154524FA2
:10AE8000CE080154524F46C6090150415553C50AD8
:10AE9000014445C70B015241C40C0152455455525F
:10AEA000CE0D014C45D40F01504F4BC5100149C682
:10AEB0001101454C53C51201454E4449C613014684
:10AEC0004FD214014E4558D415015748494CC51668
:10AED00001454E445748494CC5170152455045411C
:10AEE000D41801554E5449CC19014C4F4FD01A017A
:10AEF000454E444C4F4FD01B014558495449C61C40
:10AF000001454E44455849D41D014FCE1E014552BE
:10AF1000524FD21F01474F54CF2101474F5355C2C3
:10AF200023015255CE24014B494CCC2501494E50AA
:10AF300055D426015052494ED427014348C4280114
:10AF40004348D829014352454154C52A014F504531
:10AF5000CE2B01534545CB2C01524541C42D015701
:10AF6000524954C52E014745D42F015055D43001C4
:10AF7000434C4F53C53101524553544F52C53201D2
:10AF800044454C4554C5330143484149CE340153EF
:10AF900048454CCC3501424153C537015245CD3966
:10AFA00001454EC44003425954C54103494E5445DE
:10AFB0004745D24203524541CC4303424F4F4C4593
:10AFC00041CE4403535452494EC74503544845CEDD
:10AFD000460354CF4703535445D0480344CF490355
:10AFE0005553494EC73D0350524F4345445552C5F2
:10AFF0009204414444D2940453495AC59604504F94
:10B00000D397044552D298044D4FC49A04524EC46B
:10B010009C045355425354D29B0450C99F04534936
:10B02000CEA004434FD3A1045441CEA2044153CE39
:10B03000A3044143D3A4044154CEA5044558D0A849
:10B04000044C4FC7A9044C4F4731B09D045347CE21
:10B05000A6044142D3AA04535152D4AA045351D254
:10B06000AC04494ED4AE044649D8B004464C4F41D6
:10B07000D4B20453D1B404504545CBB5044C4E4F23
:10B08000D4B6045641CCB7044C45CEB8044153C3A2
:10B09000B9044C414EC4BA044C4FD2BB044C584F77
:10B0A000D2BC04545255C5BD0446414C53C5BE04E0
:10B0B000454FC6BF045452494DA4C0044D4944A451
:10B0C000C1044C454654A4C2045249474854A4C341
:10B0D00004434852A4C404535452A4C604444154E3
:10B0E00045A4C7045441C2CD054E4FD4D005414EAE
:10B0F000C4D1054FD2D205584FD2F7035550444121
:10B1000054C5F803455845C3F9034449D2400000EB
:10B1100000FD4900FD4D00FD5000FD5200FD5500B1
:10B12000FD5800FD5A00FD5D00FD6100FD6500FD5C
:10B130006700FD6900FD6E40000000FD6D00FD70C0
:10B1400063FD7102FD7401FD78220FD801FD7D625F
:10B15000FD8101FD8802FD8D01FD9162FD9402FDDE
:10B160009A63FD9F00FDA500FDA6200F69200F66D4
:10B17000200F5D200F5A200FA100FDAD00FDB00093
:10B18000FDB400FDB800FDBA00FDBC00FDC100FD2E
:10B19000C400FDC700FDCA00FDCE00FDD000FDD2F9
:10B1A00000FDD600FDDC00FDE100FDE5200F5E2086
:10B1B0000F5B200F91200F8900FDE8200F1E200F4C
:10B1C0001B400000200F8640205C200E1210FDD88E
:10B1D00010FDDB10FDE110FDE410FDEA200F5060D2
:10B1E000FDF260FDF300FDF600FDF7200F7A402C24
:10B1F00000403A00402800402900405B00405D00CC
:10B20000403B20403A3D403D004023002015E820CF
:10B210000E82200E7F200E7C200E79200E76200ECE
:10B2200073210E70220E6D230E6A200E63210E60B4
:10B23000220E5D230E5A260E92270EA0240E6E2497
:10B240000EAB270EBD11FDAC80000011FDAC8000DF
:10B250000010FDAC10FDAE12FDB012FDAD11FDAF42
:10B2600010FDB912FDAE11FDE611FDE311FDB111A6
:10B27000FDB311FDB511FDB711FDB911FDBB11FDF8
:10B28000BD11FDD011FDCD11FDB911FDBB11FDC9E1
:10B2900011FDC611FDCE11FDCB11FDCD11FDCA1161
:10B2A000FDCC11FDC911FDCD11FDCA11FDCB11FD64
:10B2B000CE11FDD111FDD311FDD512FDD712FDDA4E
:10B2C00012FDDC10FDDF10FDE211FDE611FDE813BB
:10B2D000FDEC12FDEF12FDF311FDF811FDFB11FD68
:10B2E000F810FDFB11FDFF800000800000800000D1
:10B2F00080000080000011FDF2512D00512D000A48
:10B30000FDEE09FDF009FDF14B3E004B3E004B3ECA
:10B31000004B3C004B3C004B3C004B3C3E4B3C3E0E
:10B320004B3C3E4B3C3E4B3D004B3D004B3D004BB0
:10B330003D004B3E3D4B3E3D4B3E3D4B3C3D4B3C33
:10B340003D4B3C3D4C2B004C2B004C2B004C2D001E
:10B350004C2D004D2A004D2A004D2F004D2F004E40
:10B360005E004E2A2A200D2C210D29220D26230DA8
:10B3700023200D1C210D19220D16230D130002028E
:10B380000374A402C78D000E0207E14259C502B73B
:10B390004449D20F05454449D40EFFC5065D4C49CA
:10B3A00053D4071B5255CE07EE4B494CCC063E53A7
:10B3B0004156C5040C4C4F41C4037452454E414D97
:10B3C000C50489504143CB024C4D45CD03534348FE
:10B3D000C403524348D8000202031BA409AC8D00E9
:10B3E0000E0209B5434F4ED4025D4449D20979D1CA
:10B3F00009F14C4953D40A9E5052494ED40B105374
:10B40000544154C50A9054524FCE0A8A54524F4662
:10B41000C60A834445C70A7E5241C40A794C45D4C2
:10B420000959535445D00B0B42524541CB000802F9
:10B430000F77CC0F74EC127AC41277E40EB2AB0E15
:10B44000AFAD0EAC8D0EC3A0000402101BD3101BB9
:10B45000C311A3D21255D10E52656164F9576861C8
:10B4600074BF20667265E550726F677261ED50526D
:10B470004F4345445552C50D0A20204E616D65204D
:10B48000202020202050726F632D53697A65202080
:10B49000446174612D53697AE55265777269746508
:10B4A0003F3A200E425245414B3AA06FEB44BA4519
:10B4B000BA42BAA6631F8BD73508344306343B34EF
:10B4C0004033C901004F5FEDC311A3E422F93506F3
:10B4D0003384DD004C97D9DD80DD828B02DD46DDD3
:10B4E000444C1F04DD0434101F014FA7805C26FB71
:10B4F0001F10DD08DD4A1F309300DD02C601D72E84
:10B500008603103F8F4C811025F88602103F8297EA
:10B51000BE308C9F103F09308DF82F34109E0030C4
:10B52000881B318DF831867EA780ECA1E3E4ED81A4
:10B53000ECA426F232628D1F3520308DF91A9F9EC1
:10B54000E6A4C10D275A308C1134208D1D17073EFB
:10B55000243717026A20329D240035208D099E046D
:10B56000EC84DD2F170556308C4235408D25344054
:10B570000F34DC00D3029308930ADD0C3362DF46FC
:10B58000DF4432E9FF026ED8FE10DEB73506DDB7C4
:10B5900016051EDCB7340610DFB7EC62AF621F057C
:10B5A000308DF7CA8D24308DF7BB8D1E8DB9308D4F
:10B5B000FEA68D16308DFEF9318DFDC40F848D0DE4
:10B5C00024C78D0220C3308DFE9316099D34300FA1
:10B5D000351709A28DBA96BD2705103F8F0FBD17ED
:10B5E0000245240EC1D32628CC6279EDA4CC650D8A
:10B5F000ED22AE6286808D15260D1701BF27113012
:10B600000386208D082709EC8432646E8B9D1E040E
:10B610004335B0170174261F30A4DC08D30A4C93BD
:10B62000003406170E2B251910A3E12516103F072D
:10B630002505830001DD02170477DC028D771609EA
:10B640002E3262433930A417040C308DFE2A1709BC
:10B6500019109E042040343086206D062702862D66
:10B66000170A1886209C2F2602862A170A0DEC043A
:10B67000308B1709EDCC11028D2ECC1C0B8D29ECD3
:10B680000BC3004010930C2505863F1709ED8DAEC6
:10B6900035300D352604AEA126BCDC0C8D17308D5F
:10B6A000FDC01708C71603A03404C6101709F935E2
:10B6B00004AE62EC8534363406318C2C8E2F003586
:10B6C0000630890100A3A424F8E3A13406ECA41FEA
:10B6D00010270E1083300027E317099F8E2F0120BB
:10B6E000DE170997326235B6271003E80064000AB6
:10B6F0000001000017009333A45F5CA6A0810D2613
:10B70000F94F1F02308DF88786015F103F032570C7
:10B710003402103F04A1E426F932615D26623986C5
:10B72000812002868430A4103F862554398D681705
:10B73000053925523410AE846D06264A8D4C2703F8
:10B740005335908D7727F9342017051F2504AC62F7
:10B75000262CAE62170FEF3510109E4AA680A7A0C8
:10B760002AFA109FABAEF1EC04318BE6881896A64E
:10B77000A788184F170F50D35EDD5E160F2DC62C0D
:10B7800017080F16FE03C62B20F6E6A0C12C2706CD
:10B79000C1202702313F398D23260E109E2F270509
:10B7A000EC2431AB39318DFCBE39C62B2008C620C4
:10B7B00034048DC73504C1D327C920C49D1E02306F
:10B7C000A48601103F8425EE97BD8D5B8D6826DA37
:10B7D0008DEA27D63420170492250810AEE4313FB5
:10B7E0001703B210AEE4170411170F5A35101707DC
:10B7F00079D63526BB8D3025B7960C810225AF8DC5
:10B8000035270C109E80DC60DD5C170B0320E29E68
:10B81000803430A680810D26FA9F809F828D32353C
:10B82000309F809F8220A996BD9E80108E010010BF
:10B830003F8B109E80398D84308DFC32A680A8A06D
:10B8400084DF26056D1F2AF44F3917012DDE4620AF
:10B85000249D210210AEA46D2610260308A6A81769
:10B860004610250300EC2D31ABEC3D58494C1093AC
:10B870000C102203F110AEC326DACC06071701E242
:10B88000109E46DF461600E93420170EB90FD98DF9
:10B89000C00CD99E623184DC00D3021F03EC1D274B
:10B8A00072344034063001EC8436066F806F80A617
:10B8B000802AFC350683000126E9109E5E200DECEF
:10B8C000A49E62308BEC0110AF01EDA1171009248A
:10B8D000EE35409E62EC1D3184335E34464FEE01FE
:10B8E000271D34101F2093622004EDC43384AEC49E
:10B8F00026F8EDC43510A684A7A0EEF802EFA1301B
:10B9000003E68081A02602E7A05D2AF53546830084
:10B910000126C69E2FEC02340631231F20932FED03
:10B9200002ECE4A302EDE4D30CDD0CDC0AA3E1DDC0
:10B930000AD308DD4AC622E706C680E78817333DEA
:10B94000CCFFFFEDC4A742C607A8855A2AFBA7086B
:10B9500010AE02313D103F1763C063C063C010AE2C
:10B96000028602103F8A86C0A788171025013D3540
:10B9700020AEA31026FF111600CE8D18A6A4810DAF
:10B98000260F9E46AE98FEEC04308B1706D41706A1
:10B99000E830A439DE46DF4417FDEF2720C12A2610
:10B9A000219E04EC8427041F103002EDC326F4DF2F
:10B9B00044A6A4810D27023121109F823917FDFC76
:10B9C000260E109F8217FDD31702A0240B16FDB67A
:10B9D00017029825F8109F82AFC3109E8217FDAA08
:10B9E000260517FDD726E94F5F20C00D0C10270252
:10B9F00075868097848D8320048D9930A49F5C8DFB
:10BA000055109E46DF462038342010AEB4109F2FCC
:10BA1000EC29D32FDD5EEC2FD32FDD60EC2DD32F5F
:10BA2000DD626D262618308C0917FB671703B216E6
:10BA3000FB570D842B08AEF4170D0B17FE133520A2
:10BA4000AEA326C48D0220E734048602103F8F96F1
:10BA5000BE103F82358417FD31C10D274E9F82CC29
:10BA6000020B34568602103F8FECE4103F832439DA
:10BA7000C1DA2638ECE4AE62103F84252F308DFA0F
:10BA800018108E000A96BE103F8C4F30E3108E00C7
:10BA900002103F8B3506885984DF26A8CC02028E1F
:10BAA00000003384103F8E250335E6398D9A16FC4D
:10BAB000CF34068601977DDC80DD82358617FCFC5D
:10BAC0002613342017FCD0AEE4A6A0A7802AFA865D
:10BAD0000DA78435201701B61025FCAAAE849F2F30
:10BAE000A606270E840F8102267B200C9D1E009D3A
:10BAF0002100A6881746256D8DF2109E4AE6A4C146
:10BB00003D2762109F5E109F5C9EAB9F609F4ADC4A
:10BB10000C34268DDA3526DD0C109F4A9E2FA68820
:10BB20001746254132E90102DC00D3021F02DD463F
:10BB3000DD44CE0000DF31DFB30CB40F36DC4A9EAB
:10BB40000C3416308C1617FA4A9E4A8D0917FF617D
:10BB50009E2F8D05200C9D24049D24023516DD4A60
:10BB60009F0C16FA24C63316FC168D205F103F0674
:10BB700017FC4927131700F3250EDE464F5F3616D4
:10BB80004C97358D170F353953C62B39109E828649
:10BB90002AA7A4973517FDFC0F2F0F30DE46DF4490
:10BBA000203EAE84E6062715C1222606E6881758F1
:10BBB0002B0B34403384103F023540201E0D3526B8
:10BBC0001FAEC41700EB10AE84DC0AA322DD0AEC22
:10BBD00022D30CDD0CDC4AA322DD4ACCFFFFEDD4DE
:10BBE000AEC326BE9E041F12EC811083FFFF27F810
:10BBF000EDA126F410A3A426F7398D6F2501393461
:10BC0000501F10C1FE275F9E0C8C00FF2558308806
:10BC1000E4DE4AC6FF5C6FC5C11826F95C301F27F9
:10BC2000456CC818A6A0A7C52AF25C9F0C4FEDC8AA
:10BC300015ED49ED4FEFF43404C30003ED42ED4D33
:10BC4000D30ADD0ACC87CDEDC4CC0019ED44CC007D
:10BC500081ED46CC0016ED4B350430CBC603A780F2
:10BC6000ED819F4A35D0C62016FB1534609E041026
:10BC7000AEE4EE812715EC4433CBA6A0A8C084DF48
:10BC800026ED4F6D5F2AF3301E35C64320F98DDB5C
:10BC90002501393470E661C1FE27CB30A44F103F37
:10BCA000002408AE624F103F012504AF62EFF43567
:10BCB000F03430DC08D30A1F02AE8410AFF4EC027B
:10BCC0008D1C34369E04200E10A362250910A36437
:10BCD0002204A3E4ED1EEC8126EE326635B0347604
:10BCE000CE00001F10A3643416E3642730A684340A
:10BCF000022008A6A4A78433411F211F10E365106A
:10BD0000A3692502E3611F0210A36326E63502A79B
:10BD1000843021AF6233411F30E3E426D0326435F2
:10BD2000F6347696368139273D0DA0267A0CA096FA
:10BD300035262FDCB3830001224C2B0D17FD72300A
:10BD40008DF76017031C17020F308DF760318DF6E9
:10BD50008817F87924F39635260817F86920EA9DA4
:10BD6000240C810226D68DF7860391BE2703103F4F
:10BD70008F4C811025F416F81017FA0E260D30A4FA
:10BD80001706CE2409398D065F2002C6014FDDB3A8
:10BD90000834430634200C17FD1708340434CC0053
:10BDA00001DDB332620FA035F6109E19ADA43476D2
:10BDB000109C46272AD67D9E80DE823454DF801771
:10BDC000FCEF863D1702B4E6A4CB01C10624053082
:10BDD000A41702E11701983554D77D9F80DF823583
:10BDE000F61701726D88172B1E9E5E0F740D352697
:10BDF000163184170AE98D141E129C6025EF9C5C95
:10BE00002605109C6025E64F399D2106347017FCED
:10BE1000A09E2F6D88172B7AAEE41F20A3E42B6F12
:10BE20003416C3002810930C1024FE3A0D842B27DF
:10BE300086209C5C22092705109C5C2302862A1719
:10BE400002399C6024111F10935E9E828DBB862058
:10BE5000A7809F821701243526109C602431DE4A7A
:10BE60001708A417008FDF5C30CB9F609F4A31C456
:10BE70000D842B0E30A41705072607308DF184178B
:10BE800000F417FC2C17095217010B8D4B0A83176E
:10BE900000DD35F09E2F6D88172A024339109E80F1
:10BEA00017046A8D509E4A1704D6272C9F5E9F5C0C
:10BEB00031849EAB9F609F4A8D189E2FA688176F76
:10BEC00088174D2613308C1017F6C89E5E8D061607
:10BED000F6B79D21049D24083476DE463736109F40
:10BEE0000A9F0CDD4A3736109F609F5EDD5CDF469F
:10BEF000DF444F35F63476DE46DC5C9E5E109E6095
:10BF00003636DC4A9E0C109E0A363620E1109E31F1
:10BF1000308DF55A8D0F170149AE238D44308C08B2
:10BF200010AE2726EF16FB8963616C6C6564206296
:10BF3000F917F888271E17FD322519AE84109E3197
:10BF400010AE27270FAC2326F768A44366A4308DD4
:10BF5000F559201643398DCD308DF5121701039E0A
:10BF60002F34103088198D0435908DB917012B1797
:10BF700001078D0720AF8DAD17011F3436DC82938A
:10BF800080230D1F029E808602103F8C24028D02AA
:10BF900035B6103F0F39109E5C109C60243CE6A41F
:10BFA000C13A260A31211701311700B8E6A40D84E1
:10BFB0002B118D4ED67434048D27350297741F983B
:10BFC000170094E6A02B088D398D168D4820031795
:10BFD00001BF109C6025EC109F5C16009C32622013
:10BFE000F6A7E22B1A84032716810126040C74207D
:10BFF0000E5A2A015F810327060A742A020F74A6CB
:10C00000E039308DF1075D2A02C02A86033D308B6E
:10C01000A684398DED3001846027068160261431B5
:10C0200022A61F3402EC84308B350284188110273D
:10C0300069202D81202604EC846E8B8D068D00A650
:10C04000802638967D81412516860A8D2E0F7D0D1E
:10C05000842B0C96748B03488B06C6108D4A4F397F
:10C060008D028D3634468DDB240DDE828620A15F65
:10C070002705119380260835C6860D3446DE82A733
:10C08000C0DC8293804D26040C7DDF8235C6862E6F
:10C090008DE9AEA1DC62308B30033410A684847F3E
:10C0A0008DD96D802AF635909D2A02C6039E4434B0
:10C0B00024313F20023424EC24ED83EC22ED83EC88
:10C0C000A4ED8331843504201EE6A44F200E308D6C
:10C0D000EE492004308DEE3D8D86ECA13420109E7B
:10C0E00044313AED21C6028DBF35A08D0EA6A08148
:10C0F000FF27088D86812226F420F0862216FF7BFA
:10C1000086248DF9C6148DA0312239308DEE871723
:10C11000FF50A63F8BFB20E5308DEE0617FF431640
:10C12000FF70308DED9E31218DF2312639308DEE4C
:10C130009B17FF2CA6A4813A27020C743928AA3039
:10C140008CFB2004308DEE5417FF17E6A05A27EC25
:10C15000A6A08DA920F703EFA501EDFF02EE0204D2
:10C16000EFA480EFA700A6A03402863A8D8F308C12
:10C17000E33002A6E4A484A18026F64D2711A8E4AA
:10C18000A7E4EC84308B17FF11862B6DE426DD3598
:10C19000823440DE446FC26FC2313FE6A42A2D17BD
:10C1A000FE601F89A6A0C58026F1CA803606C51884
:10C1B00026E9C47F3606C5042606ECA1ED4220DB45
:10C1C000313F10AF42E6A01706B520CF109F5C317B
:10C1D000C44F5FEDA3340697BF97B1ECC1C50827E4
:10C1E00025C407D1BF2213260EC10626060DB1278E
:10C1F0000620070DB1270317008FD7BFCA80EDA314
:10C20000860197B120D50FB1C5032729C50426257E
:10C21000C51026043710AFA3EDA3C4038D6B81BEF8
:10C2200026058E54FFAFA38E4B802002AFA35A2663
:10C23000FBD7BF20A6C51026043710341034068162
:10C24000892504818C2394ECA15D2B062712AEA1D5
:10C2500020E934066F61C51026EDC407D7BF20D38F
:10C26000AEC1270D3610EDA320C93520E6A017FD7D
:10C27000A2ECE1270FC50426F131E41E8917FD93D6
:10C2800032A420ED109E5C35C0AEE434108E4E001A
:10C29000AF628E4DFFAFA33917F4FC17F95C10AEF7
:10C2A000846D262647341017049C17FCA9109E5E47
:10C2B0008D489635810226031703EE308DF1F0315B
:10C2C0008DF16D17F30724EA0D3526E6308CE33443
:10C2D000109E80688464841701771025F2E81704A3
:10C2E00044A684810D2713109E80201C4339303FC3
:10C2F000688467841701041700CC109F5C17008BBB
:10C3000030A41705DA1600AE8D0624EE399D1E0AFC
:10C310000D0C27650FA08DF59E4AA684813A26470D
:10C320004F5FA7E2109E5C1703FE109C602409EC8F
:10C330000110A32123026CE4109E5EEC011703E5BB
:10C340006DE026072405109C5C241C109F5C109C4B
:10C350006024149E4AEC0110A321260B34201705FB
:10C360007E1F20A3E120024F5F109E5C1703589EA2
:10C370005C8D0D260231844F39C62017FC144339D9
:10C38000A684813A2602A603813D398E0000109EC4
:10C390005E109C5C240A3001170544109C6025F156
:10C3A000109F5C9FB54F398D2E8D1B9C5E220734EC
:10C3B0003017FBA23530DC603406109F6017FA2B73
:10C3C0003506DD604F3934149E82E684C10D2602A5
:10C3D0003594326516F1EFA6A0812027FA812A262E
:10C3E00009109F829E5E109E6039303F8D0D250A98
:10C3F0009E5C109C5C24031E124F396FE2EC84811A
:10C400002B260D109E60C12A261130029F82358294
:10C41000812D26096CE4109E5E20EB3001A68481FC
:10C4200030250481392305CC000120048D23251BF0
:10C430009F82109E5C6DE0270D109E5E3406DCB579
:10C44000A3E124024F5F17049C4F39109E5C63E008
:10C4500039109E468D0DA6A0810227054FECA4261B
:10C460000143399D2A005F2002C6013271E7E4A62C
:10C47000A46F61812A2604A7613121E6A0C120278B
:10C48000FA1F98109F82170136EF62102B02076D7A
:10C49000E42709170129EF64102B01FA810D270801
:10C4A000A6A0810D102601EEDE46EF6DA6A2A7C262
:10C4B000109C8222F7DF46DF44EC6233CB3341EF3E
:10C4C00066109E5C10AF6B6F6A1600B717F5E2102E
:10C4D0009F5C17FAC1109E803125686A676A0D3526
:10C4E0002663DC82A3629E461700E8254D8681A75D
:10C4F0006A6DE42745DC82E364A3629380108300C5
:10C50000E622379E821E12EC6217F7D21F20A3622A
:10C510001F02EE663416A6C0A7A081FF26F8313FA1
:10C52000ECE1A3E4351017F7B5109F82EC64318B72
:10C53000EC62260231216D6126A46D6A2A3F10AE9D
:10C5400068ECE4260BAE6D9F469F44326F16FDAA41
:10C5500017FA2810AF6B6DE4272330A41703801758
:10C560000159109F5C109E8017FDA5109F5C10AEB6
:10C570006817036B109C5C26146D61271010AE6861
:10C5800017035C10AF68109C601025FF3F17F52162
:10C590006D6A260F308C1D17FAC8109E4617FB4B8C
:10C5A00017F9CC10AE6B109F5CAE6D9F469F443266
:10C5B0006F16FDD763616E27742066696E64BACE0C
:10C5C000FFFF810D27083341A6A0E13F26F46F3F0E
:10C5D000633F39340620103430A68081FF2710A134
:10C5E000A027F63530312110ACE423EB43358635F6
:10C5F000304F3586CC00648E000A341630A4109E6D
:10C60000B5A684812A2608108E00003001A68481F8
:10C610002027F83420810D271817FE352574ED6288
:10C62000A680810D270B17FE282567ED642B63A6D6
:10C6300084810D265D8D74ECE1109E5E1702A610BC
:10C640009F5CECE41700DE6FE2109C5C254D8D21B1
:10C650008C00002F460D3526046CE48D143265AE37
:10C66000621700E2109E5EDCB5170279109F5C4FE6
:10C6700039109E5CAE634F5F1700AD109C602411B3
:10C680006D622702AF211702561F10E3651F012AB2
:10C69000E53932662002326F16EF2B308C0517F821
:10C6A000C920BA52414E474587326417F1A34F392A
:10C6B00017FD2417FD108D0316FC3FDC4ADDAB1F70
:10C6C000203410A3E13184347630AB3410109EABAB
:10C6D000DC4AA3E4270317F605DCABEEE4A3E12371
:10C6E0000510AE648D1EDCAB934A10AE6431AB1006
:10C6F000AF64A3E13406D360DD60DD4ADC0CA3E463
:10C70000DD0C35F69D1E06343631AB33CBC4032722
:10C710000DA6A2A7C25A20F7AEA3ECA3361610AC02
:10C720006426F535B6109E5E340620031701B0105E
:10C730009C60240FA6A4813A26F2ECE410A32122E7
:10C74000EB3586433586347617F566AE849F2FEC3D
:10C7500009D32FDD5EEC0FD32F1F02DD60DD4AEC25
:10C7600002A30F3406DC00D302A3E41F03DD663509
:10C77000068D94EC0DA30F830003DD68D366C30020
:10C7800003DD62EC02A30DC30003DD64109E5E8D29
:10C79000499E62EC1D271B340633843003E6802A51
:10C7A000FC8602C1A426028604A7C43506830001C4
:10C7B0002EE59E66DC68308B9FDA9F66D30CDD0C1D
:10C7C0000F680F6935F6E6A02A02C02A4F308D01A6
:10C7D0001AE68B545454541700B2109C6025E73964
:10C7E0001917154634492E503D21561E1C1A0FA606
:10C7F0003F8B93A73F31213121396A3F6A3F6A3F1E
:10C8000039ECA4D35E1F01EC1EEDA16A3D39A6A050
:10C81000818526033129395F8D20312739A6A081F2
:10C820004F2602312439312539A6A081FF26FA3955
:10C83000E6A44F31AB39E63FC404866034068685F2
:10C84000A73F9E62EC1DEEA4200D35068300012754
:10C850002B30036D802AFC11A30126F03406A68438
:10C8600084E0A16226E4A684841826DEA6848404DB
:10C87000A86326D61F109362EDA132623262395D41
:10C880002A02C02A308C643AE684C40F308DFF50EF
:10C89000E6856E853440E6A0E1C022FC35402708DD
:10C8A0008DDD109C6025ED4335D61F213AFF3456AF
:10C8B000338CF720ED3E3FFF3456338CF820E334C1
:10C8C00056338CF220DC2385868788898A8B8CF20C
:10C8D000F3F4F5F6F7F8F9FF3456338CE920C34F3B
:10C8E0005F8DDC250583000124F73900000000007E
:10C8F00000000000000000000000000022000064B2
:10C900000022000000220022000022922292220037
:10C910000000000000000000000000000000000017
:10C9200000007777002292777700000000000080F7
:10C9300000222200001100000000000000000000A2
:10C9400022A2A2A2A2A22222222222222222112258
:10C9500033552200000000000000B000000000B0CD
:10C960000000000000000000B0000000B000B000B7
:10C97000B000B000B00000000000000000000000A7
:10C98000000000000000B0000000000000000000F7
:10C99000B000000000B0C000B0C000B0C0D000B017
:10C9A000C0D000B0C000B0C000B0C000B000B00047
:10C9B000B00000E2E2E2E2E2E2E2E23416E6F8048B
:10C9C000308C08EC85308BAF64359602DC076C0840
:10C9D00066084407F9016A002103FAD90A3CBEFA45
:10C9E000D90A3EBCFAE40A3CBDFAE40A3DBCFAE1CD
:10C9F0000A3EBDFAE10A3DBEFA52083ABDFAF10517
:10CA00002AAAFA380128AAFA3E02DCFAD30ABEFAA8
:10CA1000D60ABCFADD09BDFAE705ABFAEA05ADFABC
:10CA2000EC05AAFAEE05AFFAF005DEFA4C0CBAFAFC
:10CA30004F0CDBFA500CDDFA510CBBFA540BA3FA85
:10CA40002601BFFA3701A1A4000C8AFA4B0CACFAFC
:10CA50004D0CA8FA4E0CA9CE890CAE239006A2006C
:10CA60009106A4FA3F028D03BA01260116012601A0
:10CA70007502CA03AC03AC03AC02CA03AC03AC033B
:10CA8000AC03C203BA0183018C01A103AC01A5016F
:10CA9000C601D001DF03AC01DB03AC01DF01E30120
:10CAA000DF01EE03DB022903BA022903BA025603AF
:10CAB000DB029702CA03DB03DB03340334032402E3
:10CAC000FB0308031203120373037D03DB03DB0381
:10CAD000DB038103810399039902CA960B34029EFA
:10CAE000A7860D68846484A18026F89EA78D39DC12
:10CAF000B993A734049EAF9FAB109EA7863D17063F
:10CB00001B1702FC17061586209E80A7806AE42A60
:10CB1000FACC5E0DED1F9E808D0E35068D079E466C
:10CB20009F449D1B069D1B02108E0100962E103FF8
:10CB30008C399D1B0435108DF917015D17031310F7
:10CB40009FA79EAB9FAF8D0F96A31705CF813E2762
:10CB5000F5813F268620CB1704EB96A48101260D94
:10CB6000D6A34F5849308DFEFEEC8B6E8B810210A0
:10CB70002602B934109EAB301F9FAB35901702EDE3
:10CB800081DD1026029F8DEB865317058F1702DD7E
:10CB9000814D26121702DD26081702D82603170238
:10CBA000D31704208D2C1702FE27E2814C261D8D01
:10CBB00021D6A42715C103261C8144260D8D13817F
:10CBC0004F26091702AE8150260B8D06815127BDD5
:10CBD00020A1160470861820661705408D4817029C
:10CBE000C627F68655170534204A1702551702BC8A
:10CBF00016024C8D4D8145260B1705201702532434
:10CC00004716FF53862620378D2A204617028A179B
:10CC1000022196A3814626118D0A96A3814726C339
:10CC20008D0220BF8DBF16021986272012170269B8
:10CC30008D028D001602458D0981482713861F1627
:10CC4000FE9B8DE2209D8DEC204C8DF6814526B417
:10CC50008D6816FF02DCAB34261703E9811E260916
:10CC600032648D32811F272B393526DDAB8DD39E63
:10CC7000AB301F3410811F270C812127088621200B
:10CC8000BE8D37863A6CF48D0A17021B27F3359058
:10CC90001701831701C616017A109FA79E4A9FAFFE
:10CCA0009FAB0FBB0FBC398DF00CA01701658D1920
:10CCB0000FA096A3813F1026FE2116045F17015690
:10CCC00034101701D4C623E7F1814D26D98DEBDC52
:10CCD000AB342617036FCC000591A42704D7A420FA
:10CCE000031701A43526DDABD6A4C105270317021F
:10CCF000721703271701B027D43402160300109FC0
:10CD0000A91701882609109FA98D1F8DAD8D871049
:10CD10009EA98190260C17032C17FF7A8D0C864B49
:10CD20008D668D5717017A27F53917017427FA2078
:10CD300054109FA9170155270981492709109EA959
:10CD4000200B814926161700F620118D3B1704147D
:10CD5000810D102700BD815C27F88D311701422716
:10CD6000EA39109FA917012427B2109EA920B310F9
:10CD70009FA917011727E520C48D050CBC160106D5
:10CD8000170109265A1701241603918DF31600B2D4
:10CD90002C012D02F703F804F980001702A7815433
:10CDA000263D8DD78DDF8DE596A3814C266E864A74
:10CDB0008DD66FE28D5D308CD7A18122FC2610E6E6
:10CDC0001FEAE4E7E48D4C81E727E9A6E026B9866F
:10CDD0000F200E1700D126448DAE1700AF27F48622
:10CDE0001C16FCF98D6C202B17037931218030271C
:10CDF000228101102600D88D1D863617031E2013B0
:10CE00009EAB17035F4F1703136C84A6A0810D26FA
:10CE1000F5313F17022F9EAD9FAB96A33996A427FD
:10CE2000FB860C20BC861B20B81702198DEF0CBCAA
:10CE30001700CF96A38152270681DD26E886531777
:10CE400002DA86399E445F1701758D6E1701192429
:10CE5000F93917030F17031D25F7863A8D25170299
:10CE6000492706EC84102E02AA861020BA8D028D66
:10CE7000AC1601D1868E8DE48DF7202B4F8D048D5D
:10CE80000220111602968DE98D9320768D858154AE
:10CE900026068DAB96A31A04398DD617FF7F16FF91
:10CEA0007296A38151270496A3814B398DF927FBF4
:10CEB000861D201D5F8D4417FF5C8D348D16814DBE
:10CEC00027F2D6A4C10627D6C10426BC16010386C4
:10CED0001216FC0981CD271181EA26CFA6A41702DC
:10CEE000942410812E270C86CEC6078D0E17FF26A0
:10CEF000160152313F17FC7B16017D9E44ED839F46
:10CF00004439CC85003406DCA18DF035068DEC1754
:10CF1000FF0417FEFE5F814D27128189262F8D3D6C
:10CF20008D2B8DCC17FEF6CC890020D98D2F5C344B
:10CF3000041700E717FF70260BE6E0C10325ED8616
:10CF40002A16FB998D7E17FECA350420CD0FBC9E94
:10CF500044EB811701C4EC819F441601B60DBC2738
:10CF60002E0FBC860E1601B4D6A34FC14E27215DED
:10CF70002A068D5B850826189E44EC81814D274A40
:10CF80008DE35D26F58139260317FBE79F4443397E
:10CF900084071F899E442004A6818D7AE10125F82B
:10CFA000221BC10627175D26EFA681814D26069F0D
:10CFB000448D5220B3813927558D5B20CF96A3ED48
:10CFC000839F443996A3814E27F9862516FB0E9D33
:10CFD0001B1217FB9E96A334028D2AE6E48DF030D7
:10CFE0008C1C34108403272A81022736223BE662F8
:10CFF000C1922744C1942740C1BE2731201B8DC454
:10D00000350217011716FE0B96A3814D27B5862210
:10D0100020BA326235021601038DED4F17FE251638
:10D02000FB518DF517FE8520F28DF720F78DD98DF8
:10D03000D4815427E616FDA78DCE5C1700DC16FEC2
:10D0400045860A2087DCABDDAD170118109FB917A4
:10D0500000E710260091A6A417011A241B308DF9B1
:10D060007986801701CB27D9E684338C346EC5A628
:10D07000A41701012525313F8D302611CC8F05974E
:10D08000A38D59A6805A2AF9860697A439CC8E0218
:10D090006D8426EBCC8D01300120E4EC01DDA32072
:10D0A0007B313F8D05CC910220D51700B730A410FD
:10D0B0009E448D091E122508A6808102399D2A00F2
:10D0C0008616201C8DD520028D52A6A0810D270E1C
:10D0D000812226F4A1A027F0313F86FF203E862939
:10D0E00016F9FA863120F99E9E17014327089FA161
:10D0F000EC84DDA320260DA02BE99E6217013026CB
:10D10000070DA026DE170093CC85008DE51F109338
:10D1100062DDA18D078D0396A3391F9834169EAB4F
:10D12000A7809FABDCAB934AC1FF24034F359686A3
:10D130000D17F9F19D1B068D2B3420C602D7A55F74
:10D140008D3D251C31215CA6A08D2624F981242645
:10D15000075C860497A52002313F8680AA3FA73F3F
:10D16000D7A635A0A6A0812027FA810A27F6313F4D
:10D17000398D0C2425813025218139231B201684EB
:10D180007F81412515815A230F815F270D816125FC
:10D1900009817A23031A01391CFE399E62EC1DC3F2
:10D1A0000001ED1DD6A64FC30003109FA98D463484
:10D1B0002096A55FEDA1E7A09EA9A680A7A02AFAC8
:10D1C000318435903446DC0CA3E42405862016F91E
:10D1D0000CDD0CDC66A3E4DD66DEDADCDAA3E4DD7C
:10D1E000DA1F02DC6693DAD3688D24DC68E3E1DDC4
:10D1F0006830C435C034468DCBA3E4DD6833843059
:10D20000239F62DC648D08E3E1DD6430C435C03403
:10D210001630CB3410C503270DA6C0A7A05A20F5A1
:10D220003716EDA1AFA111A3E425F56FE135968680
:10D23000203472EE1DE61FAF6111830000272033FA
:10D240005F10AE633085A680A8A0270CA1E4270854
:10D25000301FA6802AFC20DF6D1F2AEA10AF63353D
:10D26000F23416E6F804308C08EC85308BAF643568
:10D270009606DB0B1F01190189078A020301AC0224
:10D280000703AD070B07A207A207A2070B07A20718
:10D29000A207A203D703D5042704B304CE04E504F0
:10D2A000F7058F05DE05EC0604060B061F062306B0
:10D2B000270644042E049D044F014D044F014D06E2
:10D2C000A2078A06E8070B078A078A074907490762
:10D2D0006506E8070B07730773077D079A078A0738
:10D2E0008A078A07A207A201470147070B00DC0152
:10D2F0004D014D0140019C019C2020060043402827
:10D300002500434343434343430500434343004510
:10D310000025004500050021214727272222226001
:10D320006061878A89898185008081E0E0E0E0E0B2
:10D330006B05006C6C6C6D00006D00006E000000F1
:10D340006E0000006D00006D00000D00000600067C
:10D350000006004444ECA40DD926123406313FDC0B
:10D3600060DDABCC000317096835062002312217B7
:10D3700003682412ED841F20935E3002EE84ED8456
:10D3800030C426F82004864B8D41308DFEEBE6A09C
:10D390002A05CC03D5200A584FEC8B108303D525E2
:10D3A000160DC726120CC734061F20935E8300019A
:10D3B000DE2FEDC81535066E8B9E2F8601A78817C8
:10D3C000E6A04F31AB39109E60863034369E2F86F2
:10D3D00001A7881796842B20EC64935E327B30E49F
:10D3E0008D188620A780860230E4108E0005103F3D
:10D3F0008A3265E6E417F72D35B68D021F983402A0
:10D40000444444448D043502840F8B308139230217
:10D410008B07A78039E6A48D052602312139C13F4B
:10D420002702C13E39170810D6CF2704864C8D9BA2
:10D430003124864097CEDCC134064F5FDDC18D4478
:10D44000DCCC93602731C3000310930C102402B985
:10D45000343017091EDCC133A4EDA16FA09E60EC2F
:10D46000819362EDA16C429CCC25F41F3035309342
:10D4700066ED018625A7843506DDC1398680200248
:10D48000866097CEDC603416DDCC8D50E6A0C14BB3
:10D4900027F8C14C2706313FC60120041700975FCB
:10D4A0003424AE63DCCCED639FCC93CC5849E3636A
:10D4B0001093DA2515160251EE816DE42709A6C4F2
:10D4C00097D11708B6DDD61700AAAC6325EADCCCE5
:10D4D000ED633524E6A0C15127B03596170759D61C
:10D4E000CF2718864C17FEE33123E6A4C14D260A48
:10D4F00031218D36E6A0C14B27F839DCCCC3000AB8
:10D500001093DA102402029ECCDCD2ED8133846FBA
:10D51000803123E6A4C14D260E31218D0DED816CA5
:10D52000C4E6A0C14B27F49FCC39E6A04FC18D279C
:10D5300002A6A0E6A039A6A08185271B804097D12E
:10D540008104260EE6A4C14F260831218DDC31214D
:10D55000201F170826201A313F1706DC3123D6CFAB
:10D56000C1202705861816FE62EC01DDD29E66EC0E
:10D570008BDDD639E68027543404585858D7D05418
:10D58000543085CB04345096D181042502CB024F10
:10D5900010930C102201721707D9AEE43322CC008D
:10D5A00001EDC1EC83EDC18D4A6A6426F696D18106
:10D5B000042305DCD2EDC443DCD62502EDC48D3353
:10D5C0001F2035509366ED4132612010D7D096D19F
:10D5D00081042204DCD62002DCD2ED4196D19AD01F
:10D5E0009ACEA7C4341030C41706F99ECCEF819FA1
:10D5F000CC35903406E6223D2625A661E6223D4D37
:10D60000261DE722A6E4E6233D4D2613EB22250F37
:10D61000E722A661E6233DAB222504ED223586866E
:10D620004917FDA73586DECA26081F20935EDDC890
:10D6300020061F20935EEDC417042417050CE6A0F6
:10D64000C14B27F4109FCADCC8EDA116FDCD313FB8
:10D650008D2E31211704081704F097D11704EB9190
:10D66000D1271A81022213270486C8200286CBD62E
:10D67000D1C102220517063C20031700A516FD950F
:10D68000A6A4810E102603D731211703D2A63D810F
:10D69000852408DCD29362ED3E86858B6DA73D39EB
:10D6A0008D008D72312139E6A0C11E2714313F8DC6
:10D6B000F1ECA1340631218D0F350683000126F3EC
:10D6C00039E6A017FD582711ECA48D0EEC022403B7
:10D6D00010AF02EDA46C3F3123399E663406200959
:10D6E000EC84847F10A3E4271B301C9CDA24F1DC3B
:10D6F0000C8300042513DD0CECE48A80ED844F5F7D
:10D70000ED029FDAA6844935868620973617FCBB42
:10D710001706C816F40C17034617042E81022707B4
:10D7200025B7864716FCA486C816058817017CA66F
:10D7300023813A2705861016016A342031248D880A
:10D740001F20935EEDF139CC100217018CEE011011
:10D75000AF01312217FCBE1F20935EEDC439CC10FF
:10D760000117017531211F20935EED980116018D7F
:10D770001704C51704658160260A96D18101271018
:10D780008102270C864617FC42CCFFFFDDD2200C1D
:10D79000D6D026F08B80A7A4EC01ED219E44301951
:10D7A0009F4496D1A784DCD29362ED014F5FED05D3
:10D7B00031248D398D1AED03A6A4814726048D10DE
:10D7C000ED05312110AF838613A7829F44312339A1
:10D7D000DCC13406ED219E44A684308D0598E68692
:10D7E0004FD3C1DDC131238D049E44358617026FAE
:10D7F000170357A1C427D8810225081026FF2386C6
:10D80000C8200286CB1604AC313FCC130B1700C9DD
:10D81000EC2210A3042707864617FBAF202FD36204
:10D820001E01AE011E01ED22A6038402A721EC0613
:10D83000ED24EC08ED2627026C21EE011F20935EFB
:10D84000C30001EDC433431F30935EED28312B1725
:10D8500000AB30079F4439333F34408D4E3506EDE1
:10D86000A48615203FCC15038D6FAE01EC84935E2A
:10D87000EDA431231F20935EED84160080861717D8
:10D88000FB99204B8D258617313FC6038D4BEC014C
:10D89000935EED2131242065861920E3861920E866
:10D8A0008D09861B8D29312316FB6A1701B11702DA
:10D8B0009981032705864717FB11312139CC1B03BA
:10D8C0008D1733A4312317FE9DEF83861C20059E00
:10D8D0004410AF83A7829F443934029E4420023013
:10D8E000039C46240AA684811C27F4A1E4270C3259
:10D8F00063864517FAD531A516FB1A35829E44205A
:10D900000FA684811C260F1F20935EED9801300323
:10D910009C4625ED200230039F4439313F17031800
:10D9200096CF271981A027228160250A96D0260646
:10D9300096D181042714864C17FA90200D86A0A753
:10D9400084DCC5ED01C30002DDC53123E6A0C14D75
:10D95000260E17FD2B1701F2E6A0C14B27F431214B
:10D96000398D4B313FC190260517009B312117FDA2
:10D970000F1701D681052505864D17FA4EA6A08101
:10D980004B27EB398D28C14926048D7BE6A0C14B7E
:10D9900027FAC15127F617FA852726313F1700BF0E
:10D9A0001701A7810525E5864717FA1F20DEE6A0A7
:10D9B000C154260D17FD5FE6A0C14B27FAC15127C0
:10D9C000F639312117FCB91701808101270317FDB2
:10D9D0005131218D32A6A0814A26023122398D1E75
:10D9E0008D7D1701658142233216FD368D1017FC9F
:10D9F0008F17015620258D06C14B27FA201D312196
:10DA000016FC9F8D0220148D5617013E810427CDF0
:10DA100016FD0FE6A0C13A1027FCAD16F9F7C19626
:10DA200024051701322038C1F21024F999C096302C
:10DA30008DF8C63AE6841027F98CC41F2706338C6C
:10DA40005B58ADC5E684C4E027104F594959495980
:10DA5000498107260517027220051700D83121E6F3
:10DA6000A42BBB398D035C2002C6C81700DC8102E1
:10DA7000250D27048D4720051F9817023786013989
:10DA80008D035C2002C6CB1700C08102270D250440
:10DA90008D2B20051F9817021B860239201C20C9D8
:10DAA00020C220E120DA203020182042203E2049E8
:10DAB000204C207620722055204916F909864316FD
:10DAC000F9098D1D34028D19A1E0270E86CB2401A2
:10DAD0004C1701E0860220068D07810226026CA405
:10DAE000398D67810223048DD48602398D008D5AC9
:10DAF000810427048DC786043917FF6D20F017FFB6
:10DB00006320EB86038D132604C603200886048D4C
:10DB10000926AFC602EBA4E7A439DE44A1C026075C
:10DB2000A1C02603DF445F398D008D1E81032704C9
:10DB30008D8B8603394D26014CDE4481052606DC9B
:10DB4000D4EDC38605A7C2DF4439DE44A6C08105F3
:10DB500026023342DF4439C1851025F869C1892581
:10DB600042C08D10250095338C03586EC5201020BF
:10DB70001020142018200A201E2025201A202131D0
:10DB80003F3123860120B23126860220ACE6A0C1B7
:10DB9000FF26FA860420A217FAF38DAE86018D992E
:10DBA0003121391700928D338160270B818027073F
:10DBB000861217F816201DC685170097E6A4C185A2
:10DBC0002612D6CFC160260C810524088B80A7A41D
:10DBD000EC01ED21312396D116FF5B96CF261CC6B2
:10DBE0006097D0D7CF86609AD1A784840781042616
:10DBF00005CC0020ED011700EB96CF398D3AC68990
:10DC00008D5117FF4581052705CEFFFF2002EE5EEF
:10DC100034408DC035401183FFFF2717E642D7D629
:10DC2000DCD29362334310A3C127270AD626F78696
:10DC3000142002864216F793EC21D362DDD29ED2E5
:10DC4000A68484E097CFA684841897D0A6848407FE
:10DC500097D1393404E6A4E0E0260E96D02734CCE0
:10DC6000FFFFDDD4860597D139585858D1D0270504
:10DC7000864117F75686C897D817FECE8102250D24
:10DC80002707864717F744200496D88D270CD8C05D
:10DC90000826E696D18105261AEC01D3661F03D625
:10DCA000D027085454CB04ECC52002EC42D366DDE7
:10DCB000D496D13934149E0C8C00101023FA4A9E4D
:10DCC00060A7809FAB5F8D083594DC60DDABC6013B
:10DCD0004F9D1B140049005C0060006A00660072E2
:10DCE000007200763470318CEBE684C4E0C16027AA
:10DCF0000AC1402706C18026223128E684C418279D
:10DD000004EC262014E684C407C104250A2204EC8E
:10DD1000222006EC242002ECA4ADAB35F0A68484CE
:10DD20000731018D563406DCC1EDA4E3E1DDC139D4
:10DD30008D2D20F18D29D3661F01EC8420E78D16EF
:10DD400020E33101DCC3EDA4C30004DDC3398D0F32
:10DD500020F28D0220EEEC01D3661F02EC2239CCBA
:10DD600000048D0FAE64EC01ED221F209366ED01DF
:10DD7000EC22399D1E0801020501203410308CF67A
:10DD8000E6864F359001020307080937383E3FFF0A
:10DD9000CC0016DDC15FDDC3DDC597C7DDC8DDCAB8
:10DDA0009E2FA78817ED8815109E5E20253420171A
:10DDB000F5D83510D6D9261AA684338CC8A1C0252B
:10DDC0001126FA34101F20A3E13184DE4ADFAB179D
:10DDD000FEFF9E606F84109C6025D29E66201CA66C
:10DDE000842A18847FA78410AE02EEA4EC84EDA4EC
:10DDF0006A3F864A17F5D431C426EF301C9CDA24DA
:10DE0000DEDC6693DAD30CDD0C9E4420179D1E06E3
:10DE100010AE01864517F5B3A6848113260230079C
:10DE200030039F449C4625E8DE66109E60DC64D388
:10DE3000688DDA9E2FDCC8ED8813DCC1ED8811D324
:10DE4000C5DDC5ED0BE688184FC30019ED09D36099
:10DE5000935EED0FD368C30003ED0D830003D3641D
:10DE6000ED02D32FDD4A9308DD0ADC2FE30DDD62DE
:10DE7000DC2FE30FDD66DE62205A30C417FDC19649
:10DE8000CF8160252A81A02608EC01D3C1ED0120B5
:10DE90003D8180261AD6D0260A96D18104240430EA
:10DEA000412006EC41D3661F01EC84D3C5ED849676
:10DEB000D181052619D6D027065454CB042002C69A
:10DEC000024FE3419E66318BECA4EC8BEDA433430F
:10DED000A6C02AFC11934A25A1393416E6F804306D
:10DEE0008C08EC85308BAF64359609C800AF0926E5
:10DEF00007BB018208280832080308030803080347
:10DF000008030393008C081A082403A4080E0812BF
:10DF100003CA017402E7038601820192019902A6F5
:10DF200001A5019C01920174019C01740192019C64
:10DF3000019203E307A9080A0192080A03AA084606
:10DF400009AC049F0608072E073B043904420470FD
:10DF5000057A069306C806CF06FB07080721075176
:10DF6000076F07EE07F107FC07FC015D0172017204
:10DF70000800080A01710171030B031A0329030B3E
:10DF8000034208419D1B0C53544F5020456E636F54
:10DF9000756E74657265640AFFA68817850127048B
:10DFA000C633201C1F408301001093802404C6390F
:10DFB000200EDC0CA30B2506108301002405C620CF
:10DFC0001606E2DD0C1F20A30B1E0310EF45ED47E4
:10DFD000AF43CC0001DD42A741A7C813EFC8148DA1
:10DFE0002CEC88132702D35EDD39EC0B31CB3420C7
:10DFF000EC881131CB4F5F2002EDA110ACE425F984
:10E0000032629E2FDC5EE388151F01203F9F2FDFC9
:10E0100031EC0DD32FDD62EC0FD32FDD66DD60EC2C
:10E0200009D32FDD5EECC814DD46DD44399F5C96D4
:10E030003427172A09847F973417026396344624BD
:10E040000931841706AB0F748D088D209C6025DD87
:10E05000200D9D1B16E68417049F27031704A117A4
:10E0600006BADE3110EE45EE47393002E6802A026C
:10E07000CB40584FDE0EECCB6ECB9D166D22270A9F
:10E080003003E684C13B26E13001EC84D35E1F01FE
:10E09000393001399D166D2227F0300339318C6FEC
:10E0A000E680E6A5DE316EA5EC8431CB2017EC844A
:10E0B00031CBEC04A6CB2A0D202BEC8431CBECA485
:10E0C000C30001EDA4EC023006ECCB10A3A42CBAE3
:10E0D000300339EC8431CBEC04ECCB3402E3A4ED17
:10E0E000A46DE02AE0EC023006ECCB10A3A42F9A3A
:10E0F000300339109E465F8D50203E109E465F8D46
:10E1000048EC04C30004DE31A6CB44242C2076ABBB
:10E11000C40851959BE0E8109E465F8D2C313ACCA7
:10E120000180ED214F5FED23A725170B34EC21ED86
:10E13000C4EC23ED42A625A744C6028D0C30061779
:10E140000FB2102FFF44300339EC85D3311F033158
:10E150003A8602E6C4EDA4EC41ED22EC43ED24390D
:10E16000109E465F8DE3DFD2C6048DDDA64497D1B5
:10E17000170AEEDED2EC21EDC4EC23ED42A625A772
:10E180004404D124B4C6028DC03006170F66102C8B
:10E19000FEF8300339D634C50127F99D1B1CE680F3
:10E1A000C18227238D6C8D12E61FC14726028D0A7E
:10E1B00017FED7318DFF5C16FEE6EC81D3313406B5
:10E1C0009D16EC21EDF1398D588D0AE61FC14726C9
:10E1D000DF8D0220DBEC81D33134069D16204C9D6F
:10E1E00016810425043440DE3E344230019D16354C
:10E1F0000248338C026EC620142021202E200E20CF
:10E200004D206AEC84D331340630039D16E622E7B4
:10E21000F139EC84D331340630039D16EC21EDF155
:10E2200039EC84D331340630039D163540EC21EDB2
:10E23000C4EC23ED42A625A74439EC84D3661F0322
:10E24000ECC4D3313406EC42340630039D16354617
:10E250005D26014A973E10AE21109F48A6A0A7C098
:10E2600081FF27075A26F50A3E2AF14F3935461015
:10E27000A3232302EC2310AE211E239D1E069D1610
:10E28000EC2134069D16E622E7F139170272962E2C
:10E29000977F308DFCF117016D16E8861702619D9E
:10E2A0001B18EC843003109E31EEA81411934A22FF
:10E2B00005C6351603EFAFC3EFA814DF46D35E1FC4
:10E2C0000139109E3110ACA8142205C6361603D5AC
:10E2D000EEA814AEC1EFA814DF4639EC84811E27E6
:10E2E000359D16EC8458495849C30002338B34409D
:10E2F000EC212F2010A381221B830001584958498B
:10E30000C30001EC8B3406E684C12235162797D36F
:10E310005E1F01393590DE31C120260FEC02D35E3D
:10E32000EDC8118601A7C8133005396FC813300234
:10E33000398D1CC60B103F8320058D13103F8410B0
:10E340002503623544C10126026FC0A7C435903051
:10E35000011700CC30019D168603C14A2602A68112
:10E36000EE63AF63AE216EC41700F29D16C60E17A2
:10E3700000AB10250331393F20FF2A2A20496E7057
:10E380007574206572726F72202D207265656E74CF
:10E390006572202A2A0DFF962E1700C1862C97DD64
:10E3A0003410AEE4E684C19026089D163410AE21E8
:10E3B00020053410308CC08D4D3510967F912E265F
:10E3C00004962D977FC6068D54240DC10310260296
:10E3D000D61702F90F3620CA8D112407308C9B8D79
:10E3E0002520BFE680C14B27EF35868D33E6E4CB91
:10E3F00007109E468D271024FDF5A6E48104250212
:10E400003262326343393420327A31E4AF21DC8026
:10E41000DD82C6058D075F8D04326635A09D2A0218
:10E42000A680810E26049D16202580808104251556
:10E4300027051703012018EC81D3661F03EC42DD8A
:10E440003EECC42002EC81D3311F03A61D80803531
:10E4500020810425043440DE3E34426EA4E684C1AB
:10E4600054260C30019D16C14B2702301FA622975F
:10E470007F39E684C15426238DE30FDDC14B26028C
:10E48000301FC6068D97240CC1E427F61602181714
:10E49000FF5925F8E680C14B27F5398D5C273D8D66
:10E4A00007E680C14B27F83917FF758D31A6E426A2
:10E4B000014CA1A41027FD37810225062715C64768
:10E4C0002024A6A4810226F68D0316FD229D270C8A
:10E4D0009D270EA1A425E78DF716FD1330013410FA
:10E4E0009E392605C64F1601BC9D16C14B2706EC6A
:10E4F00084D35E1F019F393590C13F2702C13E3949
:10E50000962E17FF58DC80DD82E680C149273D8DBD
:10E51000E82722C14B2712C1512712301F9D16E652
:10E52000A4CB018D1FE61F20E6C60D8D17E6808D5A
:10E53000C826E02004C60C8D0B5F8D0896DE0FDE2A
:10E540004D26063917FED624FA16015B9D16DC4AC5
:10E55000DD8EDD8CDE4634460F94DC48DD4AE61F56
:10E560008D97271CE6808D912711301FC61117FE4D
:10E57000AC24EB3546DD4ADF4620CE318CBB200390
:10E58000318CB23546DD4ADF466EA4962E17FECD9D
:10E59000DE80DF82E68017FF602722C14B270C3028
:10E5A0001F20084FC61217FE74259E9D16E6A4CBA9
:10E5B0000117FE692593E61F17FF3E26E616FF7535
:10E5C0008D11103F8920058D0A103F8A30C4242206
:10E5D0001600D217FE8717FE4733843502810424C4
:10E5E0000B308D0227E6864F1F02200235203510A2
:10E5F000967F3917FE67103F8F25D5C14B27F43919
:10E60000E680C13B270ADE2FECC813D35EDD393923
:10E61000EC84C30001300320F29D163410AE2110AB
:10E620003F8725AC35909D1686013410AE21103FF2
:10E630008620EF9D16860420F117FDE4109E4631DA
:10E640003AD67F4FED2116FBA69D1610AE213470F1
:10E650008D1235708D3510DFB110DE80103F051042
:10E66000DEB120419D1B0E9D16345010AE218D1B36
:10E67000103F0325303402103F04A1E426F9326133
:10E680005D262235D05348454C4C0D9E48860DA73B
:10E690001F1F10308CEF33A43420A3E11F024F5F03
:10E6A000399D16E622D736DE31271A6DC813270E9C
:10E6B00010EE45AEC811ECC814DD4616F96F8D0D8D
:10E6C0008D5A16E45D17E45D16E4570EFF308CFB9F
:10E6D00017FD339E5C31848D180F7417F974D6368C
:10E6E00017E4429D1B185F2002C6014FDD42300136
:10E6F000399D1B10E6803A391E153931848DF23070
:10E70000A439C633209F860120014FDE31A7413056
:10E71000013996348501261A8A012008963485012C
:10E72000271084FE9734DC173406DC19DD17350614
:10E73000DD19399D1B009D27028DFB16FAA38DF66E
:10E740003410D6CFC1A02720109E489E3EA6C030D0
:10E750001F2708A7A081FF26F4A6A38A80A7A410DC
:10E760009E488DCF253F3384ECC4260D109ED231B8
:10E77000238DC02530EC84EDC4AEE4EDE4DE3196AB
:10E7800034A7C4D643E742DC4AED4DDC40ED4FDC14
:10E7900039ED498D7BAF4B3510A6062737812227EF
:10E7A0003381212705C62B16FEFBEC45340610EFFE
:10E7B0004532A4DC403420A3E1445644563406ECF0
:10E7C00009318DF7D4AD8BDE3110EE453510AF45F4
:10E7D000241B20D317FF459634847F973417F7B94D
:10E7E000A6C48501270717FF29A6C49734EC4DDD81
:10E7F0004AEC4FDD40EC49DD39E6421DDD42AE43D7
:10E8000017F80AAE4BDC44934ADD0C3901020501CE
:10E810003440E6804F3412C14D267731E43420E68F
:10E8200084C10E272F9D16301F8102270A810427DD
:10E8300013EC21ED24A6A4C606338CD0E0C633A584
:10E84000DF462014EE21DC48934ADD3EDC48DD4AF9
:10E850008604200430019D1635206CA48104250413
:10E860003440DE3E3442E680C14B27B13001AF2157
:10E87000308C99DE46DF403504C10425043506207E
:10E8800003E6854FEDC33506EDC36AA426E931C41E
:10E890002006109E46109F401F20934A1025F71E09
:10E8A000DD0C35D29D1610AE2134108D0235909DB1
:10E8B0001B0A8D07308DF6409F0E399D27003416B8
:10E8C000E6F804308C08EC85308BAF643596142E56
:10E8D000015B039304B206120826091808E0125DD2
:10E8E00012211239120612E512E91339130D0888A4
:10E8F00008ED08F40850088106E301F302F606CE9D
:10E9000006D406DA074D0790071F0725077207018F
:10E910000735077E0713076A073D0784070D07625F
:10E920000745078A0719072D0778070701FA030328
:10E930000832020302FD020C041A026E057A0684F4
:10E94000068400B700B700B700B700BD00BD00BD2A
:10E9500000BD00000000000000000000000001CC2D
:10E9600001E202DF06BC081400A400A400A400A475
:10E9700000B300B300B300B301C801DE02CE07E468
:10E9800001DE0A840A840A960A96093E0930024882
:10E9900009EF11190E4512B6092209140DC40DF123
:10E9A0000DFF0C690CAA0D450BA6090208FB0AEE27
:10E9B0000AE30942094208500A0B093D0888085039
:10E9C000093D0A4A0A53090D0ABE0A6411EA11FCFC
:10E9D0000AC30AD30ACB0AAD0AB21384129E0152AB
:10E9E00001680265064207A407C3109E46DC4ADDA3
:10E9F00048200758DE10ECC5ADCBE6802BF54FA6BE
:10EA0000A4398D2534C0DE1248ECC633CBEF623515
:10EA1000C08D0E20EF326286F22010326286F62020
:10EA200002868997A30F3B2006868597A3973BEC28
:10EA300081D362DDD2DED2A6C484E097CF888097EE
:10EA4000CEA6C48407E61DD0A33406A6C48418103D
:10EA5000270095EC41D3661F03ECC4DD3CA661267C
:10EA60000C8605A7E4EC42DD3E4F5F2053313A4F60
:10EA70005FED2133442007ECC4ED211700ECEC27B7
:10EA8000934210A3C12505C6379D2406E321ED2737
:10EA90006A6126E3A6E42710810225102716810467
:10EAA0002506ECC4DD3E200FEC272004EC27584956
:10EAB000312C200CCC0005ED211700AEEC213126C5
:10EAC0000DCE26183406DC3CD33110934024521F5F
:10EAD00003350610A3422249E3C42040D33C0D3B3A
:10EAE0002638E32131262034A6E48104EC41250AAE
:10EAF000D3661F03EC42DD3EECC40D3B27E4D3316B
:10EB00001F030DCE26181093402416DC3E10A3429E
:10EB10002504EC42DD3EEEC42004D3311F034F3503
:10EB200086C6389D240633802006EC81D3311F032E
:10EB3000E6C44F313AED218601A7A439338120067E
:10EB4000EC81D3311F03ECC4313AED218601A7A437
:10EB5000394F5FA321ED2139EC27E3213126ED2147
:10EB600039EC27A3213126ED2139EC2727351083F5
:10EB700000022604EC21200CEC21270A108300025D
:10EB80002608EC275849ED272019A6283DA723A6DB
:10EB900028E728E6213DEB23A627E727E6223DEBE1
:10EBA00027E7273126398D24EC23ED21396FA4EC9A
:10EBB000272A0840508200ED2763A4EC212A084050
:10EBC000508200ED2163A410830002398DDF260EF0
:10EBD000EC2727174756ED27CC0000592037EC21AA
:10EBE0002605C62D9D2406EC2726053126ED233962
:10EBF0004D26081E89ED27C6082002C610E7234FC0
:10EC00005F682869275949A3212B046C282002E357
:10EC1000216A2326ECED296DA42A0E40508200EDD6
:10EC200029EC2740508200ED27312639313AE68021
:10EC30008602EDA4EC81ED22EC81ED2439EC81D348
:10EC4000311F03313A8602E6C4EDA4EC41ED22EC1B
:10EC500043ED2439A6258801A72539E625C801E713
:10EC60002534106D2227106D282610EC21ED27EC9D
:10EC700023ED29A625A72B31263590A627A02128EC
:10EC8000042AE820F22B06811F2F0A20EA81E12DB9
:10EC9000DAE621E727E62BC401E7A4E825C401E76B
:10ECA00021E62BC4FEE72BE625C4FEE7254D2731E0
:10ECB0002A274030268D7B6D21272EA3241E01E2BA
:10ECC00023A222243843531E014353C300011E01D3
:10ECD0002403C300016AA4202430A48D55AF22ED83
:10ECE00024AE28EC2A6D2126D2E3241E01E923A9B3
:10ECF00022240A46561E0146566C271E014D2B1033
:10ED00006A27102900841E0158491E0159492AF01A
:10ED10001E01C300011E012408C300012403466C28
:10ED200027ED281F10C4FE6DA427015CED2A3126B3
:10ED30003590801025198008250797144FE602208A
:10ED4000068B089714EC028E00000D14261D398BDB
:10ED500008240E97144FE602AE030D14260F1E0171
:10ED6000398B089714EC02AE0420021E0144561E93
:10ED70000146560A1426F4398D062501399D2406CC
:10ED80003410A6222A04A6282B0C4F5FED27ED296C
:10ED9000A72B31263590A621AB2728072AEC53C68E
:10EDA000323590A727E62BE825C401E7A4A62B84DB
:10EDB000FEA72BE625C4FEE7253DA7E26FE26FE242
:10EDC000A62BE6243DE361ED6124026CE4A62AE66D
:10EDD000253DE361ED6124026CE4AEE4AF616FE4D4
:10EDE000A62BE6233DE361ED6124026CE4A62AE64E
:10EDF000243DE361ED6124026CE4A629E6253DE3B0
:10EE000061ED6124026CE4E662AEE4AF616FE4A6FA
:10EE10002BE6223DE361ED6124026CE4A62AE623A1
:10EE20003DE361ED6124026CE4A629E6243DE36143
:10EE3000ED6124026CE4A628E6253DE361ED612442
:10EE4000026CE4E662AEE4AF616FE4E72BA62AE66B
:10EE5000223DE361ED6124026CE4A629E6233DE353
:10EE600061ED6124026CE4A628E6243DE361ED61D6
:10EE700024026CE4E662AEE4AF616FE4E72AA629FF
:10EE8000E6223DE361ED6124026CE4A628E6233D21
:10EE9000E361ED6124026CE4A628E6223DE3E42B65
:10EEA0000C682B692A696259496A272919ED28A635
:10EEB00062E62AC3000124136C2926116C28260D52
:10EEC00066286C272807326316FED1C4FEEAA4ED3B
:10EED0002A312632635F35908D062501399D24063F
:10EEE00053C62D6D2227F534106D281027FE9BA6E2
:10EEF00027A0211029FEA5A7278621E625E82BC4F7
:10EF000001EDA46422662366246625EC28AE2A441B
:10EF1000561E0146566F2B20021E01A3241E0124FB
:10EF200003830001A322272F2B291A016AA4277427
:10EF3000692B692A692969281E0158491E01594906
:10EF400024D71E01E3241E012403C30001E322276A
:10EF5000062AD71CFE20D5308426CFE6A45AC0103E
:10EF60002D17C0082D08E7A4A62BC6802029CB08A2
:10EF7000E7A4CC8000AE2A2020CB082D0AE7A4AE5F
:10EF800029A62BC6802012CB07E7A4AE28EC2A1AAC
:10EF90000159491E0159491E011CFE6AA42AF21E8C
:10EFA000014D2004AE2AEC282B0E1E0159491E01EA
:10EFB00059496A271029FDD21E01C300011E0124F0
:10EFC0000CC300012407466C271029FDCFED281F34
:10EFD00010C4FEEA21ED2A6C271029FDBF31265FFF
:10EFE00035903410EC2727F5AE21260F3126CC01C1
:10EFF00080ED216F236F246F253590ED21AF27EC35
:10F0000029AE23ED23AF29A62BE625A725E72B352F
:10F010001017043817FD611604EAEC81D3311F0381
:10F02000E6C44F313AED218603A7A439E628E4224D
:10F03000200AE628EA222004E628E8223126ED21EB
:10F04000396322393430AE2110AE27109F48A6A074
:10F05000A180260481FF26F64C6C1FA11F35B08DC0
:10F06000E3254E20508DDD2348204A8DD7274220AE
:10F07000448DD1263C203E8DCB243620388DC522B0
:10F08000302032EC27A3212D28202AEC27A3212F82
:10F09000202022EC27A3212618201AEC27A32127C1
:10F0A000102012EC27A3212C08200AEC27A3212FE3
:10F0B00004C6FF20015F4F3126ED218603A7A43946
:10F0C000E628E12227EB20EDE628E12226E320E5F1
:10F0D0008D222DDD20DF8D1C2FD720D98D1626D136
:10F0E00020D38D1027CB20CD8D0A2CC520C78D04B1
:10F0F0002EBF20C134201CF0A6282610A622270AE5
:10F10000A625840126041CF01A0835A0A62226068E
:10F11000A62B880120ECA62BA825840126E2332605
:10F12000A625840127021E32EC4110A32126DBEC28
:10F130004310A3232606A645A12527CE25C81CF0EB
:10F1400035A05FD73EDE48313AEF21109F4411933E
:10F1500044241AA680A7C081FF270B5A26F00A3E36
:10F160002AEC86FFA7C0DF488604A7A439C62F9DD6
:10F170002406EC81D3661F03ECC4D331EE42DF3E9C
:10F180001F033410D63F26020A3E30C48DB7359097
:10F19000EE213126A6C0A75E81FF26F8335FDF4847
:10F1A00039DC3E313AED23EF218605A7A4394F5FC4
:10F1B000ED24EC212607E7238602A7A439CE02100E
:10F1C0004D2A07405082006C254D2605CE02081EB0
:10F1D000894D2B06335F58492AFAED22EFA43931C5
:10F1E000268DCB313A39E6212E0F2B09A6222A058E
:10F1F000CC000120474F5F204BC010223A2612EC72
:10F20000226625243F10838000262C6D242A352079
:10F2100026C1F8220E3404EC22ED236F223504CBF4
:10F220000827096422662366245C26F7EC226D24F5
:10F230002A0AC300012805C6349D24066625240435
:10F2400040508200ED218601A7A43931268D9731E7
:10F250003A39312C8D90313439A62584FEA72539D1
:10F26000EC212A0640508200ED21394FE6B801ED2D
:10F270002139A6222710A6258401260DC601200BC0
:10F28000EC212B0526F65F2002C6FF1D2007D6368F
:10F290000F364F313AED218601A7A439D67D20F2F1
:10F2A000E62557102509BFC61FD76EEC2127EC4C69
:10F2B00047A721EC22250A4456ED3CEC2446562073
:10F2C00004ED3CEC24ED3E4F5FED22ED24ED3AEDF4
:10F2D0003820101A0169256924692369220A6E27DA
:10F2E000448D57E63CC040E73CEC3AE225A224EDD1
:10F2F0003AEC38E223A222ED382AD81CFE692569AF
:10F3000024692369220A6E271C8D2FE63CCBC0E7B7
:10F310003CEC3AE925A924ED3AEC38E923A922EDA1
:10F32000382BD820AEEC2220066A211029FA5B681F
:10F3300025692459492AF2ED22398D00683F693E3A
:10F34000693D693C693B693A693969383933343414
:10F3500020ECA1EDC111A3E426F73262315417FB72
:10F36000778D0617FA1216F8F2A6212E094F5FEDD7
:10F3700021ED23E72539811F24FB3326E65FC401F5
:10F38000344433213341800824FA270CC6FF584CFB
:10F3900026FCE4C4E7C020043341A7C011A36126C2
:10F3A000F93544EA25E72539313AEC27ED2116F7FE
:10F3B000B9313AEC2AED24EC28ED22EC26EDA41626
:10F3C000F9B6DC80DE823446EC21DD80DD82DD486A
:10F3D0003126C60917CCD13546DD80DF82102508DD
:10F3E000853917F615313AEF218601A7A430013986
:10F3F0000102050117F603313A81042408338CF029
:10F40000E6C64F2002DC3EED2120DECC00FF2003CB
:10F41000CC0000313AED218603A7A4396321632291
:10F4200039EC21A427E428200EEC21A827E8282085
:10F4300006EC21AA27EA28ED27312639FFDE5BD822
:10F44000AA8D09338CF617F7FA16F92C3410E62535
:10F450005710250811EC211027080B3402C601E7CC
:10F460002131A8E630A81B33A41703FD1704F54F7C
:10F470005FEDA814EDA816A7A818308D049EAFA8BC
:10F480001917012530A81433A81B1703DC1704EE45
:10F4900031A81AC602E7A4E625CA01E72535048D7E
:10F4A0000A351016F7BB00B17217F81D2A015084F7
:10F4B000013406338CF017F78AE625A6618101270F
:10F4C0003B3DE725E624A724A6613DEB248900E720
:10F4D00024E623A723A6613DEB238900E723E62248
:10F4E000A722A6613DEB228900270D6C21445666B8
:10F4F00023662466254D26F3E722E625C4FEEAE4CA
:10F50000E72535863410E6212716C1072F09E625A1
:10F510005656C8801600A5C1E4102FFAD15D2A0AFC
:10F520006FE2E625C4012745203186713DAB21E617
:10F5300025C4013406E825E725E6E417FF6D17F733
:10F540001AE6212F08EBE4E7E4E62120EE35063445
:10F55000025D271940A7E4EA25E725338DFF471709
:10F56000F6E117F6FC6AE4E625C40126EE31A8E6CA
:10F5700030A81B33A8141702F01703E8CC1000EDD5
:10F58000A44FED22A724308D0374AFA8198D1A3033
:10F59000A433A81B1702D21703E431A81A3504EBD1
:10F5A0002129198602EDA435908601979A308D04A1
:10F5B0005B9F953089005F9F97160278313A102A39
:10F5C000F7C8C6329D240634108D32EC2110270175
:10F5D00060108301802E0C260DEC232606A6251034
:10F5E0002700CB16068017008231A8EC30A815330F
:10F5F000A417027517036D30A81B1600E1E625C499
:10F6000001D76DE825E72539338C4034508DEEEC79
:10F610002110270099108301802EC82618EC23267C
:10F62000C2A62526BE966D26055FED2135D0312672
:10F63000355016016E8D3431A8EC30A81B33A41759
:10F64000022717031F30A815160093A6258501274A
:10F6500014DE316D412708338C0C17F5E6200317B3
:10F66000014116F5FC3908B4000000966D340231F2
:10F67000A8EECC0201ED2C86805FED2E4FEDA81098
:10F68000ECA812EDA4ED26ECA814ED22ED28ECA8D0
:10F6900016ED24ED2A17F6E017F5C017FC02350227
:10F6A000976D39341017FF55E621C1182D09312601
:10F6B0001700F06A21205331A8E6CC1000EDA44FCA
:10F6C000ED22A724E6A81B200B67A466216622660C
:10F6D0002366245AC1022EF1E7A81B30A81B332A47
:10F6E00017018617027E4F5FEDA814EDA816A7A894
:10F6F00018308D01D4AFA81917012C30A81433A8E5
:10F700001B17016517027731A81AA6259A6DA72540
:10F71000DE316D41271B338D008417F52617F6580F
:10F72000200F3410170082302A8D0CA625989CA734
:10F73000258602A7A4359033A81B17012C17023E7B
:10F7400031A814308D02C0332117011D16F629345B
:10F75000108D5630A48DE0A625989B20D234108DB4
:10F7600048302A33A81B17010017021230A431A811
:10F770001433211700F3170205EC21260E3126CC95
:10F780007FFFED2186FFED234A200517F74AA625C6
:10F79000989B209902C90FDAA2FB8EFA351206E572
:10F7A0002EE0D4338CEE16F49ADE316D4127093306
:10F7B0008CE717F48E17F5C00F9BE625C401D79C84
:10F7C000E825E7258DDD6C2117F9292D0717FB7D2D
:10F7D0008DD120026A2117F91B2D0D0C9B969C8858
:10F7E00001979C17F4758DBB6A2117F9072F1396A3
:10F7F0009B8801979B6C21A62B8A01A72B17F4618C
:10F80000313A31A8EC308D00C7AFA81930A81B33AE
:10F81000A8148D5517014DCC1000EDA44FED22A773
:10F8200024ED2AED2CA72E308D019B9F9530884129
:10F830009F970F9AC625D7990F9D33A81B9E959C1D
:10F840009724088D2430059F952004C6018D6C30C7
:10F85000A433258D260D9A2606302A332F8D1CAD14
:10F86000B8190C9D0A9926D2393430A68410AE01FD
:10F87000AE03A7C410AF41AF4335B0E6841DD69D9B
:10F8800054545424015C34042705A7C05A26FBC6EF
:10F8900005E0E02707A680A7C05A26F9335BD69D6E
:10F8A000C4072724C1042513C008A68448694469F5
:10F8B000436942694169C45C26F23967C46641669E
:10F8C00042664366445A26F339A62AA8A443200375
:10F8D000A6A8144D2A1430A4332F8D50302A332576
:10F8E0008D6630A81433A81B204230A4332F8D58C6
:10F8F000302A33258D3630A81433A81B204A30A86F
:10F900001433A81B8D422B24260CEC012608EC0393
:10F910002604C601D79930A43325201030A43325FE
:10F920008D0A8120242230A81433A81BEC03E34362
:10F93000ED03EC012407C3000124026C84E341EDD4
:10F9400001A684A9C4A78439EC03A343ED03EC0109
:10F95000240783000124026A84A341ED01A684A246
:10F96000C4A78439E6C46FC4CB042C0F5016FF4BD8
:10F97000684469436942694169C45A26F339A6C497
:10F980002A094F5FEDC4ED42A74439CC20045A68E0
:10F990004469436942694169C42B074A26F05FED17
:10F9A000C439A6C4E7C4E641A741A642E742E643FC
:10F9B000C30001C4FEED43240C6C4226086C4126B2
:10F9C0000466416CC4390C90FDAA22076B19C1581A
:10F9D00003EB6EBF2601FD5BA9AB00FFAADDB900FA
:10F9E0007FF556EF003FFEAAB7001FFFD556000F68
:10F9F000FFFAAB0007FFFF550003FFFFEB0001FF1D
:10FA0000FFFD0001000000009B74EDA80B17217F93
:10FA10007E067CC8FB300391FEF8F301E27076E3CA
:10FA200000F8518601007E0A6C3A003F8151620065
:10FA30001FE02A6B000FF805510007FE00AA000323
:10FA4000FF80150001FFE0030000FFF80000007FC9
:10FA5000FE0000003FFF8000001FFFE000000FFFDE
:10FA6000F8000007FFFE00000400000E1214A2BB05
:10FA700040E62D361962E94F5FDD4CDD4E3402A6BB
:10FA8000222716E625C501260463E4200CCBFEEBF5
:10FA900021A624DD52EC22DD509653D6573DDD4E93
:10FAA0009652D6573DD34D24020C4CDD4D9653D67D
:10FAB000563DD34D24020C4CDD4D9651D6573DD3C7
:10FAC0004CDD4C9652D6563DD34CDD4C9653D65514
:10FAD0003DD34CDD4C9650D6573DDB4CD74C965120
:10FAE000D6563DDB4CD74C9652D6553DDB4CD74CC9
:10FAF0009653D6543DDB4CD74CDC4ED35ADD52DC0A
:10FB00004CD9599958DD506DE0262ADC50ED22DCA5
:10FB100052ED246F21861F3402EC222B0E6AE4275B
:10FB20000A6A216825692459492AF2ED22E625C48A
:10FB3000FEE7253584DC52C4FEEDA3DC50EDA34F77
:10FB40005FEDA38DD016F230DC48EE21A3218300B7
:10FB500001DF48ED218601A7A439EC21DD48E6B894
:10FB6000014F20EFEC214D102600FBDE48EF21E78E
:10FB7000C0170115109F441193441024F5EF39EC80
:10FB8000212F0EE3271F0310934824028D7F312677
:10FB9000393126EE212076EC212FF63410DC48A3F3
:10FBA0002183000110A327230E1F01EE27A680A7A3
:10FBB000C081FF26F8DF4831263590EC212F04EC78
:10FBC000272E08EC213126ED2120B483000127F3F4
:10FBD000E32D1093482504312620B634101F01E68A
:10FBE00022EE2DA680A7C081FF270B5A26F56A2199
:10FBF0002AF186FFA7C0DF48312C3590DE48335FFD
:10FC000011A3212708A6C2812027F5334186FFA72B
:10FC1000C0DF48393430DC48A321E327C30001AEFC
:10FC20002710AE218D0624074F5F200C9D1B081F57
:10FC300020AE62A301C300013530ED278601A7265F
:10FC4000312639C6022002C603967DDE8234521761
:10FC5000C45625129E8286FFA784AE6317F4E3354F
:10FC600052977DDF8239C6439D24063410EC212D46
:10FC7000F5109F44DE48EF218620D17D230DA7C0DB
:10FC80005A11934425F416F4E4341086FFA7C0DF1C
:10FC9000488604A7A435903410313A303ADE48EF54
:10FCA00021103F1525E5A680C62F816425068064B6
:10FCB00024FC8B648D1C862F8D12862F8D0E862042
:10FCC0008D0A863A8D06863A8D0220BFA7C0A6808F
:10FCD000C62F5C800A24FBE7C0C63A5A4C26FCE7D4
:10FCE000C039A622C606103F8D2408C1D32604C6FB
:10FCF000FF20015F4FED218603A7A439C6063434E7
:10FD00001FB8C6501F02308DFD61EC81EDA16AE481
:10FD100026F8308DEC489F10308DECC29F12867E05
:10FD20009716308DECC49F17308C049F1935B49D05
:10FD30001B1A3416E6F804308C08EC85308BAF645F
:10FD4000359600B4000A9D270C9D270E3496583036
:10FD50008C08EC85308BAF643596045F05C305C312
:10FD600004B705B305AA044A0258026B023502A281
:10FD7000027F05F905E904780A1005DA06BA05627A
:10FD800007580602271003E80064000A04A00000D8
:10FD90000007C80000000AFA0000000E9C400000A6
:10FDA00011C350000014F424000018989680001B22
:10FDB000BEBC20001EEE6B2800229502F90025BA79
:10FDC00043B74028E8D4A5102C9184E72A2FB5E644
:10FDD00020F432E35FA932368E1BC9C039B1A2BC10
:10FDE0002E3CDE0B6B3A408AC7230454727565FFC4
:10FDF00046616C7365FF3440313A4F5F9775977673
:10FE0000977797789779ED24ED22A7211702292477
:10FE100009301F812C266F16008981241027013A92
:10FE2000812B2706812D26040C78A680812E26089A
:10FE30000D7726520C7720F217064A255034020C13
:10FE400076EC24EE228D2CED24EF228D268D24E3FA
:10FE5000241E03E923A92225271E03EBE0890024A1
:10FE6000063341EF22271BED24EF220D7727BB0C31
:10FE70007920B758491E0359491E032501393262BA
:10FE80003261C63C2002C63BD7364335C088458424
:10FE9000DF2723301F0D76260220EB0D772645EC59
:10FEA000222641EC242B3D0D78270440508200EDA2
:10FEB000218601160087A684812B2706812D260422
:10FEC0000C7530011705BC25BD1F891705B5240425
:10FED000301F20073402860A3DEBE00D75260150E5
:10FEE000DB79D779C620E721EC22260910A3242646
:10FEF000046F2120464D2B0A6A216825692459493F
:10FF00002AF6ED220F75D67927292A03500C75C1E0
:10FF1000132310C0133404338DFECB8D263504100B
:10FF200025FF5F5A86053D338DFE6133C58D141064
:10FF300025FF4FA62584FE9A78A7258602A7A41C34
:10FF4000FE35C0313AECC4ED21EC42ED23E644E746
:10FF50002596751027EF8916EE26170526241081A1
:10FF600061250280208141251B8146221780370CA4
:10FF700076C604682269211025FF075A26F5AB22B0
:10FF8000A72220D6301F0D761027FEFA16FF223446
:10FF9000109E8217FE60240235908102270317FD10
:10FFA000A81700882507C63DD7364335909F824F56
:10FFB000359034109E8217FE3D25DD810126136D9C
:10FFC0002127DE200D34109E8217FE2A25CA8101CA
:10FFD00027CFC63AD7364335903450313ADE4AEF10
:10FFE000218604A7A49E82A6808D532504A7C02045
:10FFF000F69F8286FFA7C0DF484F35D03410313AD4
:020000041001E9
:100000008603A7A46F229E828D2E251B8154271163
:100010008174270D884684DF2709C63AD7364335D1
:100020009063228D0724FC9F824F3590A68081200B
:10003000260C8D0424172017A680812027FA91DD35
:10004000270D810D270781FF27031CFE39301F1A5A
:10005000013934504FA723977697788604977EEC22
:10006000212A06405082000C78338DFD150F7A331B
:1000700042A3C425040C7A20F8E3C40D7A26046D4B
:1000800023270B6C233402967A17010635020A7E69
:1000900026DB1F981700FB312635D034500F750F23
:1000A000780F7C0F7B0F790F763384CC0A30E7C052
:1000B0004A26FBEC2126044C1600D1E625C5012773
:1000C00006D778C4FEE725EC212A030C754081038E
:1000D000232DC69A3D4412121F890D75270150D752
:1000E000798113230D3402338DFCFB17FE55350245
:1000F0008013338DFC964AC6053D33CB17FE44EC86
:10010000226D2127262A10445666246625067C6C1B
:100110002126F4ED222014682569245949097B6AB7
:100120002126F4ED220C79967B8D67EC22EE240FCC
:100130007B8D66ED22EF243402967B977C35028D11
:10014000588D561E03E3241E03E923A92234029688
:100150007B997C8D3D967681093502270C108300B2
:100160000026CC1183000026C6A7A4967681092517
:1001700019E6A42A15A6824CA7848139230C86305F
:10018000A784ACE426EF6C840C7986099776312637
:1001900035D08A30A7800C76391E0358491E035982
:1001A00049097B3934309E809F828601977D108E6D
:1001B0000100967F103F8B20133430DC8293802720
:1001C0000F1F029E809F82967F103F8C2402D7369D
:1001D00035B03450A6A481022704EE212007A621C1
:1001E0002E08CE00008E0000201CAE22EE248020BF
:1001F0002505C64E4320161E1044561E0346561EA5
:10020000011E134C26F1967F103F882402D7363505
:10021000D03450327630E417FE813410860930092C
:10022000E682C13026054A810126F597763510D63B
:10023000792E21501F98C1092234DB76C109222E64
:1002400034021700A64F8D7235045D270317008C0A
:1002500096762013C10922161700901F988D4A8D9B
:10026000599676907923028D40326A4F35D08D7B36
:1002700086018D358D4496764A26014C8D2B8D0254
:1002800020E786458D3696794A34022A0660E48D49
:100290005E20028D5E35044FC00A25034C20F9CB49
:1002A0000A8D021F988B3020131F895D2707A680B7
:1002B0008D0A5A26F93986202002862E344233E8E8
:1002C000C0119382220C810D27088650973697DE45
:1002D00035C2DE82A7C0DF820C7D35C286305D2745
:1002E000058DD95A26FB390D7827CB0D7827F7864F
:1002F0002D20C9862B20C5862020E38DBFA68081B6
:10030000FF26F8393410AE218DF34F35903410307C
:100310008DFAD8A62226F1308DFAD520EB34503252
:100320007B30E417FD2C8DC3967630E417FF7A32CC
:10033000654F35D01F893440DE82D07D23028DB7D2
:100340004F35C017FF70967D840F8101270C17FF72
:100350006520F3860D0F7D17FF624F393440860408
:1003600033A46DC4260347334197861F895717016D
:100370009335C05FD787813C270C813E26035C20E4
:1003800005815E26055AD787A680812C273881FFF4
:10039000261296942704301F20159E8E0DDC270808
:1003A0000FDC2022812927031A0139969427F90AA4
:1003B000922611DE4637229792109F90DF46A68044
:1003C0000A9420C69E909F8C1CFE394900DE48008E
:1003D000DB5200CE4500CB5300D24200CF54000A7E
:1003E00058001227001A008DA12563D68617FF46F4
:1003F00020288D962558D68617FEFC201D81FF27C4
:100400004D81272608A6808D812543200D17FEAC3F
:10041000A68020E934300FDC0CDC9E8C8D4B251936
:100420008128262E9692D79227280C94DE46109E7D
:10043000903622DF469F90A680318C8F5F3402A8D1
:10044000A484DF3502271231235C6DA426EFC63F5A
:100450002002C63ED7364335B0D785EC2131AB8D6F
:10046000082402C601D7866EA48D1825271F898D02
:1004700012251C8D208D0C25168D1A4D27015FA687
:1004800080200CA6808130250B8139220580301C0C
:10049000FE391A01393402860A3DEBE089003981C0
:1004A0002E26AB8DC425A7D78917FEC725A03530CA
:1004B0000CDCD685102700A25A27125A10270150AB
:1004C0005A102701F25A102700FB1600DE9D1681F4
:1004D000042510EE215FA6C081FF27035C26F7EEFE
:1004E0002120213321A6A481022604C605201581DE
:1004F000012606C602D1862504C60133411F98484D
:10050000918622360D8727282B0D3404583404D6C3
:1005100086E0E02519200C3404583404D686E0E047
:10052000250C5734049686A0E0978617FDC935043C
:10053000A6C4444444448D12270EA6C08D0C27083F
:100540005A26EDD68617FDAF4F39840F8109230255
:100550008B0717FD500A863943399D168102250500
:1005600026F617F7E13450327B30E417FAE4D686EA
:100570005AD0762A07326535501601320D87270A80
:100580002B1917FD7217FD5F201717FD5A340496BB
:100590007617FD15350417FD5E200B17FD4917FD75
:1005A0003B967617FD0332654F35D09D16810326A5
:1005B000A73450308DF834C604A622261C308DF89E
:1005C0002FC60520149D168104268D3450AE21DCE3
:1005D00048A3218300014D2604D1862302D6861F1D
:1005E0009850DB860D87270E2B10340217FD083537
:1005F0000217FCB520173404200B5424015C340688
:1006000017FCF4350217FCA1350417FCEA4F35D06E
:100610009D16810227071024FF3E17F72C34503215
:100620007630E417FA75967981092E111700E29653
:100630008680022B0890892B04908A2A06326A351C
:1006400050206B978830E4D68727082B0C8D418D7E
:1006500014200D8D108D3920078D358D0B17FC87DB
:10066000326A4F35D017FC7F968A17FC3C17FC4A3C
:10067000D6792A2C50D1892302D689340417FC5C00
:10068000D689E0E0D789968B91892302968920123A
:10069000D68816FC6217FC4F968A17FC0C17FC1ABA
:1006A000968B17FC04D689D08B2F0B16FC2ED68682
:1006B000862A17FC294F399D16810227071024FE30
:1006C0009717F6853450327630E417F9CE967934A0
:1006D00002860197798D3A3502D679C10127014CFE
:1006E000C601D78A9779968680062B0890892B04B5
:1006F000908A2A06326A355020B49788D68727090F
:100700008D8E8D9117FB7B20058D8A17FB7416FF4C
:100710004F341096799B892606A684813524174A82
:100720002B308107222C3086E601C13525246C84CC
:10073000E684C139231CC630E784301FACE424EEC4
:10074000AEE43008A682A701ACE422F88631A78483
:100750000C79351096792A014F978A408B092A0126
:100760004F918923029689978B39C630D736433902
:100770006C8F270000000000000100000301000052
:100780000F0100000C01000006010000090100003B
:100790008806012016FF01001400A08042A642B680
:1007A00000502098CC1842BF42AF0048208801007A
:1007B000EBB88878A09808780058208842A842AF03
:1007C000E3A0886006005250D3F0754224810020D7
:1007D00006005250E182887F2C8100200600525092
:1007E000ABB360533C81002006005250BBFF3CB6C7
:1007F0004481002006005250861C03024C810020D8
:10080000060052505422A29D5881002005005250EB
:10081000DE65F468340B0110000000000000F03FBA
:1008200000000000000024400000000000005940CB
:100830000000000000408F40000000000088C3401E
:1008400000000000006AF8400000000080842E4193
:1008500000000000D01263410000000084D79741DF
:100860000000000065CDCD410D0A00000000000031
:10087000F142002000000000F5420020014300206A
:100880002D43002029430020000000000A00000042
:1008900000000306A6000800020002009C001400ED
:1008A000030057494E55534200000000000000006D
:1008B000000080000400010028004400650076006C
:1008C00069006300650049006E00740065007200F5
:1008D0006600610063006500470055004900440060
:1008E00000004E007B0062006300370033003900D7
:1008F0003800630031002D003700330063006400CE
:100900002D0034006300620037002D0039003800EC
:10091000620038002D0039003100330061003800DA
:1009200066006300610037006200660036007D00EB
:1009300000000000050F2100011C100500DF60DD34
:10094000D88945C74C9CD2659D9E648A9F00000350
:1009500006A60001000000000600525053B4F4A1A6
:100960007C8100200000000090810020A0810020F8
:10097000F03F0220A8810020B48100200902540029
:10098000030100807D080B00020202000009040040
:1009900000010202000405240020010524010001D9
:1009A000042402060524060001070581030800103F
:1009B00009040100020A00000007050202400000CD
:1009C000070582024000000904020000FF00010543
:1009D00012011002EF0201408A2E090000010102FB
:1009E0000301000000000000395C0020A95C002029
:1009F000D55C0020215D0020DD5D00209D5E002093
:100A00000000000000000000995F0020F55F00205A
:100A100011600020356000208543002039610020EE
:100A200000000000100000000000000000000100B5
:100A300000000000000000000000020000000000B4
:100A400000000000000003000000000000000000A3
:100A50000000FF000000000001B5486801318E462B
:100A60000047704609380149884701BDB912002086
:100A70000000000000000000000000000000000076
:100A800000000000F00A012041450020ED44002054
:100A900065440020D5430020000000000001000054
:100AA0009C37012010000C00000000000000000036
:100AB000000000000000000000000000FF00000037
:100AC0000000000000000000000000000000000026
:100AD000AD2400202124002055240020F9240020EA
:100AE0008D24002085230020D524002071230020A0
:100AF000A9130020D924002069170020D123002049
:100B0000C124002071240020850F0020AD0F00209B
:100B1000F972002081010020F50C002075480020AA
:100B2000D3DEFFFFFE010000FF01000018F6FEFF0C
:040B3000793512AB56
:040000051000014D99
:00000001FF
